:100000000C94C20E0C94EA0E0C94EA0E0C94EA0EB8
:100010000C94EA0E0C94EA0E0C94EA0E0C94EA0E80
:100020000C94EA0E0C94EA0E0C94EA0E0C94DA6C22
:100030000C9470700C94076D0C94EA0E0C940C19CF
:100040000C94FA180C94EA0E0C94A4750C940E748B
:100050000C94EA0E0C94EA0E0C94EA0E0C94EA0E40
:100060000C9430700C946A190C94726D0C943F6E61
:100070000C94EA0E0C94EA0E0C94EA0E0C94EA0E20
:100080000C94EA0E0C94EA0E0C94EA0E3072347260
:100090003C7246725D7277728C729B72B072C772DC
:1000A000D172EF72F572FA720073067360736A733D
:1000B0000F7315731B73247328732D733573477374
:1000C0004D7353735873387238733D734273537062
:1000D0006C617368008040000000000000000000B8
:1000E0000000000000000000000000000000000010
:1000F0000000000000000000000000000000000000
:1001000000000000000000000000000000000000EF
:1001100000000000000000000000000000000000DF
:10012000000080C0E0E0F0F8F8FCFCFCF8F8F8F023
:1001300040000000000080808000000000000000FF
:1001400000000000000000000000000080C0C0E0CF
:10015000E0E0F0F0F0E0C00000000000C0F8FFFFB9
:100160009F8783838383838383838383838383833F
:1001700083838383838383830383808383838383D2
:10018000838383838383838383838383838383833F
:100190008383C3E3733F1F0000000080E0F0F8FC9E
:1001A000FEFFFFFFFF7F3F1F1F0F0783C3E1E1E05B
:1001B000E0C0000E1F3F7F7FFFF3E0E08000000003
:1001C0000000000000000080F0FCFEFFFFFFFF7F4A
:1001D0003F0F0301010100000080F0FEFFFFC7C1D7
:1001E000C1C1C1C1C1C1C1C1C1C1C1C1C1C1C1C1FF
:1001F000C1C1C1C1C101C1F0FEFF3F0F070F0D0D0D
:100200000D1D191919193131313171616161E1C166
:10021000C1C18100000080E0F8FCFFFFFFFF2F1745
:100220000F038180C0E0F0F8FCFEFFFFFFFFFFFF3F
:100230007F010000000000000001010307070E1EFF
:100240001C3870E0F0F8FEFFFF7F1F0F0300010075
:10025000000000000000000000000000000000009E
:10026000000000000000000000000000000000008E
:10027000000000000000000000000000000000007E
:10028000000000000000000000000000000000006E
:1002900000000000007EFFFFFFFFFFFFFBF8FCFCFB
:1002A000FEFF7F3F1F0F07C3FFFFFFFFFFFF7F071B
:1002B0000000000000000000000000000000C0E09E
:1002C000F8FEFFFF7F1F0F1F3D7CF8F8F0E0800075
:1002D000000000000000000000000000000000001E
:1002E000000000000000000000000000000000000E
:1002F00000000000000000000000000000000000FE
:1003000000000000000000000000000000000000ED
:1003100000000000000000010101010103070707C0
:100320000301000000E0FCFFFFFFFFFF1F030000D0
:10033000000000000000000000C0F078DE27130974
:100340000E0703000000000000000001030F7FFF04
:10035000FC7878F800000000000000000000008039
:10036000808080808080808000808000808000008D
:1003700000000000008080808080808080808080FD
:1003800080808080808080000000000000000000ED
:10039000000000000000000000000000000000005D
:1003A000000080F0FEFFFFFFFF3F0F010000000094
:1003B00000000000C0E0381E0F0300010000000034
:1003C000000000000000000000000000000000002D
:1003D0000000030301000000000000000000000E08
:1003E0000E02020202020303000F0F000F0F0808A3
:1003F00008080808080F0F08080808080F0F000071
:1004000000000F0F000000000000000000000000CE
:1004100000000000000000000000000000000000DC
:10042000C0F8BFFFFFFF1F7F0100000000000000B9
:1004300000F0FCFF7F7830000000000000000000AA
:1004400000000000000000000000000000000000AC
:10045000000000000000000000000000000000009C
:10046000000000000000000000000000000000008C
:10047000000000000000000000000000000000007C
:10048000000000000000000000000000000000006C
:100490000000000000000000000000000000301C10
:1004A000070E0F0701000000000000000000000020
:1004B000000000000000000000000000000000003C
:1004C000000000000000000000000000000000002C
:1004D00000000000000000001B1E272D36394B4E87
:1004E000636C7278878D939CB1B4C6C9D2D8E1E4AD
:1004F00001020304010302040402030104030201D4
:1005000003010200040506076D656E75537461638F
:100510006B206F766572666C6F77006D656E7553D4
:100520007461636B20756E646572666C6F770070C2
:100530007265737320616E79204B657900414C457B
:100540005254004D455353414745004C4F41444997
:100550004E47002020202020202020202020202066
:1005600020202020202020202000506C6561736511
:1005700020526573657420537769746368657300EE
:100580005377697463686573205761726E696E672B
:1005900000204F6C642056657273696F6E2045456C
:1005A00050524F4D202020434845434B2053455443
:1005B00054494E47532F43414C494200416C6172AC
:1005C0006D732044697361626C6564005265736584
:1005D00074207468726F74746C65005468726F7400
:1005E000746C65206E6F742069646C650050726570
:1005F000737320616E79206B657920746F20736B43
:10060000697000414C45525400454550524F4D20B1
:100610006C6F77206D656D004F46464142535255D1
:1006200073525525454C73454C2554487354482501
:10063000414C73414C2550312050312550322050CF
:1006400032255033205033250054485252554445EA
:100650004C4549443049443149443241494C47456D
:100660004154524E535731535732535733535734E3
:1006700053573553573653573753573853573953C2
:100680005741535742535743004F4646004F4E2061
:10069000002D2D2D004348002D2D2D2000525544B6
:1006A00020454C45205448522041494C20005031AF
:1006B000202050322020503320204D4158204655D4
:1006C0004C4C4359433143594332435943335050BF
:1006D0004D3150504D3250504D3350504D3450509C
:1006E0004D3550504D3650504D3750504D38434891
:1006F0003120434832204348332043483420434884
:100700003520434836204348372043483820434863
:10071000392043483130434831314348313243482E
:10072000313343483134434831354348313641440D
:10073000312041443220002D2D2D2D00564552539D
:100740003A2056312E353439362D6572657A00449B
:100750004154453A2031312E30322E323031320080
:1007600054494D453A2031303A31303A3233002045
:1007700053564E3A20657239782D72373038002042
:100780004D4F443A204652534B59204E542020009E
:1007900012081200081C0808081C080000082200A3
:1007A000490022080000000000227F22000000080B
:1007B0002200490022080000082200490022080007
:1007C0000000227F220000000000082200490022D1
:1007D000080000081C0808081C08001236C34BA7B4
:1007E0004A96307E29E35CC559F750A552E621C3ED
:1007F000204A53191F39246F240F258A264E4F2073
:10080000444154410054783D0052783D0041203D20
:100810000056343D0756353D0E56363D0056313DA7
:100820000756323D0E56333D005370643D096B74DC
:1008300073204D61783D00416C743D004C6F6E3DFE
:10084000004C61743D0054783D0052783D004132C7
:100850003D0041313D00416C743D0052504D3D0022
:1008600054323D0054313D0054783D0052783D00F3
:100870004675656C3D0041203D0054546D0045783F
:1008800070457846466E654D656443727300544FFB
:10089000540053544B1153542500544D4511545397
:1008A000570053544154005B4D454E555D20746FC5
:1008B000207265667265736800537461636B0F62C2
:1008C00000746D61696E0F6D7300746D7231204A32
:1008D00069747465720F757300746D72314C617454
:1008E000206D696E0F757300746D72314C617420E8
:1008F0006D61780F7573005354415432004D6F642D
:1009000065005761726E31205761726E3220436804
:100910006561702052696E672020536369466920C3
:10092000526F626F74204368697270205461646111
:100930002020437269636B74536972656E20416C49
:100940006D436C6B5261746174615469636B2020F8
:1009500048617074633148617074633248617074C7
:10096000633300416C657274205B5265645D0041C5
:100970006C657274205B4F72675D00416C657274C8
:10098000205B59656C5D00496E742E204672736B56
:100990007920616C61726D0042616E644761700024
:1009A000506F745363726F6C6C00416C61726D2098
:1009B0005761726E696E67004D656D6F7279205771
:1009C00061726E696E6700545245303132414700A2
:1009D00054524530313241470044656661756C744C
:1009E00020537700537769746368205761726E698A
:1009F0006E67005468726F74746C65205761726E14
:100A0000696E670053706C617368204E616D65009C
:100A100053706C6173682073637265656E004F4636
:100A200046004C69676874206F6E2053746B204DCC
:100A300076004C69676874206F666620616674652D
:100A400072004C6967687420737769746368004644
:100A50006C617368206F6E20626565700042656529
:100A60007020636F756E74646F776E004D696E757C
:100A700074652062656570005468726F74746C658B
:100A800020726576657273650053494E474F534D2A
:100A90005046494C540046696C7465722041444389
:100AA00000496E616374697669747920616C617262
:100AB0006D0042617474657279207761726E696E3F
:100AC0006700436F6E74726173740048617074697B
:100AD0006320537472656E67746800537065616B50
:100AE0006572205069746368004265657065725074
:100AF0006953706B7200536F756E64204D6F64653F
:100B0000005175696574204E6F4B65792078536884
:100B10006F727453686F7274204E6F726D20204C28
:100B20006F6E672020784C6F6E672000426565709D
:100B30006572004F776E6572204E616D650052419F
:100B400044494F2053455455500043616C004D7546
:100B50006C7469706C6965720063683163683263D4
:100B60006833636834006F6666202B3D203A3D0091
:100B70006D6F64650A2520737263202073770053BC
:100B80006C61766500545241494E455200000303A2
:100B900003030056455253494F4E005472696D2D60
:100BA000202B00204D656E75204578697420446FB8
:100BB000776E20202055705269676874204C6566F6
:100BC00074004449414700424700414E41005B4D9B
:100BD000454E555D205748454E20444F4E45004DEB
:100BE0004F564520535449434B532F504F545300B5
:100BF000534554204D4944504F494E54005B4D4598
:100C00004E555D20544F205354415254005354418B
:100C100052542043414C4942524154494F4E0043A3
:100C2000414C4942524154494F4E0066726565003D
:100C30004D4F44454C53454C00434F4C2044697242
:100C4000656374696F6E0041494C20446972656345
:100C500074696F6E00454C45204469726563746920
:100C60006F6E0053776173682052696E6700436F3F
:100C70006C6C656374697665002D2D2D2020203104
:100C800032302020203132305820203134302020A2
:100C90002039302020202000537761736820547958
:100CA00070650048454C4920534554555000004458
:100CB000454C455445204D4F44454C0F5B4D454EEA
:100CC000555D00543254685472696700547261690A
:100CD0006E657200452E204C696D69747300504F2B
:100CE000534E45470053686966742053656C004C49
:100CF00050342F4C5035202044534D326F6E6C7958
:100D00002044534D322F44534D580044534D2054EA
:100D10007970650053656E64205278204E756D625F
:100D20006572205B4D454E555D0050504D2046721A
:100D30004C656E0D6D536563002052784E756D00E5
:100D40003443482036434820384348203130434814
:100D500031324348313443483136434800755300FB
:100D6000755365630050504D202020505858202066
:100D70002044534D32202050504D313620005072C7
:100D80006F746F00524554413132330042656570D3
:100D900020436E74005472696D205377004578705B
:100DA000202020457846696E6546696E6520204D95
:100DB000656469756D436F61727365005472696D26
:100DC00020496E6300542D4578706F00542D547285
:100DD000696D00436F756E7420446F776E436F7555
:100DE0006E7420557020200054696D657220005487
:100DF0007269676765720054696D6572004E616D56
:100E000065005345545550000009010000000000E2
:100E1000000602004475706C69636174696E672036
:100E20006D6F64656C005B4D454E555D20205B45E4
:100E30005849545D005945530B4E4F0044454C45AD
:100E40005445204D4F44454C004455504C49434176
:100E50005445204D4F44454C0020414243444546B3
:100E60004748494A4B4C4D4E4F505152535455569A
:100E70005758595A6162636465666768696A6B6C42
:100E80006D6E6F707172737475767778797A3031B0
:100E900032333435363738395F2D2E00657870207F
:100EA0002025202073773120737732004558504F2A
:100EB0002F4452000003445220486967680044529E
:100EC000204C6F77004452204D6964004472537780
:100ED0003200447253773100576569676874004582
:100EE00078706F004558504F2F445200002B2A5203
:100EF000004D49584552005072657373205B455848
:100F000049545D20746F2061626F7274004D617886
:100F1000206D69786572732072656163683A20009C
:100F200044454C455445204D4958205B4D454E5550
:100F30005D00536C6F772020557000536C6F7720E5
:100F400020446F776E0044656C61792055700044D1
:100F5000656C617920446F776E00416464202020C5
:100F600020204D756C7469706C795265706C61638A
:100F70006520004D756C747078004F4646005761CF
:100F8000726E696E670053776974636800437572A7
:100F9000766573004F4E204F4646005472696D00CF
:100FA0004F46464F4E2000466C4D6F646574726923
:100FB0006D004F666673657400466D5472696D56B8
:100FC000616C0057656967687400536F757263657B
:100FD0000045444954204D49582000494E5345523C
:100FE00054204D495820002D2D2D2D202020763EB7
:100FF0006F66732020763C6F667320207C767C3E83
:101000006F66737C767C3C6F6673414E4420202073
:10101000204F522020202020584F52202020207680
:10102000313D3D7632207631213D76322076313E9B
:101030007632202076313C7632202076313E3D7665
:10104000322076313C3D76322000535700435553D1
:10105000544F4D20535749544348455300000253C1
:10106000414645545920535749544348455300007D
:1010700002566F6C742054687265733D004F46468B
:1010800031323234303000416C74416C61726D0029
:101090002D2D2D59656C4F7267526564005478523E
:1010A000535349616C726D0054454C454D45545243
:1010B000593200000101003C3E002D2D2D59656C78
:1010C0004F726752656400616C726D00762D5641F7
:1010D000004120206368616E6E656C004D65744947
:1010E0006D700046724875625753486869005573C1
:1010F0007250726F746F0054454C454D45545259AF
:101100000000010102020102434F5059205452498C
:101110004D205B4D454E555D002D2D2D494E560001
:101120004C494D49545300000303030303030303D5
:1011300003030303030303030043560043555256BE
:1011400045530050524553455400454449542D3EA3
:101150000043555256450009002D2D2D494E56008D
:101160004F46464F4E20002D2D2D783E30783C3096
:101170007C787C663E30663C307C667C63312063E4
:101180003220633320633420633520633620633795
:101190002063382063392063313063313163313269
:1011A0006331336331346331356331360045455043
:1011B000524F4D206F766572666C6F7700454550D3
:1011C000524F4D206F766572666C6F770067656E63
:1011D0007772697465206572726F7200454550526E
:1011E0004F4D20466F726D617474696E6700426185
:1011F0006420454570726F6D2044617461004D4FED
:1012000044454C2020202020004D45202020202037
:101210002020200050085000000000000000006F57
:10122000000007000700147F147F14242A7F2A126D
:10123000231308646236495522500005030000005C
:101240001C2241000041221C0014083E081408081A
:101250003E080800503000000808080808006060D8
:1012600000002010080402003E49453E0000427F75
:101270004000625149460041494936001814127F26
:101280000027454539003E494932000179050300F0
:1012900036494936000649291E000036360000004E
:1012A0005636000008142241141414141441221458
:1012B0000800020151090600060909067E0909090C
:1012C0007E7F494949363E414141227F4141221CAE
:1012D0007F494949417F090909013E4149497A7FCE
:1012E0000808087F00417F41002040413F017F08FE
:1012F0001422417F404040407F020C027F7F04085F
:10130000107F3E4141413E7F090909063E4151217E
:101310005E7F09192946264949493201017F0101A9
:101320003F4040403F1F2040201F3F4030403F6330
:101330001408146307087008076151494543007F8A
:1013400041410002040810200041417F00040201D5
:101350000204404040404000010204002054545424
:10136000787F484444383844444420384444487FD3
:101370003854545418087E0901020C5252523E7FD0
:101380000804047800447D40002040443D007F1064
:1013900028440000417F40007C041804787C080445
:1013A000047838444444387C14141408081414187D
:1013B0007C7C080404084854545420043F444020D2
:1013C0003C4040207C1C2040201C3C4020403C44B1
:1013D000281028440C5050503C4464544C4400089D
:1013E00036410000007F0000004136080008082256
:1013F0001C08081C220808A06080000000000000F3
:101400000000000000000000FFFF000000000000DE
:101410001F3F00003F1F00003030FFFF3030FFFF54
:1014200030303078CCCCFFFFCCCC8C0C060F0F8644
:10143000C0E070381C0C3CFEC7E3F33B1E0C000000
:101440000000333B1F0F000000000000F0F81C0EEE
:1014500007030000000003070E1CF8F00000303006
:10146000E0C0FCFCC0E03030C0C0C0C0FCFCC0C06C
:10147000C0C000000000000000000000C0C0C0C0EC
:10148000C0C0C0C0C0C000000000000000000000DC
:1014900000000080C0E070381C0C0000000000005C
:1014A00000000000000000003838000000000000CC
:1014B000000000000000000003033F3F03033F3F24
:1014C00003030C0C0C0C3F3F0C0C07030C0E070322
:1014D0000100183C3C180F1F383133331E1E3333C4
:1014E00000000000000000000000000003070E1CC8
:1014F00038300000000030381C0E070300000303E2
:1015000001000F0F00010303000000000F0F000097
:1015100000000000333B1F0F00000000000000002F
:101520000000000000000000183C3C180000000013
:101530000C0E07030100000000000000FCFE87C342
:10154000E377FEFC00000C0EFFFF0000000000002F
:101550000C0E0783C3E77E3C00000303C3C3C3E74D
:10156000FE3C0000C0E070381C0EFFFF00003F3F53
:1015700033333373E3C30000FCFEC7C3C3C78E0C11
:1015800000000303C3E3733B1F0F00003CFEE7C3EF
:10159000C3E7FE3C00003C7EE7C3C3E7FEFC00005F
:1015A000183C3C18000000000000183C3C180000EB
:1015B00000000000C0E0F0381C0E0703303030306F
:1015C00030303030303003070E1C38F0E0C00000FF
:1015D0000C0E07030383C3E77E3C00000F1F3B3163
:1015E00030381F0F000030303F3F30300000000027
:1015F0003C3E37333130303000003030303030391D
:101600001F0F00000303030303033F3F00000C1CF4
:10161000383030381F0F00000F1F383030391F0F9F
:10162000000000003F3F0000000000000F1F3930A5
:1016300030391F0F0000000030381C0E0703000077
:10164000060F0F06000000000000333B1F0F0000D4
:1016500000000000000103070E1C383003030303E1
:1016600003030303030330381C0E070301000000CB
:101670000000000033330100000000003C7EE7C39F
:10168000C3E77E3CF0F8DCCEC7C7CEDCF8F0FFFF46
:10169000C3C3C3C3C3E7FE3CFCFE07030303030746
:1016A0000E0CFFFF030303070E1CF8F0FFFFC3C37C
:1016B000C3C3C3C30303FFFFC3C3C3C3C3C3030382
:1016C000FCFE0703C3C3C3C7CECCFFFFC0C0C0C06E
:1016D000C0C0FFFF00000303FFFF03030000000082
:1016E00000000303FFFF0303FFFFC0E0F0381C0E00
:1016F0000703FFFF0000000000000000FFFF0E1CBA
:10170000F8F81C0EFFFFFFFF3870E0C08000FFFFFD
:10171000FCFE070303030307FEFC000000000000BB
:10172000000000003F3F0000000000003F3F3F3F3F
:101730003030303030391F0F0F1F383030303038F4
:101740001C0C3F3F303030381C0E07033F3F303019
:101750003030303030303F3F0000000000000000EB
:101760000F1F3830303030303F3F3F3F0000000027
:1017700000003F3F000030303F3F303000000C1C85
:10178000383030381F0F00003F3F000103070E1CA8
:1017900038303F3F30303030303030303F3F000065
:1017A000000000003F3F3F3F0000000103033F3FB8
:1017B0000F1F3830303030381F0FFFFFC3C3C3C393
:1017C000C3E77E3CFCFE070303030307FEFCFFFFA9
:1017D000C3C3C3C3C3E77E3C3C7EE7C3C3C3C3C725
:1017E0008E0C03030303FFFF03030303FFFF00004B
:1017F00000000000FFFFFFFF000000000000FFFFEF
:10180000FFFF000000000000FFFF0F1F38F0E0E0C6
:10181000F0381F0F3F7FE0C08080C0E07F3F0303B0
:101820000383C3E3733B1F0F0000FFFF03030303A6
:1018300000000C1C3870E0C08000000000000303B2
:101840000303FFFF000030381C0E07070E1C383062
:10185000000000000000000000003F3F000000000A
:10186000000000000F1F383033371E1C3F333F3F4E
:10187000000003070E1C38300C1C38303030303973
:101880001F0F000000003F3F000000000F1F383016
:10189000303030381F0F03070E1C38381C0E07037A
:1018A0000F1F38381F1F38381F0F3C3E0703010138
:1018B00003073E3C000000013F3F010000003C3EAA
:1018C000373331303030303000003F3F303030304F
:1018D000000000000000000103070E0C0000303083
:1018E00030303F3F0000000000000000000000001A
:1018F00030303030303030303030000003070E1CD4
:10190000383000000000303030303070E0C0FFFF71
:10191000C0E070303070E0C0C0E070303030303047
:101920000000C0E070303070E0C0FFFFC0E07030F9
:1019300030303070E0C0C0C0FCFEC7C303070E0CDF
:10194000F0F89C0C0C0C0C0CFCFCFFFFC0E07030A1
:101950003070E0C000003030F3F300000000000001
:1019600000003030F3F30000FFFF0080C0E0703073
:10197000000000000303FFFF00000000F0F03070E3
:10198000E0E07070E0C0F0F0C0E070303070E0C0B7
:10199000C0E0703030303070E0C000000000000067
:1019A000000000000C1E3F33333333333F3F3F3FD3
:1019B0003030303030381F0F0F1F38303030303873
:1019C0001C0C0F1F3830303030303F3F0F1F3B337F
:1019D00033333333030300003F3F000000000000B7
:1019E000000133333333333B1F0F3F3F0000000010
:1019F00000003F3F000030303F3F303000000C1C03
:101A0000383030381F0F00003F3F03070F1C3830BD
:101A10000000000030303F3F303000003F3F00000A
:101A2000030300003F3F3F3F0000000000003F3F36
:101A30000F1F3830303030381F0FF0F0303030307A
:101A400030F0E0C0C0E0F0303030E0C0F0F0F0F056
:101A5000C0E070303070E0C0C0E0F0303030303086
:101A600000003030FFFF303000000000F0F00000D8
:101A700000000000F0F0F0F0000000000000F0F0C6
:101A8000F0F0000000000000F0F03070E0C0808056
:101A9000C0E07030F0F0800000000000F0F0303066
:101AA000303030B0F0F070300000C0E03C3E070352
:101AB000000000000000FFFF00000000000003071E
:101AC0003E3CE0C00000C0C0C0C00C1CF8F0E0C04C
:101AD000C0E0F0F81C0CC0C0C0C03F3F03030303CC
:101AE0000303010000010303030303033F3F3F3FE0
:101AF0000000000000000000303133333333333F47
:101B00001E0C00000F1F383030381C0C0F1F3830EF
:101B100030381C0C3F3F03070E1C38381C0E0703DF
:101B20000F1F38381C1C38381F0F30381C0F0707A0
:101B30000F1C3830000133333333333B1F0F303841
:101B40003C3E373331303030000000010F1F383059
:101B50000000000000003F3F00000000000030389F
:101B60001F0F01000000000000000C0E0703010021
:101B7000000103070E0C0000000040800804201044
:101B800002010000891112239B322446AD573665AD
:101B9000BF74488CC19D5AAFD3BE6CCAE5DB7EE9E9
:101BA000F7F88110080193331A22A5562C47B77510
:101BB0003E64C99C408DDBBF52AEEDDA64CBFFF9C9
:101BC00076E802218B30100299132667AF763444F1
:101BD000BD554AADC3BC588ED19F6EEBE7FA7CC8A9
:101BE000F5D983310A2091121803A7772E66B554D0
:101BF0003C45CBBD42ACD99E508FEFFB66EAFDD889
:101C000074C904428D5316619F702004A9153227B0
:101C1000BB364CCEC5DF5EEDD7FC6888E1997AAB68
:101C2000F3BA85520C4397711E60A1142805B3378F
:101C30003A26CDDE44CFDFFD56ECE9986089FBBB48
:101C400072AA06638F7214409D512225AB34300670
:101C5000B9174EEFC7FE5CCCD5DD6AA9E3B8788A28
:101C6000F19B87730E6295501C41A3352A24B1164F
:101C70003807CFFF46EEDDDC54CDEBB962A8F99A08
:101C8000708B088481951AA793B62CC2A5D33EE128
:101C9000B7F04008C919522BDB3A644EED5F766D00
:101CA000FF7C899400859BB712A6ADD224C3BFF1F7
:101CB00036E0C1184809D33B5A2AE55E6C4FF77DE0
:101CC0007E6C0AA583B4188691972EE3A7F23CC0D8
:101CD000B5D14229CB38500AD91B666FEF7E744CC0
:101CE000FD5D8BB502A499961087AFF326E2BDD0B7
:101CF00034C1C3394A28D11A580BE77F6E6EF55CA0
:101D00007C4D0CC685D71EE597F42880A1913AA397
:101D1000B3B2444ACD5B5669DF78600CE91D722F7F
:101D2000FB3E8DD604C79FF516E4A9902081BBB376
:101D300032A2C55A4C4BD7795E68E11C680DF33F5F
:101D40007A2E0EE787F61CC495D52AA1A3B0388257
:101D5000B193466BCF7A5448DD59622DEB3C700E3F
:101D6000F91F8FF706E69DD414C5ABB122A0B99236
:101D70003083C77B4E6AD5585C49E33D6A2CF11E1F
:101D8000780F891B11241FBECFEFD0E1DEBFCDBF7E
:101D900011E0A0E0B1E0E0E3F0EF02C005900D92A9
:101DA000AA32B107D9F71FE0AAE2B1E001C01D9243
:101DB000A233B107E1F71DE1C4E8DDE104C02297D9
:101DC000FE010E94D177C238D107C9F70E94B41A28
:101DD0000C9416780C94000030919D0422B78091E9
:101DE0009D043817C9F7932F80E030E0282B392B5A
:101DF000C901089529E282029001112435952795A1
:101E00003595279587FD815C86FB880F880B80F9C7
:101E1000992787FD9095281B390BC9010895F894DF
:101E20002091CE0D3091CF0D7894C9010895482F9F
:101E300050E09A01220F331F63E0440F551F6A954B
:101E4000E1F7240F351F2C553E4FC901089590E04E
:101E50009C01220F331F220F331F280F391F2C51D3
:101E60003D4FC9010895AF92BF92CF92DF92EF929A
:101E7000FF920F931F93CF93DF93C82E162FEA0183
:101E8000F22ED02E57FF10C022FF02C08CE101C0FD
:101E90008FE09C2D981B892F612F4DE22F2D0E94E2
:101EA0004965D095C195DF4F2D2D2F218C2D612FA8
:101EB0004AE30E9449658F2D90E0B4E0AB2EB12C2F
:101EC000A822B922F2FE02C0E2E001C0E0E0CE01A9
:101ED0006CE370E00E947F779B01442737FD4095BB
:101EE000542F0F2D00618E2F8C0D612FA2E0EA2E52
:101EF0000E944967A114B10411F0ECE101C0E1E1D5
:101F0000CE016CE370E00E947F779C01442737FD8F
:101F10004095542F0D2D00618E2F8C0D612FF2E016
:101F2000EF2E0E944967DF91CF911F910F91FF9093
:101F3000EF90DF90CF90BF90AF9008950F931F93D5
:101F4000062F122F206250E00E947F6817FD07C005
:101F50008091A00D602F46E7212F0E9449651F91B7
:101F60000F910895242F409108010E949E0F08951B
:101F70000F93022F442319F447E357E020C0453064
:101F8000A8F4E0916E01F0E0EE0FFF1FEE0FFF1FCF
:101F90003197E40FF11DE051FB4F449150E0440FA5
:101FA000551F440F551F4756594F09C0473250F42B
:101FB00050E0440F551F440F551F4656594F24E01B
:101FC0000E940C660F910895FF920F931F93182F94
:101FD000F62E022F442321F448E956E024E00EC0F7
:101FE0008A5E4A3008F485506F2D50E0202F0E9401
:101FF0007F68812F6F2D45E956E022E00E940C6634
:102000001F910F91FF9008950F931F93DF93CF932C
:1020100000D0CDB7DEB7382F162F942F022F4423D0
:1020200029F0463139F04A3E81F408C08A5F41E91F
:1020300056E007C08A5F4DE856E003C08A5F49E872
:1020400056E0202F0E943C6628C04095441F44273C
:10205000441F81E2841B482F832F39839A830E9477
:1020600049653981832F8A5F9A81E92FFF27E7FD30
:10207000F095F7FF03C0F095E195FF4FFF27E7FDCF
:10208000F0953197AF01440F551F4E0F5F1F475B0F
:10209000594F612F23E00E940C660F900F90CF9153
:1020A000DF911F910F91089589E496E00895DF92E2
:1020B000EF92FF920F931F93D82EE62EF42E1091DD
:1020C0009501E12FFF27E7FDF095F7FF03C0F0959D
:1020D000E195FF4FE031A4F483E0E802F001112420
:1020E000E85EF94F8D2D6E2DAF0123E00F2D0E947C
:1020F0000C661F3F3CF58D2D86506E2D41E21FC0B2
:102100008D2D8650E53264F411161CF4412F4F508A
:1021100002C0412F415F6E2D2F2D0E94041012C06E
:1021200011161CF4412F445202C0412F4C5D6E2DFC
:102130002F2D0E9404108D2D8E5E6E2D4DE62F2DBD
:102140000E9449651F910F91FF90EF90DF900895D5
:10215000CF92DF92EF92FF920F931F93CF93DF9373
:10216000F82ED62EE22F102F242F30E040E050E042
:10217000F0E0DF01AA0FBB1FAA0FBB1FA65DBB4F7C
:102180000C910295069506950370CC24C3940230F9
:1021900009F0CC24EE2071F1EE0FFF1FEE0FFF1FB0
:1021A000E95DFB4F8081C82FD0E0CC2011F0CC0F2F
:1021B000DD1FBE0180E090E00E944077033051F1C6
:1021C000C436D10580F49B01AC01CA01B901660F88
:1021D000771F881F991F23E330E040E050E00E9402
:1021E000927710631FC02FEF30E040E050E00E9474
:1021F000927718C0CC2021F0220F331F441F551FA7
:10220000033081F4CA01B9012FEF30E040E050E023
:102210000E94407724E630E040E050E00E94927750
:10222000106202C0002311F0CC2091F0012F006257
:102230008F2D6D2D75E0E72E0E94496717FD0EC0AA
:102240008091A00D6D2D46E7212F0E94496506C0A3
:102250008F2D6D2DA901212F0E947F68DF91CF91D5
:102260001F910F91FF90EF90DF90CF9008958C30E9
:1022700038F4E82FF0E0EE0FFF1FE952FB4F2AC0C1
:10228000803198F4E82FF0E0DF01AA0FBB1FAC58B3
:10229000BB4FEE0FFF1FEC5BFE4F2D913C91119752
:1022A00080819181281B390B0AC0843158F4E82FB2
:1022B000F0E0EE0FFF1FEC58FB4F20813181220F21
:1022C000331F1AC0843248F4E82FF0E0EE0FFF1FEE
:1022D000E354FB4F208131810FC0863258F4E82F40
:1022E000F0E0EE0FFF1FEE0FFF1FE55FF14F2081C3
:1022F00030E002C020E030E0C9010895AF92BF9203
:10230000CF92DF92EF92FF920F931F93DF93CF93C1
:102310000F92CDB7DEB7F82EE42E463008F0EAC0B3
:10232000882309F4EAC0863119F08A3E19F4E2C024
:1023300061E0E3C0992787FD90959C0197FF04C059
:1023400022273327281B390B2A307CF41F144CF02A
:102350002DE030E0A901481B590BCA010E94E96930
:10236000C6C00D960E94E969C7C02A50A22EBB24A0
:102370009501220F331F2A0D3B1D26573E4FF901B1
:10238000E85AFD4F4081442309F4B4C05E2D553016
:1023900029F4F501E859FB4F8081A7C0F901EA5AF9
:1023A000FD4FC080295A3D4FF901D080453008F4D7
:1023B000B1C04830C8F08C2D815049830E9437113C
:1023C0008C018D2D81500E9437110BC02D2D33278C
:1023D00027FD309523583F4F0BC08D2D49830E9418
:1023E000FA0E9C01498104C020E030E000E010E0DA
:1023F000483088F4453080F5423009F460C04330FD
:1024000020F4413009F06CC055C04330C9F044306D
:1024100009F066C01BC04A3009F44CC04B3030F4A0
:102420004830F1F1493009F05BC03FC04C3009F44D
:102430004BC04C3008F443C04D3009F051C049C086
:1024400017FF38C0109501951F4F34C017FF37C0D4
:10245000109501951F4F33C0E3948C2D60E04E2DF5
:102460000E947E11082F8D2D60E04E2D0E947E115E
:10247000F501EE0FFF1FEA0DFB1DEE51FC4F9081A1
:10248000953029F4002361F1882341F52AC0963064
:1024900029F4002319F5882319F120C0802721C0D1
:1024A00081E002171307E1F41CC081E00217130753
:1024B000C1F416C081E0201731079CF011C081E003
:1024C0000217130774F00CC081E0021713074CF4D5
:1024D00007C081E02017310724F402C081E001C069
:1024E00080E0F501E859FB4F80831F142CF061E078
:1024F000682703C060E001C0682F862F0F90CF913E
:10250000DF911F910F91FF90EF90DF90CF90BF90E0
:10251000AF9008958C2D815049830E9437118C0112
:102520004981FC2DF5320CF051CF57CF86B3809501
:102530008E7708950E9496128823E1F70E945869C9
:10254000089580915B0160E040E00E947E11882345
:1025500031F48091850490918604009711F0C79A18
:102560000895C79808950F931F93CF93DF93EC01BD
:102570008B010E94DF6482E260E043E056E024E0E9
:102580000E943C6680E2BE010E94636688E2B80158
:102590000E94636680E36DEE75E00E9463660E94B0
:1025A000E968809158010E94DF680E949A12DF91C9
:1025B000CF911F910F9108950F93AB0160E123E03C
:1025C00000E00E940C660F910895DF92EF92FF9257
:1025D0000F931F93CF93DF9380916D0181FD83C093
:1025E00080E895E06AE675E00E94B312909185015B
:1025F000892F887341F0883131F0883221F080339F
:1026000011F0883329F4892F877C886080938501B5
:1026100000E010E085E1E82EF12C08C0C701801B26
:1026200091090E94E969110F182B0F5F0830B0F370
:10263000D0908501D12680E060E143E555E026E1B8
:1026400000E00E940C66CD2DD0E0CE0180FF05C0D9
:1026500082E069E476E00E94DC12C1FF05C087E1F8
:102660006CE476E00E94DC12C2FF05C08CE26FE4ED
:1026700076E00E94DC12CE01887390700097B1F072
:10268000012F13FF05C081E462E576E00E94DC12B1
:1026900004FF05C081E465E576E00E94DC1205FFD9
:1026A00005C081E468E576E00E94DC12C6FF05C043
:1026B00086E56BE576E00E94DC12D7FE05C08BE66E
:1026C0006EE576E00E94DC120E94E9688091850147
:1026D000181749F00E949612882329F40E94A1122B
:1026E00000E010E09BCFDF91CF911F910F91FF9001
:1026F000EF90DF9008951F93CF93DF930E9496127F
:1027000020E030E011E0482F50E02F5F3F4FBA014A
:10271000022E02C0759567950A94E2F760FD03C02A
:102720001F5F183091F71150163030F5812F0E943D
:10273000535F882309F110935701812F0E94575F3F
:1027400081E00E942D600E94DF6486E160E04BE43E
:1027500055E024E00E943C66CAE8D1E01AE04991C5
:10276000812F68E124E00E944965155F1837B9F7A9
:102770000E94E9680E949A12DF91CF911F910895FB
:10278000CF93DF93EC010E94DF6482E260E043E4D8
:1027900055E024E00E943C6688E1BE010E94636629
:1027A0000E94E968809158010E94DF68DF91CF9113
:1027B00008951F93CF93DF93EC01162F0E94DF64DF
:1027C00082E260E04DE355E024E00E943C6688E14F
:1027D000BE010E9463668CE168E34FE255E00E940F
:1027E0006B660E94E968112319F48091580101C0B9
:1027F00089E10E94DF6882E10E9484730E949A123C
:102800000E9496128823C9F48091620E833019F4D5
:10281000A8951092620E80915B0160E040E00E94FA
:102820007E11882331F480917201882311F41123E1
:1028300011F0C79AE5CFC798E3CFDF91CF911F91F1
:10284000089580916704882351F081E995E060E064
:102850000E94D913809167048E7F80936704089546
:1028600080916D0187FD07C0887329F48CEB95E09A
:1028700060E00E94D913089580916D0182FD0AC025
:102880000E944E61883C910528F489E096E060E062
:102890000E94D9130895EF92FF92CF93DF93A82F50
:1028A000AF70A65090919C01923074F0292F33277D
:1028B00027FD309521503040C1E0D0E002C0CC0F60
:1028C000DD1F2A95E2F79C2FA83008F09CC06A2FE4
:1028D000659570E0FB01EE0FFF1FE050FF4F019088
:1028E000F081E02DB081992379F4CB2FDD27C7FD4E
:1028F000D095D7FF03C0D095C195DF4F9C2FC7FD62
:102900009D5F959595959F5F40916E0150E0417058
:10291000507022E030E0241B350B2617370769F48E
:1029200020919B012F7009F473C021E094E0309155
:10293000700130FF03C0919501C020E04B2F552757
:1029400047FD5095C92FDD27C7FDD095A0FF03C0D7
:10295000C40FD51F04C0BA016C1B7D0BEB0120977F
:1029600029F07E019F2D9B2797FF0BC0222349F45E
:10297000BB2339F010820E94486A86E10E9484736A
:1029800041C0CE0184589F4F893F9105B8F4C08360
:1029900086E00E942D60CE0183589F4F8B3F9105AA
:1029A00088F5D7FF03C0D095C195DF4FD595C79562
:1029B000D595C795BE01645C462F1FC01C161D0629
:1029C00014F48DE701C083E8808386E00E942D60C7
:1029D000CE0183589F4F8B3F9105A0F4CE01D7FFC6
:1029E00003C0909581959F4F64E070E00E947F77CF
:1029F000709561957F4F462F445C8FE294E065E1CE
:102A00000E94117280E0DF91CF91FF90EF900895C6
:102A100020E08DCF8F929F92AF92BF92CF92DF92A4
:102A2000EF92FF920F931F93CF93DF93182FEB0139
:102A30005A016901802E84FF06C01F70106654E0A1
:102A4000952E05E003C045E0942E04E0802F8066BB
:102A5000181761F0802F8064181741F080910605E7
:102A6000882369F0133611F0133449F47E01089479
:102A7000E11CF11C83E10E948473892D18C0992DFB
:102A80009066191761F0992D9064191741F0882309
:102A900009F474C0123619F0123409F06FC07E01C7
:102AA0000894E108F10884E10E948473802F90E08B
:102AB0000E94E969882351F0EE24FF24EC1AFD0AF4
:102AC000892D0E94486A802F0E94486AA114B1048F
:102AD00091F481E0C816D10471F4103661F41092BB
:102AE000060531E0E32EF12C209711F0EE24FF24AF
:102AF00080E60E94486A2091820430918304E21AA1
:102B0000F30ACE14DF0444F4812F0E94486A83E163
:102B10000E94847376010AC0EA14FB043CF4812FFE
:102B20000E94486A84E10E9484737501EC16FD06D8
:102B3000A9F0E114F10451F4812F0E94396AD7FF02
:102B400002C083E101C084E10E948473882D8370F8
:102B50000E942D6081E080937F0402C010927F0468
:102B6000C701DF91CF911F910F91FF90EF90DF9000
:102B7000CF90BF90AF909F908F9008957E01A6CF89
:102B80000F93772767FD7095552747FD509533279D
:102B900027FD30950E940A150F9108950F9377270E
:102BA00067FD7095552747FD5095332727FD3095D4
:102BB00002E00E940A150F9108950F93772767FD91
:102BC0007095552747FD5095332727FD309501E037
:102BD0000E940A150F910895E0917E04F0E0EE0F37
:102BE000FF1FEA58FB4F80819181089590917E04E8
:102BF000992319F4882331F418C0882319F4892FF4
:102C0000815001C080E080937E0487E10E9484733C
:102C1000E0917E04F0E0EE0FFF1FEC58FB4F0190B7
:102C2000F081E02D8EEB099508958BE195E060E051
:102C30000E94D9130895FC01A0917E04B0E0AA0F70
:102C4000BB1FAC58BB4FED93FC938FEB099587E10D
:102C50000E9484730895CF93DF93EC0180917E04EA
:102C6000982F9F5F90937E04953040F080937E0470
:102C700088E095E060E00E94D9130FC087E10E94D0
:102C80008473E0917E04F0E0EE0FFF1FEC58FB4FE1
:102C9000D183C0838FEBFE010995DF91CF91089519
:102CA0008FE294E00E941071882311F084E105C046
:102CB00080919E04882321F0815080939E0407C058
:102CC0009091630081E091FF80E080939F04809168
:102CD0009F0408951092890410928B0410928A0424
:102CE000109288040895209185043091860421155E
:102CF000310531F021503040309386042093850413
:102D0000882369F04091720150E084EF91E0489F80
:102D10009001499F300D589F300D112402C020E0D2
:102D200030E080918704882369F060917A0170E037
:102D300044EF51E0649FC001659F900D749F900D1A
:102D4000112402C080E090E04091850450918604F7
:102D50004217530720F43093860420938504209172
:102D60008504309186042817390720F4909386044F
:102D7000809385040E94A1120895E82FF0E0E050AE
:102D8000FB4FE491F0E0EE0FFF1FEE55FB4F20816B
:102D90003181C9010895CF92DF92EF92FF920F9394
:102DA0001F93DF93CF930F92CDB7DEB720E0CC24F3
:102DB000DD24822F29830E94BD16092F10E0C00E4A
:102DC000D11E29812F5F2430A1F7C6010F90CF912A
:102DD000DF911F910F91FF90EF90DF90CF900895BA
:102DE0001F930E940F0F41E02091D5043091D6042B
:102DF0008217930709F440E0409384040E940F0F68
:102E00009093D6048093D5048BE095E060E00E9417
:102E1000543A80918404882309F4CBC080918804BB
:102E200080FF14C080918904982F9F5F909389043C
:102E3000943660F083568093890480918A0490913F
:102E40008B04019690938B0480938A0480E00E9407
:102E50003B600E94DF640E945B690E944B14182F44
:102E60000E9473162091E3043091E4048091800461
:102E700090918104821B930B60E270E00E947F7747
:102E800070938304609382046115710591F08091C1
:102E9000D3049091D404821B930B62E070E00E94F3
:102EA0007F7770938304609382043093810420932E
:102EB00080043093D4042093D3048091700185FF63
:102EC00004C01092830410928204E0917E04F0E02A
:102ED000EE0FFF1FEC58FB4F0190F081E02D812F8A
:102EE00009950E94E9680E945016882321F080917C
:102EF00065008F7E03C080916500806180936500CE
:102F00000E940F0F8F7190708230910509F04FC0B1
:102F100087E00E94BD169C0164E0220F331F6A9572
:102F2000E1F768E070E00E947F7740915A015527F1
:102F300047FD50954A5F5F4F649FC001659F900DAC
:102F4000749F900D1124820F931F2091700126FD14
:102F500005C06091090170910A0102C060EF70E044
:102F60002091080130E02F5F3F4F0E946B77260FC2
:102F7000371F35952795209308018091D204805EF4
:102F80008093D204882399F480915901281778F40A
:102F9000223368F081E10E9484738091700183FF85
:102FA00006C082E390E0909386048093850410929B
:102FB00087041F910895A2EAB4E0E2EBF4E060E038
:102FC000862F806487B9369A408951898D919C916A
:102FD000119796958795840F951F8E7F11969C93D8
:102FE0008E9320813181C901840F951F9695879515
:102FF000918B808B349BFECF349A84B195B1820F34
:10300000931F96958795819391936F5F1296683081
:10301000B9F60895EF92FF920F931F93CF93DF932A
:103020008091700184FD44C00E94A1120E94DF645F
:1030300080E060E045ED50E020E000E00E94EA64BE
:103040008091760184FD08C080E068E34BE751E0A1
:103050002AE000E10E940C660E94E9688091580114
:103060000E94DF680E949A1200E20E94DB17015062
:10307000E1F70E94CB168C010E940F0FEC01C057A4
:10308000DE4F0DC00E94DB170E94CB167C010E9410
:103090009612882369F4E016F10651F406C00E94E6
:1030A0000F0FC817D90771F703C00E94A112F7CFFD
:1030B000DF91CF911F910F91FF90EF900895E2EA79
:1030C000F4E040E012C067B9369A349BFECF349AE0
:1030D00024B135B1820F931F5150A9F7969587956A
:1030E000819391934F5F483031F054E080E090E05D
:1030F000642F6064E8CF0895E2EAF4E020E0822FD4
:10310000806487B9369A349BFECF349A84B195B1E6
:10311000880F991F819391932F5F283081F708952D
:10312000FF920F931F93CF93DF9380916D0180FDEA
:103130003AC080916E0190E08170907002E010E0E2
:10314000081B190BF801EE0FFF1FE65DFE4FC18152
:10315000D281609687859089C81BD90B0E947C1804
:10316000F02E802F0E94BD16C817D907E4F40E94E4
:1031700096128823C1F40DC00E947C188F2D0E94E6
:10318000BD16C817D9077CF40E949612882341F017
:103190000AC08BED95E06CEC75E00E94B312ECCFA9
:1031A0000E94A112E9CFDF91CF911F910F91FF9063
:1031B00008958EE587B9369A349BFECF349A84B150
:1031C00095B104964091090150910A019A0163E07A
:1031D000220F331F6A95E1F7241B350B820F931FD3
:1031E00023E0969587952A95E1F790930A018093BD
:1031F0000901089578941F920F920FB60F9211242F
:103200008F9380919D048F5F80939D048F910F9089
:103210000FBE0F901F90189578941F920F920FB6C3
:103220000F9211242F933F934F935F936F937F934C
:103230008F939F93AF93BF93EF93FF93F89487B7C8
:103240008D7F87BF789481B78E5F81BF9091310465
:1032500080913304882379F080917901882349F0A3
:10326000813051F48091310F890F8093310F87FFA6
:1032700002C01B9A01C01B9880910B01982F91509E
:1032800090930B01882381F48DE480930B018FE2EE
:1032900094E00E9424710E94596A0E946176809194
:1032A000620E82608093620EF89487B7826087BF57
:1032B0007894FF91EF91BF91AF919F918F917F9102
:1032C0006F915F914F913F912F910F900FBE0F9093
:1032D0001F90189578941F920F920FB60F92112499
:1032E0001F932F933F934F935F936F937F938F938E
:1032F0009F93AF93BF93EF93FF9320918000309102
:103300008100F89480917D008F7D80937D0078947A
:103310008091A0049091A104A901481B590BCA01F6
:10332000969587953093A1042093A00410919C0456
:10333000212F2150283058F59C012152334055E06F
:103340002737350708F5E12FF0E0EE0FFF1FE657AE
:10335000FB4FAC014C5D554020917401332727FD94
:103360003095265F3F4F429FC001439F900D529F73
:10337000900D11246AE070E00E947F777183608372
:103380001F5F10939C040CC010929C0409C0815ACA
:103390009F402EE28F3D920718F481E080939C04B9
:1033A000F89480917D00806280937D007894FF91F5
:1033B000EF91BF91AF919F918F917F916F915F91AD
:1033C0004F913F912F911F910F900FBE0F901F9023
:1033D0001895E3E3FFE09F0181918535E1F32253E6
:1033E0003F40C9010895EF92FF920F931F93CF932F
:1033F000DF930E94EC0EEC0180917101813019F491
:103400000E94DB1707C0823019F40E945F1802C0C7
:103410000E947C188EE587B90E94F0160E94D91888
:103420008091620E833019F4A8951092620E0E946A
:10343000EC0E8C1B9D0B2091AD063091AE0628172B
:10344000390720F49093AE068093AD0680919A0ED2
:10345000882309F482C010929A0E8091990E8823D5
:1034600099F180919601829586958695837090E07A
:103470000097C1F08230910519F420E931E002C0D3
:103480002AE730E08091AF069091B0064091EB0EB4
:103490005091EC0E840F951F281739071CF481E01A
:1034A0000E94847320912A0F90910404EEE1FFE0C2
:1034B00080E008C03191391720F48DE10E948473B7
:1034C00003C08F5F8217B0F38091980E882309F4B0
:1034D00044C080E060E00E943A748C018330910522
:1034E00039F180E061E00E943A74EC01833091058B
:1034F00021F181E060E00E943A747C018330910503
:1035000011F181E061E00E943A748330910509F184
:103510000230110569F0C230D10579F022E0E216DF
:10352000F10489F082309105A1F00130110511F408
:1035300080E00AC0C130D10511F480E00BC021E069
:10354000E216F10419F481E060E005C081309105D4
:1035500021F481E061E00E949074DF91CF911F918E
:103560000F91FF90EF9008951F938FEF8ABB1BBAC6
:1035700091E897BB9EE798BB9EE394BB91EC95BB0B
:1035800011BA82BB88E082B987EF83B910926100DB
:103590001092620084E1809364008BEF8093650059
:1035A0000E94A9680E942E7680E487B985E886B9D2
:1035B00087E083BF8CE981BF87B7836087BF1FBC6B
:1035C0008AE08EBD10928B0082E880938A00809101
:1035D0007D00806280937D00EDB7FEB7329785E570
:1035E00002C0808331979FE0E233F90709F0C8F702
:1035F000789482E394E4909375048093740489E151
:103600000E94DF680E94E65F109157010E947B13C1
:10361000809158010E94DF685091720140917A01B7
:10362000451778F4652F70E024EF31E0629FC00108
:10363000639F900D729F900D112490938604809348
:103640008504541770F450E024EF31E0429FC0012C
:10365000439F900D529F900D112490938604809368
:1036600085040E94A11280917901813039F4809102
:10367000700184FD03C087E00E9484730E940A18D1
:103680000E943C140E947C180E9490180E94E5122F
:103690000E9430140E9421140E949A1280EF90E040
:1036A00090930A01809309010E947B6F2DE088E1CD
:1036B00090E00FB6F894A89581BD0FBE21BD8BE0B8
:1036C00095E060E00E94543A82E196E30E942B1656
:1036D00081E00E94F615809158010E94DF68809178
:1036E0005701181729F081E00E942D600E94C960DF
:1036F00080912C0F806480932C0F80ED97E09BBD10
:103700008ABD80E186BF87B7806187BF0E94F319B9
:10371000FDCF8FE294E00E940D71089529E28202AC
:1037200090011124359527953595279587FD815C66
:1037300086FB880F880B80F9992787FD9095281BB9
:10374000390BC90108959C01E5E035952795EA9567
:10375000E1F7AC01440F452F441F550B280F391FCB
:10376000892F990F990B8595280F391F241B350B2D
:10377000C9010895F8942091CE0D3091CF0D789421
:10378000C9010895AC0180E060E021E00E943C6640
:1037900008950F931F93CF93DF93182F82EA98E039
:1037A0000E94C21B113658F0133628F0133639F434
:1037B00084E69CE102C082E394E40E941B1686E04A
:1037C00068E04AE958E00E946B66409125065091F6
:1037D00026068AE268E020E000E00E94330F409174
:1037E0002706509128068EE468E020E00E94330FFF
:1037F00086E060E142E958E00E946B66409129064C
:1038000050912A068AE260E120E00E94330F409145
:103810002B0650912C06F4E056954795FA95E1F762
:103820008EE460E120E00E94330F86E660E04EE81F
:1038300058E00E946B6640912306509124068EE466
:1038400060E020E00E94330F8091A9069091AA06C3
:103850008937910528F08091A806C82FD0E002C0D2
:10386000C0E0D0E082E06CE34EE70E94E96685E0CC
:103870006CE143E20E94ED661BE0812F6BE343E0C5
:103880000E94ED661A5F1338C1F716E00CE3FE01E3
:10389000E05DF94F4081602F641B812F0E94ED662F
:1038A0002196C837D10510F0C0E0D0E02091A806DD
:1038B00030E0C217D30719F01F5F1E3741F7DF91C1
:1038C000CF911F910F9108951F93182F87EF98E0C4
:1038D0000E94C21B1236E1F0133628F4103631F084
:1038E0001136E9F418C01336D1F415C08FEF97E004
:1038F00090930D0180930C011092AC061092AB06D0
:103900001092AE061092AD0687E10E94847307C044
:1039100089EC9BE102C082E394E40E941B1688E0DC
:1039200068EE78E00E9463664091AB065091AC0669
:103930005695479584E568E00E948F6880E169EDBF
:1039400078E00E94636640910C0150910D015695FC
:10395000479584E560E10E948F6888E16AEC78E031
:103960000E9463664091AB065091AC0680910C01B9
:1039700090910D01481B590B5695479584E568E1D8
:103980000E948F6880E261EC78E00E94636620917B
:10399000AD063091AE0684E690E0289FA001299FF5
:1039A000500D389F500D1124A4E056954795AA95C7
:1039B000E1F784E560E220E30E947F6888E269EB3A
:1039C00078E00E9463660E94E919AC018FE368E227
:1039D0000E946F6682E168E347EA58E00E946B66E6
:1039E0001F91089587E691E108950F9393E0499F11
:1039F000A0011124405A5E4E01E0222309F400E0A8
:103A000023E00E940C660F9108950F9393E0499F65
:103A1000A0011124475A5E4E01E0222309F400E080
:103A200023E00E940C660F910895FF920F931F935D
:103A3000F82E062F142F80E860E0402F50E0212F51
:103A40000E947F680A3010F00FE601C005E7802F62
:103A500060E04FE2212F0E9449654F2D50E04F5FFB
:103A60005F4F802F60E0212F0E947F681F910F9190
:103A7000FF9008956F927F928F929F92AF92CF9214
:103A8000DF92EF92FF920F931F93CF93DF93EC019E
:103A9000162FD42E49016090DF047090E0048091CD
:103AA000BF089091C0088619970920E430E0B90159
:103AB0000E947F77462F60930905E091E104F09121
:103AC000E2048091BD089091BE088E1B9F0BB90146
:103AD0000E947F77862F60930A05442321F070921D
:103AE000C0086092BF08882321F0F093BE08E093DD
:103AF000BD0880910805882321F48091700185FF1D
:103B000006C01092090510920A05109208056091EE
:103B10000905662351F480910A05882331F48091C8
:103B2000820490918304009781F04091720150E0EB
:103B300024EF31E0429FC001439F900D529F900DB2
:103B4000112490938604809385048114910409F4D0
:103B500056C08881882309F04BC0662331F18091DB
:103B60000605882311F5ED2DE61BE7FDE0E0202F8B
:103B700030E08E2F992787FD90958217930714F0D8
:103B8000E02FE150FF27E7FDF0958D2D90E0E8173D
:103B9000F90749F0EE0FFF1FE80DF91D259134914B
:103BA000C9010E941B1610920905153641F4DD204B
:103BB00011F0ED2D01C0E02FF0E031970FC0143669
:103BC000C9F42D2D30E0802F90E001972817390798
:103BD0001CF4ED2DEF5F01C0E0E0F0E0EE0FFF1F01
:103BE000E80DF91D25913491C9010E941B1602C0F0
:103BF00040E001C041E08D2D602F0E94151DE114B1
:103C0000F10451F098818C2D9C1508F4892FF7014F
:103C1000E80FF11D549101C050E080910605882302
:103C200009F04FC080910A05882329F14881481B7B
:103C300047FD40E0242F332727FD30958A2D90E063
:103C4000281739070CF04A2D48838981E114F104C3
:103C500059F0C41608F44C2DF701E40FF11DE4915E
:103C60008E1718F4E82F01C0E0E0E98380E6809326
:103C7000D00D10920A058881882319F190910905C9
:103C80009923F9F04981E114F104B1F0491B47FD92
:103C900040E09C2D8C1508F4982FF701E90FF11DD9
:103CA000E491242F332727FD30958E2F90E028179D
:103CB00039071CF04E2F01C040E0498380E6809315
:103CC000D00D103651F1113690F4133409F480C040
:103CD000143430F4113279F1123409F09CC06AC006
:103CE000143409F43FC0153409F095C04FC01436A0
:103CF000E9F1153638F4123609F45FC0133609F0CD
:103D00008AC069C01138A1F01F3B21F0153609F0B7
:103D100082C040C01982188212C0552309F47BC0AA
:103D200081E090910605911180E08093060573C0B3
:103D3000109206050DC080910605882319F0109297
:103D4000060569C08881882319F08114910421F443
:103D500080E00E94F6155FC087E10E94847319829B
:103D6000188256C08981851709F455C0E114F10401
:103D700009F451C080910605882309F04CC089815F
:103D8000851710F48F5F12C0198242C08981882381
:103D900009F441C0E114F10409F43DC08091060525
:103DA0008823C9F58981882319F08150898330C01F
:103DB00059832EC088818A1571F180910605882368
:103DC00051F588818A1510F48F5F0DC018820EC0DE
:103DD0008881882301F1809106058823E1F4888198
:103DE000882319F08150888301C0A8828981E11459
:103DF000F10461F098819C1508F4C92EEC0CF11CBB
:103E0000F7019491891718F4982F01C090E09983D5
:103E100080E68093D00DDF91CF911F910F91FF909D
:103E2000EF90DF90CF90AF909F908F907F906F90AA
:103E300008954F925F926F927F928F929F92AF926E
:103E4000BF92CF92DF92EF92FF920F931F93DF9377
:103E5000CF930F92CDB7DEB7D82E85E89BE00E94B6
:103E6000C21B8FE398E06D2D41E021EF37E006E0C3
:103E70005DE8E52E5BE0F52E15E0C12EB6E0AB2E39
:103E80000E943A1D80903F08909040088091630006
:103E900081FF07C08AE268E14FE75BE00E946B6642
:103EA00060C182E168E040E75BE00E946B668A9453
:103EB00080910605882319F0A2E0CA2E02C0CC2406
:103EC000C394EE24FF2410E1A82CBB24A7FCB094DB
:103ED000F4E06F2E712C2701440C551C84E691E010
:103EE000480E591E4E2D4F5F80E0612F20E00E944A
:103EF000B80FAE14BF0411F491E0911090E0F201FC
:103F00002181229526952695237030E0A901440F42
:103F1000551F420F531F4A59544F992311F400E083
:103F200001C00C2D88E1612F23E099830E940C666B
:103F300099819923C1F0809106058823A1F0F201AF
:103F4000618162956695669563708D2D40E022E0F3
:103F50000E94DD158295880F880F807CF201918187
:103F60009F73982B9183AE14BF0421F401E0F92DC7
:103F7000F13009F000E0F2018181880F880F85950A
:103F80008595FDE08F02C0011124B3010E947F7767
:103F9000AB01002311F420E001C02C2D82E4612F3D
:103FA0000E947F680023A9F080910605882389F08C
:103FB000F2016181660F660F659565958D2D41EE65
:103FC0002FE10E94DD158F73F2019181907C982B77
:103FD0009183AE14BF0421F491E0F92DF23009F081
:103FE00090E0F2012081277030E0A901440F551FB5
:103FF000420F531F475A544F992311F400E001C058
:104000000C2D88E4612F23E099830E940C6699812E
:10401000992391F080910605882371F0F201608167
:1040200067708D2D40E023E00E94DD158770F2015E
:104030009081987F982B9083AE14BF0421F401E007
:10404000F92DF33009F000E0F201408145954595E6
:104050004595002311F420E001C02C2D8AE5612F45
:104060000E9404100023B1F080910605882391F08E
:10407000F20160816595659565958D2D4AEE26E185
:104080000E94DD15880F880F880FF20190819770CC
:10409000982B9083185F0894E11CF11C103309F0F1
:1040A0001ACF80E36EE47BE00E9463664091740166
:1040B000552747FD5095465F5F4FF82DF43011F4BA
:1040C00021E201C020E28EE460E30E947F68282D97
:1040D000243049F48D2D6091740146EF28E20E944E
:1040E000DD1580937401EE24E394882D853009F06A
:1040F000EE2480E068E34AE45BE02E2D0E943C66FB
:104100004CE8A42E44E0B42E0CE511E090E3F50158
:10411000419151915F01F801219131918F01421B31
:10412000530B440F551F892F68E320E299830E94A7
:104130007F689981985E903951F7EE2091F0FD2DBE
:10414000F03679F4ACE5B1E0ECE8F4E088E0019019
:104150000D928150E1F781E00E942D6087E10E947D
:1041600084730F90CF91DF911F910F91FF90EF908B
:10417000DF90CF90BF90AF909F908F907F906F9087
:104180005F904F9008956F927F928F929F92AF921F
:10419000BF92CF92DF92EF92FF920F931F93CF9334
:1041A000DF93B82E88EA90E10E94C21B82EA98E071
:1041B0006B2D4AE02BED37E00BE0E3EBEE2EE0E178
:1041C000FE2E73E0C72E54E0A52E0E943A1DF090FB
:1041D000A2089090A3088B2D8252843048F48091DD
:1041E0000605882329F080912C0F806380932C0F83
:1041F00080910605882319F012E0A12E02C0AA249E
:10420000A394C9EBDEE0B7EBCB2EBEE0DB2E662439
:10421000772410E1812F6DE970E10E946366862D9D
:10422000813031F480E0612F42E520E00E94496551
:104230000894611C711C4881E3E04E9FA001112489
:1042400040575F4E862CF61411F4992011F000E0CF
:1042500001C00A2D82E4612F23E00E940C66F60162
:10426000208130E040E050E0F81419F4F92DF130ED
:1042700011F000E001C00A2D86E6612FA3E0EA2ECE
:104280000E944967F81431F580910605882331F4BE
:1042900080918204909183040097E1F0992021F0AD
:1042A000892D8130B9F409C08B2D688140E023E06D
:1042B00002E00E94C01588830DC0F60160818B2D3D
:1042C00070E040E050E028E730E002E00E940A158C
:1042D000F601808321960894C11CD11C183111F07D
:1042E000185F98CF88E267E870E10E94636680916A
:1042F0009601829586958695837090E0AC01440F77
:10430000551F480F591F43585F4EFF2DF33011F0D2
:1043100000E001C00A2D82E468E223E00E940C66FE
:104320008F2D8330C9F460919601629566956695EC
:1043300063708B2D70E040E050E022E030E002E05E
:104340000E940A158295880F880F807C90919601B3
:104350009F73982B9093960180E361E770E10E9430
:1043600063662091040430E0220F331F442737FD99
:104370004095542FEF2DE43019F40A2D006301C04D
:1043800000E384E560E374E0E72E0E944967FF2DB7
:10439000F43069F4609104048B2D70E040E050E04B
:1043A00022ED30E002E00E940A1580930404DF91C0
:1043B000CF911F910F91FF90EF90DF90CF90BF9022
:1043C000AF909F908F907F906F9008952F923F9223
:1043D0004F925F926F927F928F929F92AF92BF9215
:1043E000CF92DF92EF92FF920F931F93DF93CF93C1
:1043F000CDB7DEB729970FB6F894DEBF0FBECDBF9D
:10440000982E87EF90E10E94C21B84EA98E0692D04
:1044100049E02BED37E00BE0E1E0EE2EE1E1FE2E8E
:1044200076E0C72E57E0A52E0E943A1DF090A40812
:104430001091A508892D8252843030F480910605B0
:10444000882311F00E940F7780910605882319F0C8
:1044500042E0242E02C02224239488E06EEE70E114
:104460000E946366909196019695969596959370A5
:1044700045E0949FA00111244D515F4E2F2D213016
:1044800011F401E0111100E08CE368E025E09F8366
:104490000E940C669F818F2D8130B1F41123A1F40D
:1044A00080910605882381F0892D692F40E021E065
:1044B0000E94CE158370880F880F880F9091960107
:1044C000977E982B90939601909196019295969550
:1044D000917043E0949FA001112444525F4EEF2D50
:1044E000E13019F401E0113009F000E080E668E005
:1044F00023E09F830E940C669F81FF2DF130B1F471
:104500001130A1F480910605882381F0892D692F4F
:1045100040E021E00E94CE1581708295880F807E58
:10452000909196019F7D982B9093960187E294E05D
:104530009A838983CC24DD2432E0332E20E1822E3D
:10454000922D90689E83882D61ED70E10E946366D4
:10455000CB824C2D4F5C86E0682D0E940866E98175
:10456000FA814081F31421F4112311F40E8101C06A
:1045700000E880E6682D2B81EE240E94A810F60149
:10458000EE0FFF1FEE0FFF1FE65DFB4F40814295D0
:1045900046954695437050E044535F4EF31411F432
:1045A000113011F000E001C0022D80E6682D21E0FD
:1045B0000E940C66F314E1F580910605882331F41E
:1045C0008091820490918304009791F1112319F056
:1045D000113071F510C0E981FA816081892D70E098
:1045E00040E050E02FEF30E002E00E940A15E98140
:1045F000FA8180831DC05601AA0CBB1CAA0CBB1CEF
:104600008AE294E0A80EB91EF50160816295669574
:1046100066956370892D40E023E00E94CE15829557
:10462000880F880F807CF50190819F73982B908371
:10463000532C539408E0402E480C5601AA0CBB1C86
:10464000AA0CBB1C88E294E0A80EB91E662477244D
:10465000F601EE0FFF1FEE0FFF1FE65DFB4FF98720
:10466000E887E885F9854081242F2F7030E0C30169
:10467000880F991F02C0359527958A95E2F7F22F8A
:10468000F370FC83842F8295837090E0062C02C027
:10469000959587950A94E2F7282F21702D8384E061
:1046A000642D47EC50E120E00E943C668C8193E051
:1046B000899FA001112446545F4EF51411F4112373
:1046C00011F000E001C0022D84E2642D23E00E947D
:1046D0000C66ED814E2F50E049545F4EF51411F4F5
:1046E000113011F000E001C0022D82E4642D21E0C0
:1046F0000E940C66F5014081F51421F4123011F48A
:104700000E8101C000E880E6642D2B81EE24E39445
:104710000E94A810F51409F064C080910605882352
:1047200039F48091820490918304009709F459C070
:10473000113019F1113020F0123009F052C044C08C
:10474000892D6C8140E023E002E00E94C015E885DD
:10475000F98520816114710431F0982F990F990F18
:104760002370922B03C0922F9C70982B9F70E8852A
:10477000F9858081807F892B33C0892D6D8140E050
:1047800023E002E00E94C015E885F985208122958A
:1047900023706114710429F0982F990F2D7F922BAB
:1047A00003C0922F9E7F982B93709295907FE885FF
:1047B000F98580818F7C892B808380917F04882379
:1047C00081F00E940F770DC0F5016081892D70E0A6
:1047D00040E050E02FEF30E002E00E940A15F501C2
:1047E00080835394F8E04F0E0894611C711C089468
:1047F000A11CB11C22E06216710409F032CF83E0E3
:10480000380E98E1890E0894C11CD11CE981FA8107
:104810003496FA83E983F82DF03409F094CE299682
:104820000FB6F894DEBF0FBECDBFCF91DF911F91C1
:104830000F91FF90EF90DF90CF90BF90AF909F903F
:104840008F907F906F905F904F903F902F90089542
:10485000AF92CF92EF92FF920F93AE2CEE24FF24F3
:10486000CC240E943A1D0F91FF90EF90CF90AF9013
:104870000895EF920F93DF93CF930F92CDB7DEB7EA
:10488000682F83E99BE069830E94C21B81E498E062
:10489000698142E021EF37E006E0EE240E942824FF
:1048A00080E16FE677E00E94636688E16CE377E081
:1048B0000E94636680E26FE477E00E94636688E2AC
:1048C00060E677E00E94636680E36FE777E00E942E
:1048D00063660F90CF91DF910F91EF900895CF9283
:1048E000DF92EF92FF920F931F93DF93CF9300D04D
:1048F000CDB7DEB7682F82EC9BE069830E94C21BB4
:1049000083E498E0698143E021EF37E006E0EE249C
:104910000E942824BEE0CB2ED12C00E010E0143001
:1049200020F0A8EFFA2EF00E01C0F02EC6010E9472
:10493000E969E82E1F5F8AE26F2D412F20E00E9477
:1049400004104E2D405D84E46F2D2E2D0E9449658C
:10495000085F0894C11CD11C193009F708E3CC2466
:10496000DD2410E0812F90E00E94E969F82EA60175
:104970004D55544F80E0602F25E00E9436664F2D44
:10498000405D80E2602F2F2D0E9449651F5F85E00A
:1049900090E0C80ED91E0850163021F784E568E172
:1049A0004BE95BE027E00E943666F6E0EF2EF12C43
:1049B00010E230E084E5612F40E957E0232F00E06A
:1049C0003A830E94EA64C7010E94E969282FC7015F
:1049D000019629830E94E969082F2981422F405DB1
:1049E0008CE6612F0E944965402F405D88E7612F6A
:1049F000202F0E9449653A813F5F185FE2E0F0E0B6
:104A0000EE0EFF1E3430B1F60F900F90CF91DF9174
:104A10001F910F91FF90EF90DF90CF9008958F92AC
:104A20009F92AF92BF92DF92EF92FF920F931F93EC
:104A3000CF93DF93D82E8AEC9BE00E94C21B85E4C3
:104A400098E06D2D44E021EF37E006E0EE24E3949A
:104A50000E942824F0904508C7EDD4E010E000E063
:104A6000812C84E0982EA12CB12C88E1612F41E4A7
:104A70000E940866402F4F5C8EE1612F0E940866FD
:104A8000802F0E94BD16AC018AE2612F0E946F66E2
:104A90000730B1F068817981882777FD8095982F5C
:104AA00024E630E040E050E00E944077A501940108
:104AB0000E94B4778AE5612FA9010E948F680AC01D
:104AC0008F2D813011F040E201C041E28AE5612F73
:104AD0000E94B20F0F5F185F2296083031F68CE605
:104AE00068E247EC5BE022E00E94366640910901F3
:104AF00050910A0188E760E320E00E947F688F2DD3
:104B0000813059F4F09208058D2D60915A0141E8E9
:104B10002FE70E94DD1580935A01DF91CF911F91FD
:104B20000F91FF90EF90DF90BF90AF909F908F908C
:104B30000895EF920F93E42E40E020E030E000E093
:104B40000E9428240F91EF900895AF92BF92CF92C8
:104B5000DF92EF92FF920F931F93DF93CF9300D0DA
:104B6000CDB7DEB78FE161E247E10E94ED668FE1EC
:104B700067E347E10E94E96685E361E247E10E945D
:104B8000ED668FE161E247E10E94E9668BE461E254
:104B900047E10E94ED668BE467E347E10E94E96626
:104BA00081E661E247E10E94ED668BE461E247E164
:104BB0000E94E9668AE26BE243E00E94ED6689E2C8
:104BC0006CE243E00E94E96686E56BE243E00E9406
:104BD000ED6685E56CE243E00E94E9668091D704CA
:104BE0009091D80471E7C72ED12CB6010E947F772F
:104BF000262F8091D9049091DA040FE81FEFB801B5
:104C00000E947F77362F68E2E62EE20E5AE2F52EFA
:104C1000F30E8E2D6F2D45E02A8339830E94ED66B9
:104C20003981632F625D8E2D45E00E94E9662A81FD
:104C3000822F845D6F2D45E00E94ED668E2D6F2DD5
:104C400045E00E94E9668091DD049091DE04B601A2
:104C50000E947F77262F8091DB049091DC04B801BD
:104C60000E947F77062F44E5F42EF20E162F165D74
:104C70008F2D612F45E02A830E94ED66602F625DD3
:104C80008F2D45E00E94E9662A81822F885A612F84
:104C900045E00E94ED668F2D612F45E00E94E96698
:104CA0003FEDA32E34E0B32E2AE3F22E0DE510E003
:104CB00098E3E92EF501819191915F0180509C4F1D
:104CC000B8010E947F77D62ED394CE2CCD188F2D8D
:104CD0006C2D4D2D0E94ED668F2D8F5F6C2D4D2D0F
:104CE0000E94ED668F2D8E5F6C2D4D2D0E94ED661E
:104CF000F5E0FF0E8F2D8934E9F60F900F90CF91DC
:104D0000DF911F910F91FF90EF90DF90CF90BF90B8
:104D1000AF9008954F925F926F927F928F929F9281
:104D2000AF92BF92CF92DF92EF92FF920F931F93B9
:104D3000DF93CF930F92CDB7DEB7B82E8FE19CE013
:104D40000E94C21B82E798E06B2D45E021EF37E01F
:104D500006E0EE24E3940E9428241092720836E5BF
:104D6000E32E38E0F32E28E4C22E28E0D22E86016E
:104D7000470160E0862F69830E94BD16D4014D91E2
:104D80005C911197282F392F6981421753070CF432
:104D90009A01F401219331934F01D8014D915C9117
:104DA0001197282F392F241735070CF49A01F80191
:104DB000219331938F016F5F6730E1F6809147084F
:104DC00080930805FB2DF03219F0FF3B71F40BC006
:104DD0008F5F80934708833041F487E10E9484739A
:104DE00081E00E942D601092470880914708813031
:104DF000B1F0813020F0823009F0A4C03FC08CE0D7
:104E000060E14DE05CE021E100E00E940C6682E19F
:104E100068E14DEF5BE02FE00E940C6693C08EE1ED
:104E200060E140EF5BE02CE000E00E940C6682E174
:104E300068E14EEC5BE020E10E940C6694E6892E6E
:104E400098E0992E20E008E91AE388E6A82E85EC80
:104E5000B82ED7010D931D937D01F601A192B19259
:104E60006F01822F29830E94BD16D4018D939D93DB
:104E70004D0129812F5F273061F764C082E160E135
:104E80004FED5BE020E100E00E940C6682E168E10A
:104E90004EEC5BE020E10E940C6614E6A12E18E0C7
:104EA000B12EBBE24B2EB1E05B2EF201A0E48A2EC4
:104EB000912CD7018D919D917D01D6016D907D90B2
:104EC0006D019C012619370937FF03C030952195E4
:104ED0003F4F23333105DCF0D5012D913C913183D7
:104EE00020838901081B190BC801B4010E947F7738
:104EF000061B170B17870687C301821B930B9C01A8
:104F0000B4010E947F77261B370B358F248FA2E0D8
:104F1000B0E0AA0EBB1E3296B4E6EB16B8E0FB0674
:104F200041F680E090E0F201219131912F01820F52
:104F3000931FF3E44F16F1E05F06A9F79093560133
:104F4000809355010E94A5250F90CF91DF911F916D
:104F50000F91FF90EF90DF90CF90BF90AF909F9018
:104F60008F907F906F905F904F900895282F30E042
:104F7000C901880F991FA90163E0440F551F6A9565
:104F8000E1F7840F951FA9014F5F5F4FBA01660FCC
:104F9000771FA3E0440F551FAA95E1F7640F751F13
:104FA0006C557E4F20953095205E3F4FA901440FF0
:104FB000551FE3E0220F331FEA95E1F7420F531F1D
:104FC0008C559E4F0E94E4778AE0EAEDF2E0DF0123
:104FD0001D928A95E9F782E00E942D600E94C960C7
:104FE00008950F931F93CF93DF93282F30E0E901AB
:104FF000CC0FDD1FC90113E0880F991F1A95E1F747
:10500000C80FD91F8E010C551E4FA9014F5F5F4F6E
:10501000CA01880F991FA3E0440F551FAA95E1F715
:10502000840F951F20953095205E3F4FA901440FB6
:10503000551FE3E0220F331FEA95E1F7420F531F9C
:105040008C559E4FB8010E94E4778AE0D8011D92EA
:105050008A95E9F780919608C657DE4F8A8F8B8F25
:1050600084E68C8F82E00E942D600E94C960DF91EF
:10507000CF911F910F910895FF920F931F9385EF8A
:10508000EBE2F5E0DF011D928A95E9F780912006B9
:10509000A4EAB1E050E021E030E060E07C917723C9
:1050A00011F0472F01C040E1641738F5F22E032FAD
:1050B000162F1F5F802F90E0FC01EE0FFF1FEE0FF9
:1050C000FF1FE80FF91FE55DFA4F912F9F73808155
:1050D000807C892B80648083F182F39453830F5FFB
:1050E000141738F3962F9095642F822F8F5F890FB6
:1050F000390F340F290F240F840F772359F1832F91
:1051000090E0FC01EE0FFF1FEE0FFF1FE80FF91FED
:10511000E55DFA4F4F738081807C5483842B8068D7
:10512000808322832F5F1A968C911A97781719F42F
:105130001182138205C021832F5F852F8F5F8383A8
:10514000822F5F5F1A96503219F42093200604C014
:105150003F5FA4CF809320061F910F91FF90089589
:10516000E4EAF1E080E090819150903108F48F5FA3
:105170003A9692E0E43EF907B1F708951F93182F8D
:1051800080E16DE07FE00E9463660E94B028482FB6
:1051900088E760E150E020E00E947F6880E267EFEE
:1051A0007EE00E946366113651F481E60E94486AEF
:1051B00081E00E94F6158EE799E20E942B161F915E
:1051C00008950E94B028803230F08EEB98E20E9461
:1051D0002B1681E0089580E00895EF92FF920F93DF
:1051E0001F93DF93CF9300D0CDB7DEB7182F813256
:1051F00008F07BC0882319F4442341F476C0803240
:1052000019F4442331F071C0442319F0012F0F5FCA
:1052100002C0012F0150812F4A8369830E94170F1A
:105220007C01802F0E94170FFC01D7018C91982FD1
:1052300091504A816981903108F057C02081213115
:1052400008F053C06623A1F10E94E128882309F0E9
:105250004CC0212F30E0A9014F5F5F4FCA01880F7A
:10526000991F13E0440F551F1A95E1F7840F951FFE
:10527000B901660F771FA901A3E0440F551FAA9536
:10528000E1F7640F751F6C557E4F20953095205EB9
:105290003F4FA901440F551FE3E0220F331FEA954A
:1052A000E1F7420F531F8C559E4F0E94E4771DC0BB
:1052B000281759F0442331F08031B8F48F5FF7019B
:1052C000808313C0D7019C9310C0D701CF010A96E9
:1052D00004C020813C9131932D93E817F907C9F759
:1052E00082E00E942D600E94C9600F900F90CF91C4
:1052F000DF911F910F91FF90EF9008956F927F9231
:105300008F929F92AF92BF92CF92DF92EF92FF92D5
:105310000F931F93CF93DF93182F81EF9EE00E948E
:10532000C21BE0902006EA9489E998E0612F44E0EE
:105330002BED37E00BE00E942824C0909908CC2088
:1053400011F4109298081236D9F1133670F4133410
:10535000A9F1143420F4123409F070C031C01036B1
:10536000C1F0113609F06AC045C0103809F452C0C6
:10537000113820F4133609F061C020C01E3BB9F18A
:105380001F3B09F05BC081E080939708109298085A
:105390002EC01C143CF481E090919808911180E09B
:1053A000809398088091980880939708809194083A
:1053B000882309F443C01092980840C010929708BF
:1053C000809198088823D1F141E0123609F040E03D
:1053D00080919508609197080E94ED288091970828
:1053E000882319F0133609F4CA94109297080E9482
:1053F0003C2824C080919808882301F18091950869
:105400000E94B627109298080E943C2881E60E94CC
:10541000486A14C01C1494F480919408882341F0C5
:105420000E94E128882321F4809195080E94F127A9
:10543000109298088CE99AE50E942B1638E0D32E3A
:1054400077247A9423E6822E9924BB24BA94662486
:105450006394E0900505E90CFF24F701EE0FFF1FB0
:10546000EE0FFF1FEE0DFF1DE55DFA4F4081842F0B
:10547000807C09F462C146FF06C04F7380E06D2D49
:1054800020E00E94E40F1C14E4F4E701CC0FDD1FC0
:10549000CC0FDD1FCE0DDF1DC55DDA4F8981C8162B
:1054A00081F46D2D695F80E048E10E94E9668B819F
:1054B0008093950888818F738093960860929408F2
:1054C000B92CF701EE0FFF1FEE0FFF1FEE0DFF1DB2
:1054D000E55DFA4F808187FF05C19481C92FDD27E3
:1054E000C7FDD095AA24A3949281C912AA2486FD4F
:1054F0001FC0FE01EE0FFF1FCE01A3E0880F991F12
:10550000AA95E1F7E80FF91FE555FE4F4081469552
:10551000477050E04351514F80919808882311F40F
:1055200000E001C00A2D82E16D2D21E00E940C6691
:10553000FE01EE0FFF1FCE0163E0880F991F6A95F1
:10554000E1F7E80FF91FE657FE4F448D552747FD59
:1055500050958DE26D2D2A2D0E947F6880919808CC
:10556000882311F420E001C02A2D8DE26D2D45E243
:105570000E944965FE01EE0FFF1FCE0143E0880F38
:10558000991F4A95E1F7E80FF91FE657FE4F438D43
:1055900080919808882311F420E001C02A2D86E329
:1055A0006D2D0E94B80FFE01EE0FFF1FCE0123E00C
:1055B000880F991F2A95E1F7E80FF91FE657FE4F6C
:1055C000458D442359F080919808882311F420E0F8
:1055D00001C02A2D8EE46D2D0E940410FE01EE0FF5
:1055E000FF1FCE01B3E0880F991FBA95E1F7E80FCE
:1055F000F91FE657FE4F468D442391F023E0429F6A
:10560000A001112449595E4E80919808882311F415
:1056100000E001C00A2D86E66D2D23E00E940C6695
:10562000FE01EE0FFF1FCE0173E0880F991F7A95E0
:10563000E1F7E80FF91FEC55FE4F21E08581882343
:1056400009F420E0FE01EE0FFF1FCE0153E0880FAA
:10565000991F5A95E1F7E80FF91FEC55FE4F868127
:10566000882329F0222309F498C04AE203C02223A8
:1056700061F044E480910605882311F420E001C024
:105680002A2D89E76D2D0E9449658A2D813051F5BB
:105690005E01AA0CBB1C33E0CC0FDD1F3A95E1F78D
:1056A000AC0EBD1EEAE8F1E0AE0EBF1E812FF50183
:1056B000648D43E82DE70E94CE15F501848FF70134
:1056C000EE0FFF1FEE0FFF1FEE0DFF1DE55DFA4F02
:1056D00084818093950880818F73809396081092BF
:1056E0009408B92CF701EE0FFF1FEE0FFF1FEE0D10
:1056F000FF1DE55DFA4F8181882331F088150CF498
:10570000882E87150CF0782EF701EE0FFF1FEE0F95
:10571000FF1FEE0DFF1DE55DFA4F8281882331F0FA
:1057200088150CF4882E87150CF0782E9394F8E0E9
:10573000DF0E292D273009F08CCECC20A1F08B2D47
:105740008F3FF9F4C81464F48091050590E0019747
:10575000EFEF8F3F9E0711F480E090E08093050506
:105760007C14ECF414C0FB2DFF3F59F48091050527
:1057700090E001972FEF8F3F920761F480E090E077
:1057800009C08B2D86305CF0992D983040F08091C7
:1057900005058F5F8093050502C043E56BCFDF9160
:1057A000CF911F910F91FF90EF90DF90CF90BF901E
:1057B000AF909F908F907F906F9008952F923F921F
:1057C0004F925F926F927F928F929F92AF92BF9211
:1057D000CF92DF92EF92FF920F931F935C01CC2444
:1057E000DD243B018824992464E6262E312C412CAB
:1057F000512CC201B1016619770988099909A601DE
:1058000095010E9440777B018C0182E390E0A0E04B
:10581000B0E0E80EF91E0A1F1B1FC601B5010E9469
:1058200040770E944077BC0188279927A401930103
:105830000E94407744E096958795779567954A95BD
:10584000D1F7E60EF71E081F191FC801B701A20104
:1058500091010E949277C9011F910F91FF90EF90E3
:10586000DF90CF90BF90AF909F908F907F906F9080
:105870005F904F903F902F9008951F93CF93DF93A9
:105880009C016115710511F1132F111F1127111FB3
:1058900019F0309521953F4F77FF0EC0C0E0D4E05E
:1058A000709561957F4FCE01821B930B0E94DE2B7A
:1058B0009E01281B390B05C0C9010E94DE2B282F31
:1058C000392F112319F0309521953F4FC901DF91F0
:1058D000CF911F9108956F927F928F929F92AF9276
:1058E000BF92CF92DF92EF92FF920F931F93DF93BD
:1058F000CF93CDB7DEB7982E962F322F802F6E2DF7
:10590000222359F0442361F440918204509183048E
:105910004115510539F421E001C020E0FF2405C004
:1059200022E001C021E0FF24F394332311F0911110
:1059300021E04A2D433679F44C2D50E0440F551F99
:105940008A0173E0000F111F7A95E1F7041B150B14
:10595000005C1C4F11C0FA2DF236D9F44C2D50E0EA
:10596000440F551F8A0193E0000F111F9A95E1F72C
:10597000041B150B0F5B1C4FF80140810E940410A3
:10598000FF2009F463C0F8016081892D4AEE26E109
:1059900059C069887724BB24882051F54C2D50E0EC
:1059A000440F551F6A01B3E0CC0CDD1CBA95E1F73A
:1059B000C41AD50AAA0CBB1CAA0CBB1CCA0CDB1C43
:1059C000C60CD71C44E353E0C40ED51EF60140813B
:1059D000552747FD50950E947F68FF20B9F1F601D9
:1059E0006081892D4CE924E60E94CE15F6012DC078
:1059F000DD24AA0CBB1CA601E3E0440F551FEA9569
:105A0000E1F74C195D09A40EB51EA80CB11CAA0C37
:105A1000BB1CF301EA0DFB1DEC5CFC4F40815527DC
:105A200047FD50954C595F4F0E947F68FF2071F0F1
:105A30008501060D171D0C5C1C4F892DF801608136
:105A40004CE920E00E94CE15F8018083CF91DF91D0
:105A50001F910F91FF90EF90DF90CF90BF90AF908C
:105A60009F908F907F906F9008952F923F924F92CA
:105A70005F926F927F928F929F92AF92BF92CF92DE
:105A8000DF92EF92FF920F931F93DF93CF93CDB7E7
:105A9000DEB72A970FB6F894DEBF0FBECDBFD82E63
:105AA00084EE9EE00E94C21B82E998E06D2D40E0EA
:105AB00020E030E000E07CEEE72E7EE0F72ECC2404
:105AC00053E0A52E0E943A1D40918A084F5F80E363
:105AD00060E020E00E94B80FF090920880918A0860
:105AE00090E0880F991FFC0123E0EE0FFF1F2A951D
:105AF000E1F7E81BF90BE05CFC4F808160E040E0DF
:105B00000E947E118823C1F080918A0890E0880F5E
:105B1000991FFC0113E0EE0FFF1F1A95E1F7E81B38
:105B2000F90BEF5BFC4F808160E040E00E947E114A
:105B3000882321F411E003C010E001C012E060915D
:105B40008A08462F50E0FA01EE0FFF1FE952FB4F83
:105B5000808191818A3191051CF01092910807C0D3
:105B60002FEF873E92071CF481E0809391082091EB
:105B70006E0130E02170307082E090E0821B930B68
:105B80008417950741F4643030F480919B01807F45
:105B900011F01092910880E16FED7EE00E94636643
:105BA0000F92EDB7FEB7319621E0F11020E0809121
:105BB000910880838D2D61E041E006E3A0E1EA2EAB
:105BC000C0908A08A12E88240E946B2C0F9088E137
:105BD00068ED7EE00E9463660F92EDB7FEB73196E6
:105BE00021E03F2D313009F020E080919108808341
:105BF0008D2D61E041E006E3F8E1EF2EC0908A08C8
:105C0000A12E882483940E946B2C0F9080E262ED79
:105C10007EE00E9463660F92EDB7FEB7319621E0F9
:105C20008F2D823009F020E010828D2D61E041E05F
:105C30000EE1E0E2EE2EC0908A0873E6A72E8824DB
:105C40000E946B2C0F9088E26CEC7EE00E946366F1
:105C50000F92EDB7FEB7319621E09F2D933009F0FA
:105C600020E010828D2D61E041E00EE158E2E52E4A
:105C7000C0908A0832E6A32E88240E946B2C0F90D5
:105C8000113019F0123049F404C080E365EC7EE075
:105C900007C080E36EEB7EE003C080E366EB7EE04E
:105CA0000E94636600918A08402F50E0812F90E0A7
:105CB000880F991F880F991FBA01660F771F9B01E4
:105CC000B3E0220F331FBA95E1F7261B370B820F83
:105CD000931F86579E4FFC01E655FE4FA081A98376
:105CE000FC01E555FE4FB081BA83FC01E455FE4F3F
:105CF0009080E4E69E0E83559E4FDC018C908E0EC4
:105D000020916E0130E02170307082E090E0821BC3
:105D1000930B8417950709F062C0043008F05FC048
:105D200080919B01807F09F45AC0EE24FF248701F3
:105D300020E030E0B9816B2E772467FC7094A1E2FB
:105D40004A2E512C292C332427FC3094F0E4CF2EFA
:105D5000D22ED801C701B595A79597958795B30120
:105D600029873A870E943D2C880F991FB2010E9413
:105D70007F77629DC001639D900D729D900D1124EF
:105D80006FE3A62EAD0C64E670E00E946B77EC2DFD
:105D9000E61B6E2F8A2D0E949D6629853A85C901D2
:105DA00083709070009761F48A2D6FE30E949D6666
:105DB0006D2D6695605E8FE30E949D663A8529850C
:105DC0002F5F3F4F81E290E0A0E0B0E0E80EF91EC7
:105DD0000A1F1B1F2E33310509F0BACF7CC0DD240A
:105DE0009981492E552447FC509401E210E0A92DD9
:105DF000BB27A7FDB095BC83AB8354E6652E712C01
:105E000040E2A42EBA812B2E332427FC3094E82DB7
:105E1000FF27E7FDF095FE83ED83FD2D21E2F29F44
:105E200070011124C701B2010E943D2CB8010E94EB
:105E30007F77AB81BC816A9FC0016B9F900D7A9F79
:105E4000900D11243EE5C32ECD0CB3010E946B775B
:105E5000BA2DB61B6B2F8C2D0E949D66ED2DF0E0A8
:105E6000E370F070F887EF83309749F48C2D60E28F
:105E70000E949D666D2D605E8EE50E949D66C70145
:105E8000B1010E943D2CB8010E947F772D813E8197
:105E9000629FC001639F900D729F900D11242EE5AB
:105EA000F22EFD18B3010E946B77605E8F2D0E9469
:105EB0009D668F819885009749F48F2D60E20E943E
:105EC0009D666A2D6D198EE50E949D66D3949D2D69
:105ED0009F3109F0A2CFE0918A08F0E0EE0FFF1F9A
:105EE000E952FB4F408051805201CC24B7FCC09452
:105EF000DC2CC601B50121E230E040E050E00E9418
:105F0000B477822F825A61E04EE30E94ED664091A1
:105F10008A0820916E0130E02170307082E090E0BC
:105F2000821B930B242F30E08217930709F050C097
:105F3000443008F04DC080919B01807F09F448C037
:105F4000C601B50160507C4F8F4F9F4F22E030E07B
:105F500040E050E00E94B477A9816A2F772767FD5F
:105F60007095C9010E943D2CBC01660F771F8827E0
:105F700077FD8095982F292D97FC2D5F25952595E8
:105F8000332727FD3095432F532F0E94407729E177
:105F900030E040E050E00E94B47779018A01CA0104
:105FA000B9012FED3FEF4FEF5FEF0E94B477622F03
:105FB000605C8FE34EE30E94E966C801B70122E00E
:105FC00030E040E050E00E94B47779018A013CC0A3
:105FD0001A141B041C041D0414F4698101C06A8195
:105FE000772767FD7095C2010E943D2C9C014427D4
:105FF00037FD4095542F1A141B041C041D0414F47F
:10600000692D01C0682D67FD6D5F659565957727E2
:1060100067FD7095872F972F0E94407729E130E028
:1060200040E050E00E94B47779018A01CA01B901C9
:106030002FED3FEF4FEF5FEF0E94B477622F605E6E
:106040008FE34EE30E94E966C601B50129E130E025
:1060500040E050E00E944077612CB1E07B2E812C23
:10606000912CA40193010E94B47782E760E3A90117
:1060700020E00E947F68C801B70129E130E040E0DC
:1060800050E00E944077A40193010E94B47784E518
:1060900068E0A90120E00E947F681A141B041C0418
:1060A0001D0474F4B9816B2F772767FD7095C201C9
:1060B00044970E943D2CF701E81BF90BCF010BC060
:1060C000FA816F2F772767FD7095C20144960E9471
:1060D0003D2C8E199F099C01220F331F220F331F65
:1060E000280F391F442737FD4095542F84E560E180
:1060F00000E3F3E0EF2E0E9449672A960FB6F8946A
:10610000DEBF0FBECDBFCF91DF911F910F91FF90EA
:10611000EF90DF90CF90BF90AF909F908F907F9047
:106120006F905F904F903F902F9008952F923F92E5
:106130004F925F926F927F928F929F92AF92BF9297
:10614000CF92DF92EF92FF920F931F93DF93CF9343
:10615000CDB7DEB72F970FB6F894DEBF0FBECDBF19
:10616000982E8CEA9EE00E94C21B8FE898E0692D71
:1061700043E02BED37E00BE0F4EBEF2EFEE0FF2EDB
:10618000CC24C394E4E0AE2E0E943A1DF0908F0818
:10619000FA9430909008292D203841F4F7FC06C07D
:1061A000F0928A0885E39DE20E942B1685E168E063
:1061B0004CE95EE00E946B6680E493E09C838B83F5
:1061C0007BE8472E78E0572EE7EDF4E0FB87EA877F
:1061D00010E1662477242F2D332727FD30953A834D
:1061E0002983C901880F991FFC0153E0EE0FFF1F9F
:1061F0005A95E1F7E81BF90BFE83ED83F62CEB8152
:10620000FC81808160E040E00E947E11882361F083
:10621000EB81FC81818160E040E00E947E11882357
:1062200029F4BB24B39404C0BB2402C042E0B42EC2
:106230002B2D30E038872F83C901880F991F880FD5
:10624000991FA301440F551F9A0103E0220F331F2A
:106250000A95E1F7241B350B820F931F86579E4F3B
:10626000DC01A355BE4FFC01E455FE4F3C9120815B
:10627000321751F4FC01E555FE4F86559E4F41E023
:106280002081FC018081281340E0EA85FB85819113
:106290009191FB87EA879C0197FF04C0222733274F
:1062A000281B390B2A3131050CF040E0242E8A31AD
:1062B00091051CF0F201108207C0FFEF873E9F0797
:1062C0001CF421E0F201208380916E0190E0817046
:1062D0009070E2E0F0E0E81BF90BE615F70551F4E9
:1062E00080919B01807F31F0F301E557F74F1082D9
:1062F000222423944F2D4F5F80E0612F20E00E94E5
:10630000B80F5D864C86F2013081F1E0F9873111DA
:10631000198680910605882351F4DD24D394809159
:10632000820490918304009721F4DD2402C0DD24CF
:10633000D39489819A818615970511F421E0311053
:1063400020E00F92EDB7FEB73183892D60E04D2D2F
:1063500007E2E12ECF2CAB2C88240E946B2C0F90EF
:1063600029813A812615370509F0D2C0332009F07A
:10637000CBC0DD2009F4CCC0222009F4C9C08F8134
:106380009885880F991F880F991FED81FE818E0FC8
:106390009F1F86579E4FF9858F0F911D86559E4FE3
:1063A0009F878E87892DEE85FF8560814CE924E6E5
:1063B0000E94CE15EE85FF858083AAC021E00F9252
:1063C000F2018081EDB7FEB78183892D60E04D2D0C
:1063D00009E3E12ECF2CAB2C882483940E946B2CF4
:1063E0000F9029813A812615370509F097C0332D82
:1063F000313009F08FC0DD2009F490C0222009F46B
:106400008DC08F819885880F991F880F991FED8106
:10641000FE818E0F9F1F86579E4FF9858F0F911D0E
:1064200084559E4F98878F83892DEF81F8856081F1
:106430004CE920E00E94CE15EF81F88580836EC084
:1064400021E00F92EDB7FEB71182892D60E04D2D4E
:106450000FE3E12ECF2CF3E6AF2E88240E946B2CA5
:106460000F9029813A812615370521F421E0332D3B
:10647000333009F020E00F92EDB7FEB71182892D7D
:1064800060E04D2D07E5E12ECF2CE2E6AE2E88240C
:106490000E946B2C0894411C511C0F90EC85FD85CB
:1064A0008081882319F4222031F008C0222031F4A1
:1064B0008AE34FE705C08BE34EE702C08AE34DE273
:1064C000612F0E940866FB2DF13019F0F23049F47B
:1064D00004C085E7612F4DE407C085E7612F4CE4D8
:1064E00003C085E7612F48E40E9408660894611C98
:1064F000711C2B813C81225F3F4F3C832B83185FB3
:10650000103309F07BCE0CC0332D313009F456CF57
:1065100020E055CF832D823009F492CF20E091CF37
:106520002F960FB6F894DEBF0FBECDBFCF91DF918F
:106530001F910F91FF90EF90DF90CF90BF90AF90A1
:106540009F908F907F906F905F904F903F902F9093
:10655000089520E030E0F901E75AF14FE491E8179F
:1065600011F4822F08952F5F3F4FEE23A1F780E0B3
:106570000895823430F4E82FF0E0E75AF14F849127
:10658000089580E20895EF92FF920F931F93182FC2
:10659000F62EE22E862FBA010E94636686E66F2DE4
:1065A000412F2E2D0E94F51CEE2039F0802F612FF7
:1065B00040E021E00E94DD15182F812F1F910F91DF
:1065C000FF90EF900895FF920F931F93F82E109174
:1065D0009501212F332727FD309537FF03C03095D4
:1065E00021953F4F022F25320CF43DC020913908F0
:1065F00030913A088091370890913808282B392B30
:1066000080913B0890913C08282B392B80913608CB
:1066100090E0282B392B4091330850E0242B352B68
:106620002115310531F4812F881F8827881F809319
:10663000330811161CF4812F845202C0812F8C5D07
:1066400060E040E00E947E11882359F09091330869
:10665000992339F491E020913608211190E090932C
:106660003608809333082091390830913A082F5F1B
:106670003F4F30933A0820933908209137083091E2
:1066800038082F0D311D30933808209337080E94A9
:106690000F0F20913B0830913C08821B930B8436EE
:1066A000910508F471C12C593F4F30933C08209359
:1066B0003B082091370830913808E0913908F09173
:1066C0003A08C901BF010E946B77F62E462F50E0B1
:1066D0004E9FC0014F9F900D5E9F900D1124281B6F
:1066E000390B309338082093370810923A081092EB
:1066F000390800311CF4109236080FC005326CF4D2
:1067000011161CF4812F8F5002C0812F815F60E031
:1067100040E00E947E11809336088091230690917C
:106720002406019690932406809323064091250623
:10673000509126064F5F5F4F5093260640932506E3
:10674000FF2049F08091290690912A0601969093A6
:106750002A068093290680913608882349F0809183
:106760002706909128060196909328068093270685
:10677000F69420912B0630912C062F0D311D30936D
:106780002C0620932B06809197019091980190936D
:106790002F0680932E0660919501772767FD7095EF
:1067A00077FF03C0709561957F4F662319F41092AF
:1067B0002D061EC0613019F4841B950B15C0603185
:1067C00068F460FF06C0A4E036952795AA95E1F726
:1067D00009C02091290630912A0604C0209127067D
:1067E00030912806821B930B90932F0680932E06E0
:1067F00080912D06813051F0813018F0823049F5BA
:1068000014C080919501882321F120C080912E062B
:1068100090912F0618161906E4F080919701909137
:1068200098010097B1F082E012C080912E069091FD
:106830002F062FEF853C92071CF483E080932D06F2
:106840008091970190919801009719F481E08093CD
:106850002D0680912E0690912F06209134083091BC
:1068600035082817390709F479C020912D06213001
:1068700009F065C02091700122FF45C02091970169
:106880003091980121153105F1F18E31910519F4FE
:1068900089E10E94847380912E0690912F068431A5
:1068A000910519F48AE10E94847380912E069091DB
:1068B0002F068A30910519F48BE10E948473809130
:1068C0002E0690912F06843091051CF48CE10E94D5
:1068D00084738091700183FF16C080912E06909181
:1068E0002F068E31910549F08431910531F08A30BF
:1068F000910519F08430910534F482E390E090938F
:106900008604809385048091700181FF27C0809167
:10691000960120912E0630912F0680FF07C08091AE
:10692000970190919801821B930B01C0C9016CE300
:1069300070E00E946B77009789F480E003C02230FA
:1069400069F48CE10E9484738091700183FF06C01A
:1069500082E390E0909386048093850420912E0634
:1069600030912F063093350820933408809196019A
:1069700080FF0AC08091970190919801821B930B30
:1069800090932F0680932E061F910F91FF900895EC
:1069900080919501992787FD909597FF03C0909569
:1069A00081959F4F982F823034F1803124F5859561
:1069B0009A3024F40E94126B90E003C0992787FD5F
:1069C00090950197FC01EE0FFF1FE952FB4F2081CC
:1069D00031818091950187FF05C080E094E0821BA2
:1069E000930B03C0C90180509C4F26E09695879574
:1069F0002A95E1F702C080E090E00E94E33283E054
:106A00000E94126BE82FF0E0EE0FFF1FEB52FB4FDE
:106A10008081918180509C4FB6E096958795BA957C
:106A2000E1F72091960122FF0AC08530910538F0E8
:106A300020918804222319F423E0209388042091D4
:106A40002F08309130082F5F3F4F3093300820934C
:106A50002F0820912D0830912E08280F391F3093D0
:106A60002E0820932D080E940F0F2091310830919D
:106A70003208821B930B23E0883E9207E8F10E94C4
:106A80000F0F9093320880933108809199018230E2
:106A900051F485E160E040E00E947E11882319F006
:106AA00087E00E94847380912D0890912E08609158
:106AB0002F08709130080E946B7710922E08109268
:106AC0002D081092300810922F088091A9069091FD
:106AD000AA0601969093AA068093A9068091A8061B
:106AE000E82FF0E0E05DF94F60838F5F8093A806A8
:106AF000883710F01092A806089510922D06109273
:106B000026061092250610922A0610922906109247
:106B100028061092270610922C0610922B06089534
:106B20000F931F93182F80912106882319F069E491
:106B30007EE002C06CE37EE088E00E94636681E054
:106B400060E14AE851E02AE000E10E940C6682E43C
:106B500060E14FE30E94086682E168E245E35EE09F
:106B60000E946B6682E160E346E25EE00E946B6633
:106B7000113609F44AC01F3B21F0103609F04FC00E
:106B800004C080E00E9484734AC08091210688235B
:106B9000A9F084E19EE00E94C013809122060E9429
:106BA000955F882339F087E10E94847382E08093A7
:106BB000210629C080E00E94847325C0809157017E
:106BC0008F5F0E9459621091570108C01150113116
:106BD00008F01FE080915701181739F0812F8F5F5F
:106BE0000E940C62882391F301C010E010935701BA
:106BF00081E00E942D600E94C960809157010E942F
:106C0000575F0E947D3580E601C081E60E94486A98
:106C100081E00E94F61582E196E30E942B161F91F7
:106C20000F910895AF92BF92DF92EF92FF920F9370
:106C30001F93CF93DF93182F80E39CE00E94C21B29
:106C4000809106058823A1F4E0910905E7FF10C0B3
:106C5000E195EB3008F0EAE0F0E0EE0FFF1FE552BF
:106C6000F84F25913491C9010E941B161092090515
:106C7000F090840884E898E0612F4FE00E94992505
:106C800086E360E04BE25CE00E946B660E944E612E
:106C9000AC0186E660E020E00E947F6880E06BE067
:106CA00041E00E94151DD090840880912106823019
:106CB00021F41092830810922106163648F41436F7
:106CC00090F5103609F456C0113609F075C00AC0A7
:106CD000113809F456C01F3B09F465C0103809F09B
:106CE0006BC053C0809183088823E9F01092830819
:106CF00087E10E94847381E60E94486A0E94C9600D
:106D000080918408809357010E94575F0E947D35CF
:106D100081E00E942D600E94C96082E00E942D6087
:106D20000E94C96049C0809157018D15B9F0812F2B
:106D30000E94486A80918408809357010E94C9602C
:106D4000809157010E94575F0E947D3581E00E942B
:106D50002D600E94C96081E00E948473153619F489
:106D600083EC90E204C0143639F583EC9BE40E9476
:106D70001B1622C081E08093830887E10E94847300
:106D80001BC081E00E94F61517C0809183088823FC
:106D900099F081E080932106D092220680E995E364
:106DA0000E942B1609C0109283088091570180938E
:106DB000840881E00E943B6080918308882341F031
:106DC000FD1431F06D2D6F5F8F2D8F5F0E941A6261
:106DD000CD2DDD27C7FDD095809105059E01281B8F
:106DE0003109C901181619065CF0CE01019797FF09
:106DF00002C080E090E08093050510E1DD240BC027
:106E000025303105D4F3CE0104978B3091059CF3E6
:106E10008AE090E0F0CFF0900505FD0CAF2CBB248C
:106E200095012F5F3F4F442737FD4095542FCA15DA
:106E3000DB0511F401E101C000E182E1612F72E0A4
:106E4000E72E0E94496780915701F81629F481E0E6
:106E5000612F4AE20E9408668F2D64E778E04FE0D8
:106E60000E940F5FCA15DB0531F4809183088823E7
:106E700011F001E101C000E188E1612F44E758E031
:106E80002FE00E940C66D394185F3D2D363019F622
:106E9000DF91CF911F910F91FF90EF90DF90BF9006
:106EA000AF900895AF92BF92CF92DF92EF92FF9290
:106EB0000F931F93CF93DF935B016C0110E1E12EE1
:106EC000F12CC0E0D0E800E010E89E0140E050E086
:106ED000CA01B9010E944077A616B706C806D906AE
:106EE00010F4C027D127169507950894E108F108FA
:106EF000E114F10461F4CE01DF91CF911F910F9164
:106F0000FF90EF90DF90CF90BF90AF900895C02B8F
:106F1000D12BDBCFE1E0683068F4E0E070E09B016A
:106F2000220F331F220F331F260F371FA90140598D
:106F30005C4F0EC070E0685070409B0153E0220F20
:106F4000331F5A95E1F7260F371FA90148565C4FAA
:106F5000DA012C9180509C4F97FD0FC0B8E0803033
:106F60009B078CF0EE2319F028E030E002C024E00B
:106F700030E0240F351FF9012081332727FD30959C
:106F8000322F222730C0EE2329F0692F9070880F0E
:106F9000991F03C0692F66959170262F30E0FA0182
:106FA000E20FF31F6181772767FD7095AC0155955E
:106FB0004795649F9001659F300D749F300D11249B
:106FC0006081772767FD709540E052E0481B590BC0
:106FD00055954795649FC001659F900D749F900DD6
:106FE0001124280F391FC90169E170E00E947F77E1
:106FF000CB0108952F923F924F925F926F927F92B2
:107000009F92AF92BF92CF92DF92EF92FF920F9337
:107010001F93DF93CF9300D00F92CDB7DEB7182F19
:107020009924939480919B08883008F4992481E5F1
:1070300091E10E94C21B992011F05AE001C056E074
:107040008BEB98E0612F40E020E030E000E077E556
:10705000E72E71E1F72ECC24C394A52E0E943A1D91
:1070600040919B0850E04F5F5F4F84E260E021E079
:107070000E947F6880919B08992079F090E00897A2
:107080007C0103E0EE0CFF1C0A95E1F7E80EF91E07
:1070900028E933E0E20EF31E0CC090E07C01EE0C18
:1070A000FF1CEE0CFF1CE80EF91E80E793E0E80ED3
:1070B000F91E0091BB080150D090BC08113661F058
:1070C000123628F41434D1F0153471F50EC014368C
:1070D000A9F0153649F509C0DD2031F11092BC0840
:1070E00081E60E94486ADD241FC08091060588233E
:1070F000D9F01D14CCF48D2D815014C0809106055B
:10710000882391F02D2D332727FD3095992019F0F4
:1071100089E090E002C085E090E02817390724F468
:107120008D2D8F5F8093BC088091BC0880930605ED
:10713000CE2C4F2C6E2C7F2C90E122243324A02EB9
:10714000BB24A7FCB094F30141913F01552747FDB3
:10715000509521E0A214B30409F020E088E1692FE2
:1071600099830E947F680894211C311C9981985F43
:10717000983349F7992001F1A5E06A2E712C6E0C25
:107180007F1C90E1F5E02F2E312CF30141913F015E
:10719000552747FD509521E0A214B30409F020E0E3
:1071A00080E3692F99830E947F680894211C311C19
:1071B0009981985F903349F70F3F11F421E0D11086
:1071C00020E08CE068E04AE451E10E943C669920AE
:1071D00019F089E090E002C085E090E021E0A81677
:1071E000B90609F020E08CE068E343E451E10E9435
:1071F0003C66992019F089E090E002C085E090E0BB
:10720000A816B90694F407FD4EC0A02EBB24A7FC17
:10721000B094AE0CBF1C812FF50160814CE924E6CF
:107220000E94CE15F50180833EC01016E4F5812F33
:107230006091BA084CEF24E000E00E94C0158093F2
:10724000BA0890917F04992371F1992021F050E1BF
:1072500094E049E003C058E092E045E024E6820271
:1072600030011124892F90E0909581959F4F869D44
:107270009001879D300D969D300D1124EC2DF42D3D
:10728000A52E00E0C9016A2D702F0E947F776193BF
:10729000260D371D8E2F8C198417A0F382E00E94D3
:1072A0002D600E94C96080910605882351F0AA24B0
:1072B000ECE92E2EEFEF3E2E4D2C552447FC50943A
:1072C000A5C000E01CEFAA24BB2470E2D72EACC0FE
:1072D000C90165E0880F991F6A95E1F7992019F0B7
:1072E00064E070E002C062E070E00E947F77462FA9
:1072F000062F055C37016A0C711CF3018081992708
:1073000087FD909555E0880F991F5A95E1F7B101D7
:107310000E947F77562F90E2D92ED60E2F5F3F4FD7
:107320008D2D90E09B838A834216530609F050C04E
:1073300082349105ACF48AE3C82EC40E625E8C2DB3
:1073400045E059830E94E9665981EA81FB81E13475
:10735000F10531F0652F615E8C2D45E00E94E966F4
:10736000FD2DF03430F4802F81506D2D45E00E94CA
:10737000E9662A813B812F33310594F401506D2D4C
:107380006F5F802F45E00E94E9668A819B818E3382
:10739000910531F06D2D6E5F802F45E00E94E9660A
:1073A0008091820490918304009741F4123631F069
:1073B000133621F0123411F0133439F5812FF30113
:1073C00060814CE924E60E94CE15F30180831DC044
:1073D0002A813B81213431052CF4615E802F43E00A
:1073E0000E94E9663D2D303428F4802F6D2D43E056
:1073F0000E94E9668A819B818F33910534F46D2D5B
:107400006F5F802F43E00E94E966A3942A2D30E04D
:10741000992019F089E090E002C085E090E02817FB
:1074200039070CF455CF4DCFC80160919B080E94DD
:107430008A37BCE3EB2EEA0C9C01A5E03695279534
:10744000AA95E1F76D2D621B8E2D0E949D66950118
:10745000237030702115310521F48E2D60E20E94D9
:107460009D660894A11CB11C005E1F4F90E4A916F4
:10747000B104D1F68CE560E040E40E94ED660F9027
:107480000F900F90CF91DF911F910F91FF90EF9090
:10749000DF90CF90BF90AF909F907F906F905F9064
:1074A0004F903F902F9008952F923F924F925F926E
:1074B0006F927F928F929F92AF92BF92CF92DF9204
:1074C000EF92FF920F931F93DF93CF93CDB7DEB769
:1074D000A2970FB6F894DEBF0FBECDBF8F8F98A3D3
:1074E0006A8B80918404882309F474C08091070515
:1074F000882319F08150809307058091B3069091FD
:10750000B4062091B1063091B206820F931F2091EC
:10751000B5063091B606820F931F2091B7063091C1
:10752000B806820F931F20914007309141072C012C
:10753000421A530A920157FE03C0309521953F4FDE
:1075400041E0213034073CF090934107809340079D
:1075500081E08093870480916F01863FD9F19091FB
:1075600008019233B8F190913D079F5F90933D07DA
:10757000903160F020913E0730913F072F5F3F4FE1
:1075800030933F0720933E0710923D079091870468
:10759000992321F010923F0710923E0720913E0759
:1075A00030913F07992787FD90950A9667E771E02C
:1075B000869FA001879F500D969F500D1124421762
:1075C000530740F4237030702130310519F480E105
:1075D0000E94847380916E01582F51705F5F5987AC
:1075E00081FF02C01D8602C063E06D876090A2012A
:1075F000662009F44AC08985E82FF0E0EE0FFF1FEE
:10760000E952FB4FA080B180CC24B7FCC094DC2CA5
:107610009D85E92FF0E0EE0FFF1FE952FB4F20811F
:107620003181442737FD4095542FCA01B9010E948A
:1076300040777B018C01C601B501A60195010E942E
:107640004077E60EF71E081F191F662D70E080E0D8
:1076500090E0EAE0660F771F881F991FEA95D1F73F
:1076600024E630E040E050E00E94B477B901CA015E
:107670000E9440776E157F058007910730F4C8019E
:10768000B7010E9452374C0102C088249924B401EA
:1076900080E090E024E630E040E050E00E94407757
:1076A0006B8F7C8F8D8F9E8F6AE2662E61E0762EC7
:1076B000A1EBB6E0BE8BAD8BFE013196F88FEF8B60
:1076C00050E0252E51E0352E2AE831E03F872E8705
:1076D00047ED54E05A8F498F2901F98BE88BBC8B19
:1076E000AB8BEE24FF241B865A89517059A3AE2C14
:1076F0008E2D0E94BD169C01D30111968D919C91F7
:107700001297281B390BB901882777FD8095982F90
:107710004AE0660F771F881F991F4A95D1F7121606
:1077200013062CF45D962D913C915E9703C0F301F6
:10773000278530892436310514F424E630E04427C7
:1077400037FD4095542F0E94B4778901FCEF21301A
:107750003F072CF024E00030120724F405C000E0BD
:107760001CEF02C000E014E08091700180FF0FC0A8
:1077700080916E0190E08170907042E050E0481B73
:10778000590BE416F50619F4109501951F4FA98DB4
:10779000BA8D0D931D93BA8FA98FC8010F968F31A3
:1077A0009105F0F4B4E0EB16F1047CF48A2D8F5FC0
:1077B0000E94126B90E00197E1E0F0E002C0EE0F52
:1077C000FF1F8A95E2F7CF0108C081E090E00E2C00
:1077D00002C0880F991F0A94E2F7FB85F82BFB87FC
:1077E0002A2D243008F07AC139A1332309F05FC073
:1077F0008091960181FF5BC06701CC0CDD1C44E6E3
:1078000051E0C40ED51ED60111968C911197807C43
:1078100009F44DC08C9185958595859561E040E092
:107820000E947E11882309F442C0D601EC91E770D2
:10783000F0E0DF01AA0FBB1FA457BB4FEE0FFF1FE5
:10784000E45AFE4F8D919C91119720813181821BCA
:10785000930B62E070E00E947F77F701EE0FFF1F4D
:10786000EB59FE4F2081422F440F440F459545951B
:10787000552747FD5095649FC001659F900D749FEB
:10788000900D11246FE170E00E947F77660F771FE3
:10789000660F771F2295269526952370213019F0C3
:1078A000223029F403C0060F171F01C08B01811479
:1078B000910409F1B985AB1619F0ED85AE16D9F42E
:1078C0006091A20170E080E090E04AE0660F771FCF
:1078D000881F991F4A95D1F79801442737FD409595
:1078E000542F0E9440772B8D3C8D4D8D5E8D0E94D4
:1078F000B477022F132FF201EA54FE4F808160E02B
:1079000040E00E947E11882369F0F201E954FE4FA5
:10791000808160E040E00E947E11882329F4CC241D
:10792000C39404C0CC2402C032E0C32E80916E0107
:1079300090E08170907022E0A22EB12CA81AB90AB2
:10794000AE14BF0469F580919B01807F49F1C801A5
:1079500080509C4F62E070E00E947F779B01EC2D8D
:10796000F0E0EE0FFF1FEE0FFF1FA701440F551FA2
:10797000CA01A3E0880F991FAA95E1F7841B950B14
:10798000E80FF91FEC5CFC4F6081772767FD70956D
:10799000C9010E943D2CAC01440F551F30E028C0A6
:1079A00031E0101611060CF430E08C2D90E0A701A8
:1079B000440F551FFA0163E0EE0FFF1F6A95E1F7D0
:1079C000E41BF50B880F991F880F991FE80FF91F0B
:1079D000E657FE4FE30FF11DE655FE4F6081772716
:1079E00067FD7095C8013AA30E943D2CAC013AA1F5
:1079F000EC2DF0E0EE0FFF1FEE0FFF1FB701660F3B
:107A0000771FCB0113E0880F991F1A95E1F7861BAA
:107A1000970BE80FF91FE657FE4FE30FF11DE455F2
:107A2000FE4F6081772767FD70956C597F4F8827DF
:107A300077FD8095982FDA019D01442737FD409509
:107A4000542F0E94407724E630E040E050E00E944E
:107A5000B477022F132FAE14BF0499F580919B01C8
:107A6000982F907F09F466C60050144063C6D10178
:107A7000ED91FC91119760818091700180FD61957D
:107A8000772767FD7095872F972F63587F4F8F4F0C
:107A90009F4F20E034E0201B310B442737FD4095F9
:107AA000542F0E94407720E038E040E050E00E94F0
:107AB000B4772030B8E03B07B0E04B07B0E05B079D
:107AC00039F4D101ED91FC912081332727FD3095C8
:107AD000220F331FE889F98931832083AB89BC8960
:107AE0000D931D93BC8BAB8B0894E11CF11CE2E061
:107AF000F0E06E0E7F1E288939892E5F3F4F398B4B
:107B0000288B2E0E3F1E4EE050E0440E551E57E0CF
:107B1000E516F10409F0EBCD00919F016B8506237A
:107B2000809142078095802319F088E10E94847338
:107B30000093420780E094E09093C0068093BF06D4
:107B40009093C2068093C106ECE8F4E02CE531E0A6
:107B5000A9ECB6E0BD0181919191D9014D915D9162
:107B60009D01841B950B880F991FDB018D939D93BD
:107B7000BD01B4E0E439FB0771F780919404909162
:107B80009504880F991F9093D2068093D106809117
:107B9000960490919704880F991F9093D406809330
:107BA000D3068091980490919904880F991F90931F
:107BB000D6068093D50680919A0490919B04880FF5
:107BC000991F9093D8068093D706EDEFF6E0FC87D7
:107BD000EB8729ED36E04191519161917191D90185
:107BE0004D935D939D01B7E0ED33FB07A1F7C09086
:107BF000A201CC2009F47AC0E985AE2EBB24AA0CE0
:107C0000BB1C21EB422E26E0522EA40CB51CD50144
:107C10002D903C90442437FC4094542CBD850B2F70
:107C200010E0000F111F0F54194FF801208131810E
:107C3000442737FD4095542FCA01B9010E9440776F
:107C40003B014C01C201B101A20191010E944077A8
:107C5000660E771E881E991EDD24EE24FF248AE01E
:107C6000CC0CDD1CEE1CFF1C8A95D1F7C701B601B8
:107C700024E630E040E050E00E94B477B901CA0148
:107C80000E944077661577058805990578F5C40147
:107C9000B3010E945237BC0180E090E024E630E05E
:107CA00040E050E00E9440773B014C01C201B1012D
:107CB000A70196010E944077A40193010E94B47726
:107CC000D5012D933C93F80160817181882777FD60
:107CD0008095982FA70196010E944077A4019301F7
:107CE0000E94B477D80111963C932E93E090A001A6
:107CF0008E2D807E09F4DEC0B9852B2F30E0220F57
:107D0000331FF901EF54F94F40815181CE010196A3
:107D1000280F391FD901ED91FC91BD856B2F70E0C3
:107D2000660F771FDB01AF54B94F2D913C91860F41
:107D3000971FDC018D919C91BA89B1FD05C0E40FBC
:107D4000F51F280F391F04C020E030E0E0E0F0E02C
:107D5000A091A101AA2349F0B0E0AA0FBB1FA15531
:107D6000B94F0D911C91119702C000E010E0E2FEA6
:107D700003C0F095E195FF4FE3FE03C030952195D8
:107D80003F4FE4FE03C0109501951F4F8091A00165
:107D9000829586958770823071F1833020F481302E
:107DA00009F088C007C0833009F459C0843009F055
:107DB00081C06CC0C90168E070E00E947F777B01E0
:107DC000C90160E870E00E947F7729014E185F08C2
:107DD0007201E61AF70AC90160E072E00E947F773B
:107DE000E61AF70AC8018E1B9F0B9093C406809376
:107DF000C306CF0120C0CF0168E070E00E947F770A
:107E00007B01CF0160E870E00E947F773F016E1830
:107E10007F087301E61AF70ACF0160E072E00E9462
:107E20007F77E61AF70AC801821B930B9093C4066A
:107E30008093C306C90162E070E00E947F77600F03
:107E4000711FCB018E0D9F1D9093C6068093C506B2
:107E50006E197F097093C8066093C7062BC0C801CE
:107E60008E1B9F0B9093C4068093C306E00FF11FF7
:107E7000CF01820F931F9093C6068093C506E21B25
:107E8000F30BF093C806E093C70614C0C8018E1B1D
:107E90009F0B9093C4068093C306C801820F931F63
:107EA0009093C6068093C506021B130B1093C80659
:107EB0000093C70680918404882311F00E94C8347F
:107EC00080E4EDEFF6E0DF011D928A95E9F7BA89CB
:107ED000B1FF2DC080916E0190E08170907022E022
:107EE00030E0281B390B80E090E0ED89FE89AF89F6
:107EF000B88D2817390729F01182108211961C922B
:107F00001E920196329612968430910591F7109246
:107F1000CA061092C9061092CC061092CB06109297
:107F2000CE061092CD061092D0061092CF068CE6A7
:107F300093E090930101809300019C012F5F3F4FDC
:107F400030930301209302019C012E5F3F4F309339
:107F50000501209304010396909307018093060185
:107F600023E0422E28E0522E93E8692E97E0792EE6
:107F700083E4282E87E0382E19861D8689850E9485
:107F8000170F7C01FC0180818150803108F0ADC267
:107F9000838161E040E00E947E11D2019C918823A0
:107FA000A1F4292F1C92F7019181892F88508230EA
:107FB00008F08AC287818E70843009F485C29930B6
:107FC00009F04BC000E01CEF4AC021E0911120E015
:107FD00081E0D2018C93D7011196EC913E2F315064
:107FE000832F90E0DC01AA0FBB1FAF54B94F0D9156
:107FF0001C911197343160F0B9853B1748F4DC01CE
:10800000AA0FBB1FAA0FBB1FA350B94F0D911C9104
:10801000D70117963C911797832F807381F0832F98
:108020008295837090E0019741E050E002C0440FD8
:10803000551F8A95E2F7CA015D85582B5D8736FF8B
:108040000EC0E53060F4F0E0EE0FFF1FE250FF4F8E
:10805000C70108969183808302C000E010E0D70139
:108060001796CC901797C6FC0BC018968C91189752
:10807000882331F02AA30E94FA0E080F191F2AA1A3
:10808000F7018681882321F48581882309F458C16A
:10809000D3016D917D918D919C911397222389F449
:1080A00020E031E040E050E00E94B47750954095E8
:1080B000309521953F4F4F4F5F4F4801820E931EE1
:1080C0005AC08C2D8E70843051F5D701EC91F0E0C0
:1080D000EE0FFF1FE952F94F60817181882777FD0C
:1080E0008095982F20E034E640E050E00E944077F1
:1080F000F3016083718382839383D70112962C915D
:108100001297222361F0332727FD3095432F532FF9
:108110000E94B477F3012083318342835383D301D8
:108120006D917D918D919C91139720E031E040E01D
:1081300050E00E94B47750954095309521953F4F7F
:108140004F4F5F4F4801820E931E8114910499F0A6
:10815000F701258197FE22952F7030E044E650E02C
:10816000249FC001259F900D349F900D1124D101B3
:1081700011969C938E93F10180819181009799F0E3
:1081800020918404222319F0019791838083D101E7
:108190008D919C911197009731F0F301608171816D
:1081A00082819381B7C08114910409F4C9C0D701B9
:1081B00016968C911697882309F4B4C08091840494
:1081C000882309F476C012962C9112972223B1F0DD
:1081D000332727FD309537FF03C0309521953F4F5A
:1081E000332727FD3095432F532F60E070E080E266
:1081F00093E00E94B47759016A0106C0A12CB12C0A
:10820000F0E2CF2EF3E0DF2EF70186811814190477
:10821000FCF48F7090E00097F1F144E650E0849F09
:108220009001859F300D949F300D1124442737FD18
:108230004095542FC601B5010E94B477F3018081A7
:108240009181A281B381280F391F4A1F5B1F2CC067
:1082500082958F7090E00097F1F044E650E0849FA3
:108260009001859F300D949F300D1124442737FDD8
:108270004095542FC601B5010E94B47759016A0197
:10828000D3012D913D914D915C9113972A193B0992
:108290004C095D0909C09801442737FD4095542FCA
:1082A000542F432F322F2227F3012083318342831F
:1082B0005383D3016D917D918D919C9120E031E0AC
:1082C00040E050E00E94B477C801AA2797FDA0952E
:1082D000BA2F1814190434F482179307A407B507AA
:1082E00034F012C0281739074A075B076CF42227BD
:1082F00017FD2095322F322F212F102F0027F30149
:108300000083118322833383D3016D917D918D91FD
:108310009C91139720E031E040E050E00E94B47758
:1083200089010EC0C801AA2797FDA095BA2FBA2FC0
:10833000A92F982F8827F30180839183A283B38389
:10834000D70114966C911497633061F1643028F46E
:10835000613051F06230A0F444C0653069F165309D
:1083600038F1663081F52BC0F7018181893029F41D
:1083700017FD35C0005012400EC017FF32C02CC090
:10838000D70111968C911197893041F4101611067E
:1083900004F100501E4F000F111F23C010161106CC
:1083A000DCF01FC017FF1DC0109501951F4F19C0AD
:1083B0001016110674F010C017FF0EC010C0101672
:1083C00011063CF00CC06750C8010E948A378C012E
:1083D00008C000E014E005C000E010E002C000E0CA
:1083E0001CEFF701878180FD13C0E181EE2381F04E
:1083F000E53070F4F0E03197EE0FFF1F21E030E040
:108400002C0F3D1FE20FF31F80819181080F191F70
:10841000B801882777FD8095982FD70112962C9167
:108420001297332727FD3095432F532F0E94407713
:10843000F701008110E00150104027812695277038
:10844000213071F0F801EE0FFF1FEE0FFF1F2230F9
:1084500069F5E350F94F608371838283938334C05D
:1084600024E630E040E050E00E94B477E22EC32ED4
:10847000DA01000F111F000F111F0350194FF801EF
:1084800020813181428153816E2D7C2DCD010E944E
:10849000407720E034E040E050E00E94B477D8011B
:1084A0002D933D934D935C9313970EC0E350F94F7A
:1084B0002081318142815381260F371F481F591F68
:1084C0002083318342835383B985BF5FB987089482
:1084D000411C511CE4E0F0E06E0E7F1E22E030E013
:1084E000220E331EB03209F049CD0E940F0F8C01CD
:1084F000ED84E0FE05C0882319F48EE10E948473A8
:10850000E1FE0BC0C80190708034910519F08834E9
:10851000910519F48FE10E948473E2FE0DC0107082
:108520000038110531F00838110519F0003911052E
:1085300019F480E20E948473B5EE4B2EB4E05B2EFA
:108540003F8D28A1832F922F9A8789872224332455
:10855000598A488AAB85BC85ED90FD900D911C91A0
:10856000C801B70124E630E040E050E00E94B47753
:10857000EB85FC852083318342835383A889B989A5
:108580002D933D93B98BA88BEE85FF85E35AFE4F63
:1085900080819181EE85FF85E55AFE4F2081BAE00A
:1085A0002B0260011124E8EEF3E0CE0EDF1EEE8513
:1085B000FF85E65AFE4F20812B0250011124A8E1CD
:1085C0004A2EACEF5A2EA40CB51C96014C2D232F2D
:1085D0008C159D0514F4482F292F842E922E8A1471
:1085E0009B040CF44501E114F1040105110569F146
:1085F0009401442737FD4095542F1E141F04100684
:10860000110654F4B601882777FD8095982F621BD8
:10861000730B840B950B0DC0C501AA2797FDA09580
:10862000BA2F29013A01481A590A6A0A7B0AC3017A
:10863000B201A80197010E94407720EA36E841E0A4
:1086400050E00E94B47779018A01C4010E94A31B03
:108650003C01882477FC8094982C6E0C7F1C801E33
:10866000911EC6010E94A31B8C01C5010E94A31B81
:10867000222717FD2095322F0615170528053905E5
:1086800014F438014901AA2797FDA095BA2F840157
:108690007301681679068A069B0614F47C018D0125
:1086A000EE85FF85E45AFE4F8081882341F01095C6
:1086B0000095F094E094E11CF11C011D111DFAE8F5
:1086C000CF2EF1E0DF2EC20CD31CF601E358FD4F94
:1086D0008081882389F060E040E00E947E11882339
:1086E00059F0F601E258FD4F80810E94FA0E7C019C
:1086F0000027F7FC0095102FF894A985BA85ED9214
:10870000FD92BA87A9877894EB85FC853496FC871F
:10871000EB87E2E04E2E512C240C351C2E853F8534
:108720002B5F3F4F3F872E8730E22316310409F03D
:1087300011CF04C08F7009F09AC9C3C9A2960FB6B1
:10874000F894DEBF0FBECDBFCF91DF911F910F9187
:10875000FF90EF90DF90CF90BF90AF909F908F9061
:108760007F906F905F904F903F902F900895EF9281
:10877000FF920F931F93DF93CF93CDB7DEB7C05413
:10878000D0400FB6F894DEBF0FBECDBF8E010F5F95
:108790001F4FC80163E00E94543A81E2E82EF12C99
:1087A000EC0EFD1EC70161E00E94543AE6EEF2E0D5
:1087B000418152816081D8012D913C91D7018D91E9
:1087C0009C911197662329F0B901681B790BCB01A5
:1087D00002C0821B930B840F951F73E0883E97079E
:1087E0002CF4ACEF89319A0724F005C088EE93E0B1
:1087F00002C088E19CEF9283818335960E5F1F4F04
:1088000062E070E0E60EF71E73E0E633F70781F6EC
:1088100080916E0190E08170907022E030E0281B22
:10882000390B80E090E02817390721F0FC01E4596A
:10883000FC4F1082019684309105A9F786E00E94D2
:108840002D6081E00E948473C05CDF4F0FB6F89406
:10885000DEBF0FBECDBFCF91DF911F910F91FF9073
:10886000EF9008952F923F924F925F926F927F9276
:108870008F929F92AF92BF92CF92DF92EF92FF9230
:108880000F931F93DF93CF9300D000D0CDB7DEB707
:1088900090916C01192F1F708038B9F18138A8F4BC
:1088A000833209F47EC0843230F4803221F1823286
:1088B00009F0C3C083C0853209F465C0853208F46D
:1088C0005DC0813609F0B9C092C0833809F483C015
:1088D000843838F4813809F49AC0823809F0ADC080
:1088E00080C0853809F457C0853808F43FC08F3BF5
:1088F00009F0A3C096C0153009F09FC0809188048C
:1089000091E089278093880488C0163049F5892F23
:1089100090E0807390708032910561F48091EB0E4D
:108920009091EC0E909581959F4F9093B006809317
:10893000AF0683C00097A1F480912A04807C803C1C
:1089400021F48BE99EE00E94247580912E04807CA6
:10895000803C09F072C08FE99EE00E9424756DC0D2
:108960000E94EC150E942B1680E805C082E196E378
:108970000E942B1684E80E94486A5FC0163009F0F6
:108980005CC0905F04C0163009F057C090519F73CF
:1089900090936C0142C08AE493E50E942B1685E80F
:1089A000EACF812F8F5F80936C01883010F0109296
:1089B0006C0181E00E942D6083E130C0112319F029
:1089C000812F815001C087E080936C0181E00E947B
:1089D0002D6084E123C089EC9BE10E941B1683E893
:1089E000CACF84E69CE10E941B1682E8C4CF809126
:1089F0002D06823021F483E080932D060EC01530C1
:108A000019F40E946A1609C01630B9F404C00E9415
:108A10007D350E946A160E941E7687E10E9484734B
:108A20000CC081E00E94486A83E00E94486A82E0AC
:108A30000E94486A81E080932C0880919E0160E04A
:108A400040E00E947E11882331F080912C08882319
:108A500011F40E94B74380919E0160E040E00E94C3
:108A60007E1180932C0880916C01803108F0D3C076
:108A70009091080180915901981710F496E001C077
:108A800094E0EAE8EE2EE1E0FE2E0AE0D7014D91F7
:108A90007D01802F60E024E09A830E944965055F94
:108AA0009A81083799F7492F406884E260E10E9473
:108AB000B20F84E268E146E50E94086680912D06C7
:108AC000882399F0823011F406E001C004E040915F
:108AD0002E0650912F068EE560E1202F0E94330F65
:108AE00083E368E140E00E94571040919C0183E0DD
:108AF0004802A00111244258574F84E260E123E06C
:108B000000E00E940C6680919B018F7031F089E338
:108B100060E14AE758E00E946B667EE0C72E71E094
:108B2000D72E60E0A62E61E0B62E662477245FE1A2
:108B3000E52EF60101916F01D501ED91FD915D01E9
:108B4000808187FD8D5F85958595843E0CF484EE4C
:108B5000F82E8D3114F04CE1F42E862D81508230A8
:108B6000F8F4802F64E046E30E94ED6620916E01E8
:108B700030E02625372520FD04C080919B018F70B1
:108B800061F4802F81506EE143E00E94ED66802FFA
:108B90008F5F6EE143E00E94ED669E2D9F1914C029
:108BA000802F8B516BE346E30E94E966802E8A9406
:108BB000882D6AE343E00E94E966882D6CE343E078
:108BC0000E94E9660F0D9BE33DEF832E800E2DEF93
:108BD000F22EF90E882D6F2D47E09A830E94ED66E4
:108BE0009A81692F6D5F882D47E00E94E966802F8A
:108BF0008D5F6F2D47E00E94ED66882D6F2D47E059
:108C00000E94E9660894611C711CB4E06B16710443
:108C100009F08FCF27C080E060E04AE851E02AE009
:108C200001E10E940C66909108018091590198170A
:108C300010F442E001C040E084E560E00E94B20F21
:108C400080912D06882371F0823011F402E001C07A
:108C500000E040912E0650912F068FE660E0202F15
:108C60000E94330F123008F08DC09BE0C92E95E0B2
:108C7000D92E00E089E1882E912CBBE1EB2EA0E2F9
:108C80004A2E512CF0E82F2E312CF60121913191F2
:108C90006F013C832B83113031F1802F83708E9DC7
:108CA000A02C1124F02EF694F694FF0CFF0CFF0C70
:108CB00038E2F30E8B819C81B2010E947F779B0189
:108CC0008B819C81B1010E947F77AB01421B530BCA
:108CD0008B819C81480F591F8A2D8F5D6F2D20E25B
:108CE0000E947F684AC0043018F4E2E2AE2E02C04F
:108CF0007EE5A72E802F8370F82EFF0CFF0CF80E58
:108D000096E2F90E8B819C8197FF03C09095819527
:108D10009F4F889DA001899D500D989D500D112455
:108D200040505E4F452F550F550B45954595642E88
:108D30004A3114F049E1642E8A2D89516F2D43E3A5
:108D400025E50E94BB666F2D62508A2D45E00E948A
:108D5000ED66EB81FC811E161F0614F4A39401C07E
:108D6000A6186F2D6F5F8A2D462D0E94E9666F2D24
:108D700061508A2D462D0E94E9660F5F083009F088
:108D800084CFAEC3163009F021C38091980E88239A
:108D900009F414C380912B088F5F80932B088233D2
:108DA00060F110922B080BE91EE037E2A32E38E0A9
:108DB000B32E23E2C22E28E0D22EEE24FF24D801C7
:108DC0008C91F50181935F01F2E0EF16F10444F418
:108DD0008E2D62E00E943A74D60111969C938E9378
:108DE0000894E11CF11C0C5F1F4FE2E0F0E0CE0E96
:108DF000DF1EF4E0EF16F10411F780916C0190E0B2
:108E0000807390708031910509F0C9C097E2A92E56
:108E100094E0B92E8FEA882E8EE0982E0CE9C02EB1
:108E20000EE0D02E13E2612E18E0712E222433249E
:108E300010E0D5018C91882309F453C001E0F301BF
:108E400080819181009709F400E0812F68E146E775
:108E500058E00E946B66F22C422D4F5C812F8A5F96
:108E600068E10E940866B2E14B2E410EF101E95D16
:108E7000F74F0464812F805F60E14081222DEE2452
:108E8000E3940E94A810F101EE0FFF1FEE0FFF1FE9
:108E9000E65DFB4F90819295969596959370812F04
:108EA000885E933041F4D4014D915C9160E220E002
:108EB0000E947F6809C060E2F6014081222D00E037
:108EC000EE24E3940E94A810842D8E5E60E2D60109
:108ED00011964C912F2D00E4EE24E3940E94A810EB
:108EE00010E40894211C311CE4E0F0E0AE0EBF1E3B
:108EF00026E030E0820E931ECE0EDF1E82E090E070
:108F0000680E791E92E02916310409F092CF809103
:108F1000990E882369F088E060E778E00E94636634
:108F20004091D30E8EE168E050E020E40E947F681B
:108F300080E36CE678E00E9463664091290880E156
:108F400068E250E024E40E947F684091A40E88E12A
:108F500068E350E020E00E947F684091A50E84E223
:108F600068E350E020E40E947F6880E460E348E624
:108F700058E00E946B6640912A0880E568E250E064
:108F800024E40E947F684091A80E88E568E350E0E1
:108F900020E00E947F684091A90E84E6FDC08032E7
:108FA000910509F0FFC08091990E882309F4A5C0AE
:108FB00080E164E678E00E946366E090CF0EF09076
:108FC000D00E8091960185FF13C097012E5E3F4F12
:108FD00083E790E0289F7001299FF00C389FF00CE8
:108FE0001124E6E0F594E794EA95E1F716E401C070
:108FF00013E48CE068E0412F0E94086686E168E097
:10900000A70124E40E947F6884E568E340E658E015
:109010000E946B6688E768E3412F0E9408664091D2
:10902000D50E5091D60E8091960185FF11C09A0100
:109030002E5E3F4F83E790E0289FA001299F500DAF
:10904000389F500D112476E0559547957A95E1F7B4
:1090500086E668E320E40E947F6886E360E14BE5F2
:1090600058E00E946B664091D10E5091D20ECA0119
:10907000880F991F35E0440F551F3A95E1F7481BBB
:10908000590B8EE468E024E40E947F6880E266E584
:1090900078E00E9463660091AF061091B00680915F
:1090A000EB0E9091EC0E080F191F80919601982FEE
:1090B00098719830A9F085FF15C0C80195958795DE
:1090C000959587959801220F331F200F311F820F2E
:1090D000931FA5E015950795AA95E1F7080F191FAD
:1090E00046E601C04DE682E168E10E94086688E13B
:1090F00068E1A80124E40E947F6880912704882306
:10910000C1F08091230890912408009711F003E0AA
:1091100001C000E080E362E578E00E9463660464D9
:1091200080E168E24091270820E0EE24E3940E9469
:10913000A81080912B048823C9F080912508909174
:109140002608009711F003E001C000E080E460E32E
:109150004EE458E00E946B66046482E568E2409148
:10916000280821E0EE24E3940E94A81088E36AE432
:1091700078E00E9463664091290882E168E350E04C
:1091800020E40E947F6880E368E346E458E00E94A0
:109190006B6640912A0882E468E350E020E40E9474
:1091A0007F689EC18033910509F0ADC080E161E424
:1091B00078E00E9463662091F10E3091F20E442710
:1091C00037FD4095542F80E360E100E1FBEFEF2E87
:1091D0000E94496780E360E14EE20E9408662091A8
:1091E000010F3091020F442737FD4095542F88E43A
:1091F00060E1ECEFEE2E0E94496788E16CE378E0D5
:109200000E9463662091EF0E3091F00E442737FDE7
:109210004095542F80E368E17BEFE72E0E94496779
:1092200080E368E14EE20E9408662091FF0E3091D3
:10923000000F442737FD4095542F88E468E19CEFE8
:10924000E92E0E94496780E267E378E00E94636646
:109250004091CD0E5091CE0E80E360E220E00E945E
:109260007F6888E269E278E00E9463664091ED0ED3
:109270005091EE0E80E368E220E00E947F6840910A
:109280001D0F88E768E250E020E00E947F6880E3DD
:109290006DE178E00E94636688E361E178E00E9416
:1092A00063661EE1C12E1FE0D12E10E070E394E250
:1092B00025C0133011F478E394E2D6012D916D01AD
:1092C00080910404281710F000E001C002E030E0B3
:1092D000220F331F442737FD4095542F0063892FF9
:1092E000672FA4E0EA2E79839A830E9449677981E7
:1092F0009A81153009F4F4C0965D1F5F80912A0FA2
:109300001817B8F2EDC0F7E2CF2EF4E0DF2EE3E25B
:10931000AE2EE8E0BE2E8824992415E1F601808166
:10932000882321F1D5012D913C911197211531050B
:1093300011F003E401C000E4812F68E24DE058E041
:109340000E946B66482D4F5C812F8A5F68E20E9405
:109350000866F401E95DF74F812F8E5E68E2408177
:10936000282DEE24E3940E94A8101BE40894811C8D
:10937000911CE4E0F0E0CE0EDF1E22E030E0A20E11
:10938000B31E32E08316910449F685E160E349E0BB
:1093900058E00E946B664091290887E260E350E044
:1093A00020E40E947F688BE460E345E058E00E947F
:1093B0006B6640912A088DE560E3EFCE86E168E2B6
:1093C0004DEF57E024E00E943C668AC0153008F05B
:1093D0007DC00E94A525123061F0812F880F810F7A
:1093E000880F8950912F9150192F110F190F110FBC
:1093F00002C080E016E0A82E992787FD90951C01F9
:10940000220C331C280E391E60E2F62ECC24DD24FB
:1094100052E0652E712C680E791E2C011AC00E9434
:1094200054104C018A2D60E040E00E947E11082F0C
:10943000A401420D531D8AE06F2D23E00E940C66AB
:109440000894C11CD11C83E090E0280E391E98E0DE
:10945000F90EA394C601840D951D68167906FCF6D5
:10946000812F992787FD90952C01440C551C480E9F
:10947000591E30E2F32ECC24DD2422E0822E912CE2
:10948000880E991E3C011AC00E9454105C01812F65
:1094900060E040E00E947E11082FA501440D551D9B
:1094A00085E66F2D23E00E940C660894C11CD11C38
:1094B000A3E0B0E04A0E5B1EB8E0FB0E1F5FC601E2
:1094C000860D971D88169906FCF60AC040918A04FD
:1094D00050918B048CE368E224E004E00E94330F97
:1094E0000F900F900F900F90CF91DF911F910F91E0
:1094F000FF90EF90DF90CF90BF90AF909F908F90B4
:109500007F906F905F904F903F902F900895181626
:109510001CF0109205050895282F332727FD30955C
:1095200090910505291B3109462F50E0421753073A
:1095300024F4861B80930505089546505040241757
:10954000350724F48A5F861B809305050895AF9242
:10955000CF92DF92EF92FF920F931F93DF93CF93FF
:109560000F92CDB7DEB7182F83EA9CE00E94C21B92
:1095700086E898E0612F42E02BED37E00BE05EEAF1
:10958000E52E5CE0F52ECC24B6E0AB2E0E943A1D11
:10959000F09086088F2D67E00E94874A88E068E98E
:1095A0007CE00E94636631E08F2D813009F030E06D
:1095B0008091A00182958695877090E0AC01440F60
:1095C000551F480F591F440F551F4758534F84E5E7
:1095D00068E026E0032F39830E940C66398133232B
:1095E00099F06091A001629566956770812F40E0C7
:1095F00024E00E94CE158295880F807E9091A00174
:109600009F71982B9093A00180E16EE67CE00E9410
:10961000636601E0EF2DE23009F000E084E560E1EF
:109620004091A101202F0E94B80F002349F0812F03
:109630006091A10140E026E20E94CE158093A10135
:1096400088E163E67CE00E9463664091A201FF2D01
:10965000F33011F421E401C020E484E568E150E036
:109660000E947F688F2D833049F4812F6091A20181
:1096700040E024E60E94CE158093A2010091A00153
:1096800006950695017080E265E57CE00E946366C0
:10969000CF2CDD24C7FCD09421E0E4E0CE16D10429
:1096A00009F020E084E560E2402F0E94051DFF2DB7
:1096B000F43079F4812F602F40E021E00E94CE1534
:1096C0008170880F880F9091A0019B7F982B9093B9
:1096D000A0010091A001069506950695017088E20B
:1096E00067E47CE00E94636621E085E0C816D1044F
:1096F00009F020E084E568E2402F0E94051DEF2D6F
:10970000E53081F4812F602F40E021E00E94CE15EA
:109710008170880F880F880F9091A001977F982BF8
:109720009093A0010091A0010295017080E369E38C
:109730007CE00E94636621E0F6E0CF16D10409F0D8
:1097400020E084E560E3402F0E94051D8F2D8630C8
:1097500079F4812F602F40E021E00E94CE158170C6
:109760008295807F9091A0019F7E982B9093A0017D
:109770000F90CF91DF911F910F91FF90EF90DF90AD
:10978000CF90AF900895AF92BF92CF92DF92EF92B9
:10979000FF920F931F93DF93CF930F92CDB7DEB756
:1097A000D82E82E09EE00E94C21B88E898E06D2DD2
:1097B00041E02BED37E00BE0E8E0EE2EEEE0FE2E90
:1097C0007BE0C72E50E1A52E0E943A1D109188081B
:1097D000F0908908812F67E00E94874A2091570105
:1097E00030E02F5F3F4F442737FD4095542F8AE2EA
:1097F00060E001E192E0E92E0E9449672D2D2534B9
:1098000051F0263418F4243401F511C03D2D3436BE
:1098100071F03536D1F41130C1F4FF20B1F08091F0
:109820000605882391F08091890881500CC0113081
:1098300061F44F2D493048F480910605882329F0C2
:10984000809189088F5F809389088091050588231E
:1098500009F088C088E06DEF7DE00E9463661130FA
:1098600031F481E090E020910605222311F080E0A0
:1098700090E0082F00618CE368E04AE851E02AE0BC
:109880000E940C6680910605882359F48091090591
:1098900087FF07C081E080930605109209051092AA
:1098A000890880910605882381F0209109053327D6
:1098B00027FD30958F2D90E08217930734F4109296
:1098C00006051092090510928908113009F04DC063
:1098D00080910605882309F448C0809189089091F9
:1098E0000905891B8093890887FF02C010928908A7
:1098F000809189088A301CF089E080938908109251
:109900000905AF2CBB24F501E657FE4F80810E946C
:10991000A932682F209182043091830421153105EA
:1099200049F47D2D723631F0733621F0723411F026
:10993000733431F48D2D40E021E40E94CE15682F60
:10994000862F0E94B932482FF501E657FE4F8083DB
:109950008F2D880F8F0D880F845C68E021E00E94B6
:10996000496503C008E0E02E02C0B0E1EB2E809113
:109970000505823008F084C08E2D67EF7DE00E94DF
:1099800063664091970150919801123099F4FF203D
:1099900039F480910605882309F01AC421E019C41E
:1099A0008F2D813039F480910605882329F020E03D
:1099B00002E004C020E00DC420E001E087E46E2D49
:1099C0000E94330F123009F059C080910605882398
:1099D00039F48091820490918304009709F44EC079
:1099E000FF2029F09F2D913009F048C022C08091BE
:1099F000970190919801ACE3AA2EB12CB5010E9479
:109A00006B778D2D40E02BE30E94CE152CE3482F81
:109A10004203900111248091970190919801B50122
:109A20000E946B77280F391F30939801209397017C
:109A300025C080919701909198016CE370E00E949D
:109A40006B77082F0E5F8D2D602F41E02EE30E9473
:109A5000CE15081B602F772767FD70952091970121
:109A600030919801261B370B309398012093970172
:109A700037FF04C0109298011092970168E0E60E3B
:109A8000809105058330F8F48E2D6FEE7DE00E9405
:109A9000636601E0133009F000E08CE36E2D402F87
:109AA0000E945710002349F08D2D6091950147ECDD
:109AB00029E30E94CE158093950178E0E70E8E2D64
:109AC000893308F088C3809105058430C8F58E2D50
:109AD00068EE7DE00E94636691E0143009F090E04A
:109AE00080919601282F217030E0A901440F551F65
:109AF000E3E0220F331FEA95E1F7420F531F4D5267
:109B0000524F8CE36E2D2AE0092F99830E940C6638
:109B10009981992379F06091960161708D2D40E0D3
:109B200021E00E94CE158170909196019E7F982B26
:109B30009093960198E0E90EEE2DE93308F04BC3BF
:109B400080910505853030F500919B010F708E2DB9
:109B50006CEC7DE00E94636621E0153009F020E0A6
:109B60008CE36E2D402F0E94F51C153069F48D2D6D
:109B7000602F40E021E00E94CE158F7090919B01F4
:109B8000907F982B90939B01F8E0EF0E2E2D2933B8
:109B900008F021C380910505863040F500919B01B6
:109BA00002950F708E2D65EC7DE00E94636621E0CA
:109BB000163009F020E08CE36E2D402F0E94F51C3A
:109BC000163071F48D2D602F40E021E00E94CE15FB
:109BD0008295807F90919B019F70982B90939B0121
:109BE00038E0E30E4E2D493308F0F5C280910505AB
:109BF000873050F58E2D6CEB7DE00E94636691E01E
:109C0000173009F090E040919C0186E04802A001E5
:109C100011244356524F8CE36E2D26E0092F998371
:109C20000E940C669981992349F08D2D60919C01C9
:109C300040E024E00E94CE1580939C0168E0E60E8F
:109C40007E2D793308F0C7C280910505883008F56C
:109C50008E2D65E97DE00E94636601E0183009F011
:109C600000E086E36E2D40919E01202F0E9404109B
:109C7000002349F08D2D60919E014AEE26E10E945D
:109C8000CE1580939E0188E0E80E9E2D993308F052
:109C9000A2C280910505893008F051C08E2D6CE874
:109CA0007DE00E9463669CE3AA24BB24A5014C5777
:109CB000524FFA1411F4193061F020919F0130E0F5
:109CC0000A2C02C0359527950A94E2F7022F0170FD
:109CD00001C002E0892F6E2D21E099830E940C665D
:109CE0000894A11CB11C99819A5F9636F9F6193037
:109CF00001F5ED2DE03631F08091820490918304DE
:109D00000097B9F08D2D0E94486A1092060581E0F7
:109D100090E00F2C02C0880F991F0A94E2F720915F
:109D20009F01282720939F0182E00E942D600E94BE
:109D3000C960F8E0EF0E2E2D293308F04CC2809157
:109D400005058A3008F0E3C08E2D6EE77DE00E94A5
:109D500063664091990186E0489FA00111244B5908
:109D6000524F1A3041F4FF2031F4809106058823C8
:109D700021F002E003C000E001C001E084E26E2DAA
:109D800026E00E940C6680919901882321F083309F
:109D900009F04DC009C086E66E2D40E65DE020E08A
:109DA0000E943C669CE308C082E76E2D4DE55DE0B5
:109DB00020E00E943C6698E440919A01552747FDB7
:109DC0005095440F551F440F551F485B524F1A3092
:109DD00049F43F2D313031F480910605882321F07C
:109DE00002E003C000E001C001E0892F6E2D24E0F5
:109DF00099830E940C669981892F865D40919D010F
:109E000092E34902A0011124445D5E4F1A3049F4E7
:109E10006F2D623031F490910605992321F022E0F4
:109E200003C020E001C021E06E2D0E947F68809178
:109E30009901813001F582E46E2D49E35DE020E077
:109E40000E943C6640919A01552747FD50954F5F0F
:109E50005F4F1A3049F47F2D713031F4809106053F
:109E6000882321F022E003C020E001C021E08EE73A
:109E70006E2D0E947F681A3009F043C0809106055C
:109E8000882331F480918204909183040097C9F172
:109E90008F2D813079F0813018F0823091F522C019
:109EA0008D2D6091990140E023E00E94CE158093B2
:109EB000990127C080919901882311F0833031F4F2
:109EC0008D2D60919A014EEF24E007C08130C9F4D6
:109ED0008D2D60919A0140E02CE70E94CE15809371
:109EE0009A010FC080919901882311F0833049F4C1
:109EF0008D2D60919D014CEF2AE00E94CE1580933C
:109F00009D0198E0E90EEE2DE93308F064C18091DF
:109F100005058B3008F07AC080919901882311F0F3
:109F2000833019F58E2D6AE27DE00E9463664091D0
:109F3000A30185E04802A00111244F515F4F1B305F
:109F400011F421E201C020E28EE46E2D0E947F68B0
:109F50001B3009F055C08D2D6091A3014CEE24E11A
:109F60000E94CE158093A3014BC08130B9F401E06B
:109F70001B3009F000E080E06E2D44E15DE0202F11
:109F80000E943C660023E1F1FD2DF038C9F581E027
:109F90008093640E80E00E94847332C08E2D6BE04B
:109FA0007DE00E94636680919A0187FD03C0833043
:109FB0001CF403C080E001C082E080939A0149E074
:109FC0008402A00111244151534F1B3031F4809180
:109FD0000605882321F002E003C000E001C001E093
:109FE0008CE36E2D29E00E940C661B3049F48D2D08
:109FF00060919A0140E022E00E94CE1580939A0180
:10A0000028E0E20E3E2D393308F0E5C080910505C9
:10A010008C3098F58E2D65EE7CE00E94636631E011
:10A020001C3009F030E08091A001817090E0AC011B
:10A03000440F551F480F591F4252534F8CE36E2D4A
:10A0400023E0032F39830E940C663981332379F092
:10A050006091A00161708D2D40E021E00E94CE153D
:10A0600081709091A0019E7F982B9093A00148E071
:10A07000E40E6E2D693308F0AEC0809105058D3079
:10A0800040F50091A001069501708E2D64ED7CE0F5
:10A090000E94636621E01D3009F020E08CE36E2D04
:10A0A000402F0E94F51C1D3071F48D2D602F40E073
:10A0B00021E00E94CE158170880F9091A0019D7FB4
:10A0C000982B9093A00178E0E70E8E2D893308F04D
:10A0D00082C0809105058E3040F50091960106956D
:10A0E00001708E2D6CEC7CE00E94636621E01E30D6
:10A0F00009F020E08CE36E2D402F0E94F51C1E30ED
:10A1000071F48D2D602F40E021E00E94CE1581700A
:10A11000880F909196019D7F982B9093960198E0DF
:10A12000E90EEE2DE93308F056C0809105058F3019
:10A1300048F5009196010695069501708E2D63EC09
:10A140007CE00E94636621E01F3009F020E08CE390
:10A150006E2D402F0E94F51C1F3079F48D2D602F3D
:10A1600040E021E00E94CE158170880F880F909109
:10A1700096019B7F982B90939601F8E0EF0E2E2D81
:10A18000293348F580910505803128F58091070530
:10A19000882319F421E0103109F020E080E06E2DD1
:10A1A0004FEA5CE00E943C661031A9F43D2D303846
:10A1B00091F41092060589E18093070580E80E94DA
:10A1C000486A1092210680E995E30E942B1603C08D
:10A1D00022E000E0F3CB0F90CF91DF911F910F9120
:10A1E000FF90EF90DF90CF90BF90AF9008956F9267
:10A1F0007F928F929F92AF92BF92CF92DF92EF9217
:10A20000FF920F931F93DF93CF930F92CDB7DEB7DB
:10A21000B82E8DE490E10E94C21B8EE998E06B2D70
:10A2200047E02BED37E00BE05DE5E52E50E1F52E44
:10A23000CC24C3941CE0A12E0E943A1D80909E085D
:10A240008A94D0909F08882D66E00E94874A18E083
:10A25000CC24992487FC9094909105059C0D9C300A
:10A2600009F463C1E92EFF248E149F0439F4809110
:10A270000605882329F0B2E0AB2E04C0AA2402C050
:10A28000AA24A39480E0612F4AE450E122E000E098
:10A2900099830E940C669981993010F048E301C0BF
:10A2A00041E3490F8CE0612F0E940866F701EE0F31
:10A2B000FF1FEE0DFF1DEE51FC4F408187E0489FD0
:10A2C000A00111244951504FDD2011F000E001C0E0
:10A2D0000A2D88E1612F27E00E940C66C701880FD4
:10A2E000991F8E0D9F1D86579E4FFC01E85AFD4F0A
:10A2F0002081253008F40AC1FC01EA5AFD4F2830BC
:10A3000008F40DC140819D2D913009F04DC04EC023
:10A3100020E001C02A2D88E4612F0E94B80FC701F8
:10A32000880F991F8E0D9F1D86579E4FFC01EA5A7C
:10A33000FD4F2081FC01E95AFD4F253254F0408148
:10A34000552747FD509543585F4FED2DE23041F4BE
:10A3500009C04081552747FD5095FD2DF23011F081
:10A3600020E001C02A2D88E7612F0E947F6800E06D
:10A3700035C020E001C02A2D88E4612F0E9404101E
:10A38000F701EE0FFF1FEE0DFF1DEF51FC4F408157
:10A390008D2D823011F020E001C02A2D80E6612F42
:10A3A0000E94041001E01AC020E001C02A2D88E4B8
:10A3B000612F0E94B80FF701EE0FFF1FEE0DFF1D7A
:10A3C000EF51FC4F40819D2D923011F020E001C0F3
:10A3D0002A2D86E6612F0E94B80F02E080910605C3
:10A3E000882339F48091820490918304009709F4C2
:10A3F00086C0AA2009F483C0ED2DE130D1F1E1300F
:10A4000020F0E23009F07BC046C03701660C771CB3
:10A410006E0C7F1C82EE93E0680E791E8B2DF3018B
:10A42000608140E02DE00E94CE15F3018083202F53
:10A4300030E0853028F0883030F481E090E005C0CD
:10A4400080E090E002C082E090E02817390709F42C
:10A4500056C0C701880F991F8E0D9F1D86579E4FAE
:10A46000FC01EA5AFD4F1082895A9D4FFC0110826F
:10A4700046C0013041F0C701880F991FE80EF91E50
:10A4800080EE93E031C03701660C771C6E0C7F1CA8
:10A4900080EE93E01AC0013089F0C701880F991F40
:10A4A0000230F1F0E80EF91E81EE93E0E80EF91E9D
:10A4B0008B2DF701608143E82DE71DC03701660C45
:10A4C000771C6E0C7F1C81EE93E0680E791E8B2D3D
:10A4D000F30160814AEE26E10E94CE15F3010EC021
:10A4E000E80EF91E81EE93E0E80EF91E8B2DF701C0
:10A4F000608140E026E20E94CE15F7018083C3947C
:10A50000185FFC2DF73009F0A7CE0FC08A5A9D4F77
:10A51000FC014081FD2DF13009F0FACEFBCE4081E7
:10A520008D2D813009F025CF26CF0F90CF91DF916F
:10A530001F910F91FF90EF90DF90CF90BF90AF9061
:10A540009F908F907F906F9008956F927F928F92DF
:10A550009F92AF92BF92CF92DF92EF92FF920F93B2
:10A560001F93CF93DF93982E8FE590E10E94C21B3B
:10A5700080EA98E0692D48E02BED37E00BE0AFE68C
:10A58000EA2EA0E1FA2ECC24C394F0E1AF2E0E9473
:10A590003A1D6090A0086A948090A108862D66E01C
:10A5A0000E94874AE8E0FE2EDD24772467FC709441
:10A5B000409105054D0D403109F45DC0A42EBB242A
:10A5C0004F5F80E06F2D20E00E94E40FEE24E50154
:10A5D000CC0FDD1FC85FDB4F8501000F111F095F26
:10A5E0001B4F6A147B0471F48E1461F4809106058C
:10A5F000882359F48091820490918304009739F460
:10A6000021E001C020E0CC2405C022E001C021E00F
:10A61000CC24C394EE2091F48EE16F2DF80140819B
:10A620000E940410CC20D9F0892DF80160814AEEF7
:10A6300026E10E94CE15F801808311C0488155277C
:10A6400047FD509580E66F2D0E947F68CC2039F041
:10A65000892D688143E82DE70E94CE158883E39415
:10A66000FE2DF33009F0BDCFD39488E0F80EED2D28
:10A67000E73009F09DCFDF91CF911F910F91FF90AF
:10A68000EF90DF90CF90BF90AF909F908F907F9092
:10A690006F900895AF92BF92CF92DF92EF92FF92A8
:10A6A0000F931F93DF93CF9300D0CDB7DEB7182F52
:10A6B00090917901992321F08AEF913011F403C030
:10A6C0008BEF58E101C05BE19150923030F49091F2
:10A6D000700197FF02C05D5F8350F82EF50E8EE388
:10A6E0009BE059830E94C21B8DE398E0612F40E0FC
:10A6F00021EF37E006E05981E52E0E942824D09012
:10A700003D08C0903E088D2D67E00E94874A609109
:10A7100005055981852F90E0462F50E09C01275078
:10A7200030404217530761F42D2D30E0049728176D
:10A73000390714F48FEF01C081E0680F60930505BD
:10A74000113629F1123678F4143409F448C015345E
:10A7500020F4123408F46AC063C0153419F11036BD
:10A7600009F064C009C0143608F45AC01436B9F1AF
:10A77000153609F05BC016C0DD2009F457C081E032
:10A7800090910605911180E0809306054FC080915D
:10A790000605882309F44AC01092060581E60E9446
:10A7A000486A44C02D2D213059F4CC2049F08091C5
:10A7B0000605882329F080913E08815080933E0849
:10A7C0002D2D30E08F2D992787FD9095281739077B
:10A7D00069F5CC2059F180913E0881501EC03D2D75
:10A7E000313061F48C2D893048F48091060588233E
:10A7F00029F080913E088F5F80933E082D2D30E038
:10A800008F2D992787FD90952817390779F49C2D6E
:10A81000973060F480913E088F5F80933E0806C0B9
:10A8200080910605882311F410923E088091050559
:10A83000882309F089C088E063E37BE00E946366B7
:10A84000ED2DE13031F481E090E0209106052223E6
:10A8500011F080E090E0082F006182E468E04BE7AF
:10A8600051E02AE00E940C6680910605882359F485
:10A870008091090587FF07C081E08093060510924B
:10A88000090510923E0880910605882381F02091E9
:10A890000905332727FD30958C2D90E0821793070B
:10A8A00034F4109206051092090510923E08FD2D11
:10A8B000F13009F04CC080910605882309F447C0A7
:10A8C00080913E0890910905891B80933E0887FF7F
:10A8D00002C010923E0880913E088A301CF089E048
:10A8E00080933E0810920905EC2CFF24F701E558EF
:10A8F000FE4F80810E94A932682F209182043091FE
:10A9000083042115310541F4123631F0133621F05C
:10A91000123411F0133431F4812F40E021E40E940D
:10A92000DD15682F862F0E94B932482FF701E558B0
:10A93000FE4F80838C2D880F8C0D880F8E5B68E016
:10A9400021E00E94496503C098E0F92E02C080E131
:10A95000F82E809105058230A0F5E0906D01E69417
:10A96000E694E69427E0E2228F2D6CE27BE00E94E1
:10A97000636691E03D2D323009F090E046E08E2D87
:10A98000849FA00111244F5F544F8CE56F2D26E06A
:10A99000092F9A830E940C669A81992381F0812F56
:10A9A0006E2D40E026E00E94DD158770880F880F2D
:10A9B000880F90916D01977C982B90936D0198E092
:10A9C000F90E80910505833058F5E09079018F2DBF
:10A9D00066EF7AE00E94636691E0ED2DE33009F0C6
:10A9E00090E046E0FE2DF49FA00111244751554F01
:10A9F0008CE56F2D26E0092F9A830E940C669A81C0
:10AA0000992341F0812F6E2D40E021E00E94DD1559
:10AA10008093790128E0F20E3F2D393308F0A8C465
:10AA200080917901813041F580910505843030F5C0
:10AA30008F2D6BED7AE00E946366409177018D2D3A
:10AA4000843011F421E401C020E486E66F2D50E04B
:10AA50000E947F689D2D943049F4812F6091770189
:10AA600041E024E60E94DD1580937701E8E0FE0EC8
:10AA7000FF2DF93318F07CC404E001C005E080919B
:10AA800079018150823038F580910505801710F5E5
:10AA90008F2D6BEC7AE00E94636640917801D016AE
:10AAA00011F421E401C020E486E66F2D50E00E94FD
:10AAB0007F68D01649F4812F6091780140E025E04D
:10AAC0000E94DD158093780128E0F20E3F2D393386
:10AAD00008F04EC40F5F80910505801720F58F2D7B
:10AAE00062EC7AE00E94636640915801D01611F43E
:10AAF00021E401C020E486E66F2D50E00E947F68CB
:10AB0000D01659F4812F609158014AE02DE20E943D
:10AB1000DD15809358010E94DF6888E0F80E9F2DB4
:10AB2000993308F025C4E02EE394809105058E1535
:10AB300008F58F2D62EB7AE00E946366409159011F
:10AB4000DE1411F421E401C020E486E66F2D0E949A
:10AB50009E0FDE1449F4812F6091590148E228E7E5
:10AB60000E94DD1580935901E8E0FE0EFF2DF933B8
:10AB700008F0FEC3E394809105058E1560F58F2DD6
:10AB800061EA7AE00E94636640916F01552747FDB4
:10AB90005095465F5F4FDE1411F421E401C020E4BC
:10ABA00086E66F2D0E947F688091A00D6F2D4DE687
:10ABB0000E940866DE1449F4812F60916F0146EF10
:10ABC0002EE60E94DD1580936F0128E0F20E3F2DE6
:10ABD000393308F0CDC3E394809105058E1550F507
:10ABE0008F2D66E97AE00E94636691E0DE1090E0C6
:10ABF0004091710150E0440F551F440F551F4757B6
:10AC0000554F86E66F2D24E0092F9A830E940C662B
:10AC10009A81992349F0812F6091710140E022E0EF
:10AC20000E94DD158093710188E0F80E9F2D993305
:10AC300008F09EC3E394809105058E15C8F48091B9
:10AC40007001817021E0DE1020E06F2D48E75AE0AE
:10AC5000012F0E94C3328170909170019E7F982BCA
:10AC600090937001E8E0FE0EFF2DF93308F080C3E9
:10AC7000E394809105058E15D8F480917001869536
:10AC8000817021E0DE1020E06F2D4CE65AE0012FAC
:10AC90000E94C3328170880F909170019D7F982B24
:10ACA0009093700128E0F20E3F2D393308F060C315
:10ACB000E394809105058E15E8F4809170018695E6
:10ACC0008695817021E0DE1020E06F2D4DE55AE081
:10ACD000012F0E94C3328170880F880F90917001FC
:10ACE0009B7F982B9093700188E0F80E9F2D9933ED
:10ACF00008F03EC3E394809105058E15F8F4809129
:10AD00007001869586958695817021E0DE1020E0A1
:10AD10006F2D4FE45AE0012F0E94C3328170880FDB
:10AD2000880F880F90917001977F982B90937001F6
:10AD3000E8E0FE0EFF2DF93308F01AC3E39480918A
:10AD400005058E1500F58F2D62E47AE00E9463669A
:10AD500001E0DE1000E080E66F2D40915B01202FC6
:10AD60000E940410002349F0812F60915B014AEE9C
:10AD700026E10E94DD1580935B0128E0F20E3F2D55
:10AD8000393308F0F5C2E394BB24809105058E1594
:10AD900008F048C0BB2019F462E37AE002C062E226
:10ADA0007AE08F2D0E946366BB2019F4A090720197
:10ADB00002C0A0907A01AA20A9F08A2D95E0899F6F
:10ADC000A0011124DE1411F421E401C020E486E680
:10ADD0006F2D0E947F688091A00D6F2D43E70E9428
:10ADE00008660AC001E0DE1000E086E66F2D4EE145
:10ADF0005AE023E00E940C66DE1439F4812F6A2D9C
:10AE000040E028E70E94DD15A82EBB2019F4A0928F
:10AE1000720102C0A0927A01E8E0FE0EFF2DF93324
:10AE200008F0A6C2E394B3942B2D223009F0ADCFE5
:10AE3000809105058E15F8F48091700182958F70D0
:10AE40008095817021E0DE1020E06F2D40E15AE016
:10AE5000012F0E94C332809581708295807F9091EE
:10AE600070019F7E982B9093700138E0F30E8F2D28
:10AE7000893308F07DC2E394809105058E15F8F4BE
:10AE80008091760182958F708095817021E0DE102F
:10AE900020E06F2D44E05AE0012F0E94C3328095DC
:10AEA00081708295807F909176019F7E982B909300
:10AEB000760198E0F90EEF2DE93308F059C2E394DA
:10AEC000809105058E15D8F480916D018095817073
:10AED00021E0DE1020E06F2D43EF59E0012F0E94AA
:10AEE000C3328095817090916D019E7F982B9093D5
:10AEF0006D01F8E0FF0E2F2D293308F039C2E394DD
:10AF0000809105058E15E8F480916D0186958095F8
:10AF1000817021E0DE1020E06F2D44EE59E0012F1A
:10AF20000E94C33280958170880F90916D019D7F42
:10AF3000982B90936D0138E0F30E8F2D893308F034
:10AF400017C2E394809105058E1508F086C08F2DF9
:10AF500069ED79E00E94636692E4AA24BB24A5010E
:10AF60004053564FE0918501F0E00A2C02C0F59560
:10AF7000E7950A94E2F7E170F070892F6F2D21E0D8
:10AF80000E2F9A830E940C660894A11CB11C9A8112
:10AF90009A5F923721F7DE1409F059C080913E087C
:10AFA00090910905891B80933E0887FF02C010928B
:10AFB0003E0880913E088A301CF089E080933E086C
:10AFC000109209058C2D880F8C0D880F4C2D50E0A8
:10AFD0004953564F8E5B6F2D21E002E00E940C66B4
:10AFE000103631F08091820490918304009779F1BA
:10AFF000812F0E94486A1092060581E090E002C00D
:10B00000880F991FCA94E2F7909185019827909331
:10B010008501803151F0803271F0883099F493FFCE
:10B0200002C09F7C0DC098600BC094FF02C0977D4A
:10B0300007C0906105C095FF02C0977E01C0906275
:10B040009093850181E00E942D600E94C96098E084
:10B05000F90EEF2DE93308F08BC1E39480910505DB
:10B060008E15F8F480916D01869586958095817096
:10B0700021E0DE1020E06F2D48EB59E0012F0E9407
:10B08000C33280958170880F880F90916D019B7FEE
:10B09000982B90936D01F8E0FF0E2F2D293308F0C7
:10B0A00067C1E394809105058E1500F590916D01BF
:10B0B000991F9927991F81E0891B21E0DE1020E06C
:10B0C0006F2D4AEA59E0012F0E94C332809587957F
:10B0D0008827879590916D019F77982B90936D01AC
:10B0E00038E0F30E8F2D893308F042C1E39480914C
:10B0F00005058E1508F580917001829586958770FB
:10B100008095817021E0DE1020E06F2D40EA59E04B
:10B11000012F0E94C332809581708295880F807EB6
:10B12000909170019F7D982B9093700198E0F90E9B
:10B13000EF2DE93308F01CC1E394809105058E15CD
:10B1400018F580917001829586958695837080951B
:10B15000817021E0DE1020E06F2D48E959E0012FD9
:10B160000E94C332809581708295880F880F807C01
:10B17000909170019F7B982B90937001F8E0FF0EE7
:10B180002F2D293308F0F4C0E39480917901815088
:10B19000823048F5809105058E1520F5C09070012C
:10B1A000CC1CCC24CC1C21E0DE1020E08C2D6F2D9B
:10B1B00047E859E0012F0E94C3328170282F27955C
:10B1C00022272795909170019F77922B9093700181
:10B1D000C81611F00E940F7738E0F30E8F2D8933D7
:10B1E00008F0C6C0E394809179018150823008F064
:10B1F00075C08091700187FF71C0CC24809175016A
:10B20000982F9F70209105052E1508F061C0CC2065
:10B2100029F4B92E8F2D6BE779E012C09C2D913067
:10B2200041F4B82EB294BFE0BB228F2D6FE679E0D7
:10B2300007C0B0907601EFE0BE228F2D63E679E083
:10B240000E94636691E0DE1090E0FB2D26E0F29F05
:10B25000A00111244E5F564F8CE56F2D092F9A8364
:10B260000E940C669A81992369F1812F6B2D40E031
:10B270002FE00E94DD15682FCC2031F4982F9F70AD
:10B2800080917501807F09C03C2D313051F4982F99
:10B290009295907F809175018F70892B80937501B5
:10B2A00008C0982F9F7080917601807F892B8093B2
:10B2B000760180917F04882329F08FE294E046E4B0
:10B2C0000E94117288E0F80E9F2D993308F050C04B
:10B2D000E394C394EC2DE33009F090CF8091050501
:10B2E0008E1508F045C086E06F2D4DEF58E00E94A6
:10B2F0006B66FF2DF83390F434E290E0832F6F2DCE
:10B3000040E957E0292F00E039839A830E94EA64DC
:10B310009A819F5F3981385E943081F728E0F20E80
:10B320003F2D393328F5CC24C394DE10CC24409132
:10B330006E014F5C82E16F2D2C2D0E94496594E2D5
:10B3400000E00F5F892F6F2D402F20E09A830E942D
:10B35000B80F9A81985E0430A1F7CC2049F0812F74
:10B3600060916E0140E023E00E94DD1580936E0144
:10B370000F900F90CF91DF911F910F91FF90EF9061
:10B38000DF90CF90BF90AF9008954F925F926F92F1
:10B390007F928F929F92BF92CF92DF92EF92FF9215
:10B3A0000F931F93DF93CF9300D0CDB7DEB7182F45
:10B3B0008CE391E10E94C21B88EB98E0612F46E08C
:10B3C0002BED37E00BE050E1E52E0E942824609041
:10B3D000B8086A94862D66E00E94874A103611F0FC
:10B3E000143641F467FC06C060929B088AEF97E32D
:10B3F0000E942B16CC24DD24EE24E39448E0F42EA6
:10B40000772467FC7094309105053C0DBB24B39400
:10B41000383028F4BB248E2D883028F074C09E2D3F
:10B42000973008F070C0032F10E091E060167106AD
:10B4300009F090E0DD2019F0DD24D39401C0D92E6D
:10B4400080E06F2D49E351E1292F3A8399830E94CF
:10B450003C663A819981393010F482E101C087E17C
:10B46000A8014F5F5F4F6F2D292F0E947F68BB207F
:10B4700079F008501040280133E0440C551C3A95EF
:10B48000E1F7400E511EE8E9F3E04E0E5F1E0BC0DF
:10B490002801440C551C440C551C400E511E80E7DD
:10B4A00093E0480E591E42010AE2F40141914F0116
:10B4B000552747FD5095802F6F2D20E00E947F6813
:10B4C0000B5E033991F7F8E0FF0EE394BB20B1F077
:10B4D00085E090E0480E591E0AE2F20141912F01E9
:10B4E000552747FD5095802F6F2D20E00E947F68E3
:10B4F0000B5E0E3791F7F8E0FF0EE394C3948C2DAA
:10B50000873009F080CFDD2029F4809105058F5F19
:10B51000809305050F900F90CF91DF911F910F91B0
:10B52000FF90EF90DF90CF90BF909F908F907F9093
:10B530006F905F904F900895AF92BF92CF92DF923D
:10B54000EF92FF920F931F93CF93DF93F82E8CE926
:10B5500098E06F2D4DE00E949925809194088823F2
:10B5600019F08BED9FE002C081ED9FE00E94C21BAD
:10B57000182F809195080E94170FEC01812F8A5F88
:10B5800060E0488120E00E94E40FA0909C088A2D92
:10B5900066E00E94874A18E0EE24BB24A7FCB09422
:10B5A000209105052E0D822F90E0DD24D394A8165E
:10B5B000B90609F0DD24263009F4FAC0273090F4EA
:10B5C000223009F457C0233030F4222309F121300E
:10B5D00009F0E8C134C0243009F499C0253008F0DE
:10B5E000BAC069C02A3009F46BC12B3038F4283056
:10B5F00009F420C1293008F044C1F1C02C3009F40D
:10B600009CC12C3008F47AC12D3009F0CBC1B2C1F5
:10B610008CE0612F4AEC5FE00E946B6684E5612F4D
:10B6200049812D2D0E94B80FDD2009F4BBC18F2D5B
:10B63000698141E026E20E94CE158983B3C18CE086
:10B64000612F43EC5FE00E946B664A81552747FDFE
:10B6500050952D2D206484E5612F0E947F68DD20A8
:10B6600009F4A0C18F2D6A8143E82DE70E94CE1511
:10B670008A8398C18F8186FF03C049EB5FE002C0D7
:10B6800042EB5FE08CE0612F0E946B664885552796
:10B6900047FD50952D2D206484E5612F0E947F6821
:10B6A000DD2009F47FC18F2D688543E82DE70E94D6
:10B6B000CE15888777C1CF80C294C694C694E3E044
:10B6C000CE2281E0C8228CE0612F47EA5FE00E9431
:10B6D0006B6643E09C2D949FA00111244056504F6F
:10B6E00084E5612F23E00D2D0E940C66DD2009F416
:10B6F00059C18F2D6C2D40E021E00E94CE15817044
:10B700008295880F880F807C9F819F7B90C08CE002
:10B71000612F4BE95FE00E946B668F81817090E042
:10B72000AC01440F551F480F591F4C56504F84E52C
:10B73000612F23E00D2D0E940C66DD2009F432C13B
:10B740006F8161708F2D40E021E00E94CE158170E5
:10B750009F819E7F6CC08CE0612F4DE85FE020E010
:10B760000E943C664C8183E0489FA0011124495906
:10B770005E4E84E5612F23E00D2D0E940C66DD20D6
:10B7800009F410C18F2D6C8140E026E10E94CE1596
:10B790008C83873008F406C19F2D903609F002C1D2
:10B7A000875080939B088AEF97E30E942B16FAC07C
:10B7B0008CE0612F46E85FE00E946B668EE4612FAB
:10B7C0004B812D2D0E940410DD2009F4EBC08F2D3C
:10B7D0006B814AEE26E10E94CE158B83E3C08CE09C
:10B7E000612F4EE75FE00E946B660F810295037048
:10B7F00049F02D2D206484E5612F402F50E00E94F8
:10B800007F6807C084E5612F4AE75FE02D2D0E9425
:10B810003C66DD2009F4C6C08F2D602F40E023E098
:10B820000E94CE1583708295807F9F819F7C982B8C
:10B830009F83B8C08CE0612F43E75FE00E946B6696
:10B840004F814695477050E063E0440F551F6A955D
:10B85000E1F7465A504F84E5612F28E00D2D0E94F4
:10B860000C66DD2009F49EC06F81669567708F2D90
:10B8700040E022E00E94CE158770880F9F81917F63
:10B88000D6CF8CE0612F4FE45FE00E946B664D8164
:10B8900042954F7080E6612F50E02D2D0E947F6809
:10B8A000DD2009F47FC06D8162956F708F2D40E0BF
:10B8B0002FE00E94CE158295807F9D819F701BC0D6
:10B8C0008CE0612F46E45FE00E946B664D814F7013
:10B8D00080E6612F50E02D2D0E947F68DD2009F465
:10B8E00061C06D816F708F2D40E02FE00E94CE15FA
:10B8F0008F709D81907F982B9D8354C08CE0612F29
:10B900004BE35FE00E946B664E8142954F7080E68C
:10B91000612F50E02D2D0E947F68DD2009F442C088
:10B920006E8162956F708F2D40E02FE00E94CE15E2
:10B930008295807F9E819F701AC08CE0612F42E3C8
:10B940005FE00E946B664E814F7080E6612F50E091
:10B950002D2D0E947F68DD2029F16E816F708F2D63
:10B9600040E02FE00E94CE158F709E81907F982B33
:10B970009E8318C08CE0612F40E25FE02D2D0E9475
:10B980003C66DD2079F08F2D803861F40E94486A92
:10B99000809195080E94B62781E00E94847380E020
:10B9A0000E94F615E394185F9E2D973009F0F8CDAC
:10B9B000DF91CF911F910F91FF90EF90DF90CF908B
:10B9C000BF90AF9008955F926F927F928F929F92F7
:10B9D000AF92BF92CF92DF92EF92FF920F931F939D
:10B9E000CF93DF93D82E80E291E10E94C21B86EBB9
:10B9F00098E06D2D45E02BED37E00BE077E2E72E88
:10BA000071E1F72E51E1C52E11E1A12E0E943A1DE0
:10BA1000F090B608FA948090B7088F2D66E00E94E7
:10BA2000874A8D2D803821F59F2D903108F5EF2D17
:10BA3000FF27E7FDF09580910505E81BF109EE0F62
:10BA4000FF1FE55FFA4FC081D1818F2D0E94270F24
:10BA5000FC01882069F48281882319F0D095C19572
:10BA6000DF4FD483C38382E00E942D600E94C960AF
:10BA700018E09924552453946F2C772467FC709414
:10BA800000910505090D003109F4E1C0802F0E94E5
:10BA9000270FEC018A816B817C81882319F07095D6
:10BAA00061957F4FA02EBB24F501EE0FFF1FE55FD0
:10BAB000FA4F20813181261B370B2333310524F0C7
:10BAC000F501EA55F74F08C09FEF2E3C39072CF4DB
:10BAD000F501EA55F74F85258083402F4F5F80E0C1
:10BAE000612F20E00E94E40FF501EA55F74F8081B5
:10BAF000882311F04FE701C04EE78BE4612F20E06F
:10BB00000E944965EE246A147B0471F48E1461F47A
:10BB100080910605882359F48091820490918304D2
:10BB2000009739F401E001C000E0CC2405C002E038
:10BB300001C001E0CC24C3948E2D823009F43FC0B3
:10BB4000833009F45DC08130C1F04B815C81202FCE
:10BB5000206280E3612F0E947F68CC2009F46BC0D3
:10BB60006B817C818D2D48E15CEF28EE33E002E0B3
:10BB70000E940A159C838B835EC0488144565527DA
:10BB800047FD509588E4612F202F0E947F68CC20CC
:10BB900009F451C06881645668838091A00181FFD7
:10BBA00004C08D2D43E82DE703C08D2D4CE924E61C
:10BBB0000E94CE15888388818C5988833CC0498136
:10BBC0004C59552747FD509586E6612F202F0E943E
:10BBD0007F68CC2081F169816C5969838091A001D3
:10BBE00081FF04C08D2D43E82DE703C08D2D4CE966
:10BBF00024E60E94CE1589838981845689831BC0DF
:10BC00008A8190E0AC01440F551F480F591F475ED1
:10BC10005E4E8CE6612F23E00E940C66CC2059F02A
:10BC20008D2D6A8140E021E00E94CE1591E08823AD
:10BC300009F490E09A83E3949E2D943009F063CF49
:10BC40009394185F892D873009F01ACF1FC001E047
:10BC50009F2D903109F000E080910705882311F0B5
:10BC600020E001C0202F82E1612F48E051E10E94D5
:10BC70003C66002359F08D2D803841F489E1809392
:10BC8000070580E80E94486A0E94B743DF91CF9180
:10BC90001F910F91FF90EF90DF90CF90BF90AF90EA
:10BCA0009F908F907F906F905F900895F89420916F
:10BCB000CE0D3091CF0D7894C9010895CF93DF93C5
:10BCC000CAE2D1E080E6FE0111928A95E9F78AE0A6
:10BCD00080932A0189E1809358018AE58093590174
:10BCE00081E080936E012196FE0120E032E080E841
:10BCF00091E02193319395878487938F828F41E0E0
:10BD0000E933F407B1F78BE791E069E072E14AE0CB
:10BD100050E00E94D57780E090E029913991820F20
:10BD2000931FE1E0C334DE07C1F79093560180937F
:10BD30005501DF91CF9108951F93CF93DF9381EC4D
:10BD400098E060E00E9489626AE271E080E6FB01AF
:10BD500011928A95E9F781EC98E040E650E00E9464
:10BD60001563182FCBE7D1E088810E94A9320E9489
:10BD7000B9328993F1E0C538DF07B1F780912A0124
:10BD80008A3028F4809167048160809367048AE098
:10BD900080932A011D3468F0EBE2F1E020E030E00E
:10BDA00081919191280F391F81E0E334F807C1F7A1
:10BDB00002C020E030E081E04091550150915601F1
:10BDC0004217530709F080E0DF91CF911F9108954A
:10BDD0001F93182FEAE8F1E025EA32E0DF01C901FC
:10BDE0001D920197E9F7CF016EEF71E14AE050E053
:10BDF0000E94D577812F90E001966AE070E00E9462
:10BE00007F77605D60938F01805D809390018AE011
:10BE10008093940180E00E941F6B1F910895CF9240
:10BE2000DF92EF92FF920F931F93DF93CF930F92C6
:10BE3000CDB7DEB76B01803160F5682F6F5F81ECA5
:10BE400098E049830E9489624981042F10E0C6016D
:10BE500060E270E050E00E94F67781EC98E0B60175
:10BE60004AE050E00E9415638A30910591F481EC1C
:10BE700098E00E947B62F601E00FF11F2AE030E0BB
:10BE800006C0B9010E946B77805D8293CB01009759
:10BE9000C1F70F90CF91DF911F910F91FF90EF901D
:10BEA000DF90CF9008958F5F0E940C6208951F93DA
:10BEB000CF93DF93182F8031A0F5682F6F5F81EC4F
:10BEC00098E00E9489626AE871E025EA32E0FB01AD
:10BED000C90111920197E9F781EC98E045EA52E037
:10BEE0000E9415638F3F910509F018F4812F0E947D
:10BEF000E85ECAE8D1E088810E94A9320E94B93286
:10BF0000899391E0C439D907B1F78AE0809394010D
:10BF10000E946A1680912C0F806480932C0F0E94DF
:10BF20000F77DF91CF911F9108950F931F93DF93A8
:10BF3000CF93CDB7DEB760970FB6F894DEBF0FBED4
:10BF4000CDBF682F6F5F062F0AC0102F1F5F812F94
:10BF5000688B0E940C626889882329F0012F0031C8
:10BF6000A0F3003139F181EC98E00E948962602FE2
:10BF70006F5F8AEC98E042E028E532E00E94FB63C4
:10BF80008E010F5F1F4F06C08AEC98E0B8010E9437
:10BF90007663A89581EC98E0B8014FE050E00E94EC
:10BFA000A462482F882381F78AEC98E00E942464D9
:10BFB00081E001C080E060960FB6F894DEBF0FBE4E
:10BFC000CDBFCF91DF911F910F910895EF920F9305
:10BFD0001F930E94F761882341F00E94626187FDF0
:10BFE00004C00E949C5E882381F58EEE91E161E0A1
:10BFF0000E94D9138CED91E10E94C0130E94D1617F
:10C000000E945E5E81EC98E060E041E02AE231E06F
:10C0100000E610E078ECE72E0E945364803691052C
:10C0200029F08DEC91E160E00E94D91380E00E943C
:10C03000E85E81EC98E061E042E02AE831E005EA60
:10C0400012E058ECE52E0E945364809157010E9443
:10C05000575F1F910F91EF900895882359F09091A9
:10C06000DD08982B9093DD080E940F0F9093DF0856
:10C070008093DE080895EF920F931F93CF93DF9381
:10C080001091DD08112309F47EC0882309F076C0E1
:10C090000E940F0F2091DE083091DF08AC01421B97
:10C0A000530B4436510508F46EC068C081E080939C
:10C0B000DC08812F90E0EC01C470D07012FF03C047
:10C0C00023E02093DC081092DD0880FF1CC083ED84
:10C0D00098E061E141E02AE231E000E610E0F4E1BD
:10C0E000EF2E0E9453648036910511F480E020C049
:10C0F0008091D908823021F48091DD08816029C0C7
:10C100008DEB91E135C081FF36C083ED98E061E1B0
:10C1100042E02AE831E005EA12E0E4E1EE2E0E9476
:10C12000536452E0853A950739F4809157018F5F47
:10C1300061E10E941A621FC08091D9088230A1F487
:10C140008091DD08982F92609093DD08209719F078
:10C1500086608093DD080E940F0F84569040909374
:10C16000DF088093DE0807C0209729F48DEA91E16B
:10C1700060E00E94D9131092DC0805C08091DC08B1
:10C18000882309F493CFDF91CF911F910F91EF9006
:10C1900008950AC081E00E943B608091620E833066
:10C1A00019F4A8951092620E8091DD08882391F70A
:10C1B0000895DF93CF930F92CDB7DEB7682F70E06D
:10C1C00084E0660F771F8A95E1F7CE01019641E082
:10C1D00050E00E94FD7789810F90CF91DF91089503
:10C1E000DF93CF930F92CDB7DEB76983682F70E0EE
:10C1F00094E0660F771F9A95E1F7CE01019641E032
:10C2000050E00E941C690F90CF91DF91089580EE5D
:10C2100098E060E070E040E450E00E941C690895FE
:10C2200082EE98E062E070E041E050E00E941C691C
:10C2300008950F931F93182F082F04C0802F0E947A
:10C24000D960082F802F0E94D9608823B9F7802FEA
:10C250006091E2080E94F0601093E2080E94106171
:10C260001F910F9108951F931091E208112359F027
:10C27000812F0E94D9608093E2080E941061812F73
:10C2800060E00E94F060812F1F910895F894209142
:10C29000CE0D3091CF0D7894C9010895EF92FF92A1
:10C2A000CF93DF938091E208C0E0D0E003C02F96E7
:10C2B0000E94D9608823D9F7CE01DF91CF91FF90FA
:10C2C000EF900895CF92DF92EF92FF920F931F931A
:10C2D000CF93DF9380E8E0E2F9E0DF011D928A95D9
:10C2E000E9F704EE18E0C0E0D0E08C2FC43139F457
:10C2F000D090E20832EEE32E38E0F32E0BC07E0140
:10C30000EE0CFF1CEC0EFD1E24EE38E0E20EF31ED8
:10C31000D801DC9090E0C82EC3941DC08D2D8450B0
:10C320008C3738F4ED2DF0E0E05EF64F8081882305
:10C3300061F0992329F0892F60E00E94F0600DC020
:10C34000F70110820E94076108C0C0828D2D0E94F3
:10C35000D9609D2DD82EDD2009F721960D5F1F4F46
:10C36000C531D10511F604E0E02FF0E0E05EF64FB4
:10C370008081882349F4802F6091E2080E94F06058
:10C380000093E2080E9410610F5F003869F780E0B7
:10C39000DF91CF911F910F91FF90EF90DF90CF90A1
:10C3A00008951F9380E4E0EEF8E0DF01982F1D92DE
:10C3B0009A95E9F794E09093E0088093E10880E192
:10C3C0008093E30884E001C0812F182F1F5F612F45
:10C3D0000E94F0601038C1F78FE760E00E94F060C3
:10C3E00084E08093E2080E9407611F91089580EE27
:10C3F00098E060E070E040E450E00E94FD778091BA
:10C40000E008843039F481E09091E108903419F02B
:10C4100080E0089580E0089590E0FC01EE0FFF1F9A
:10C42000E80FF91FE052F74F81E09481992309F456
:10C4300080E00895DF93CF9300D00F92CDB7DEB7A1
:10C4400090E0FC01EE0FFF1FE80FF91FDE011196CF
:10C45000EC51F74F23E001900D922150E1F770E08D
:10C46000DC01AA0FBB1FA80FB91FFB01EE0FFF1FB6
:10C47000E60FF71FAC51B74FEC51F74F83E0019037
:10C480000D928150E1F7FB01EE0FFF1FE60FF71F42
:10C49000EC51F74FDE01119683E00D90019281502F
:10C4A000E1F70E9407610F900F900F90CF91DF91FD
:10C4B0000895DF93CF930F92CDB7DEB790E09C0144
:10C4C000220F331F280F391FF901E052F74F8481E3
:10C4D0002C51374F93E0D9011D929A95E9F7898342
:10C4E0000E9407618981882311F00E9419610F90D1
:10C4F000CF91DF910895FC01808190E0FC01EE0F67
:10C50000FF1FE80FF91FEB51F74F918180819F705A
:10C510000895FC0160831282118270E0CB01880FC4
:10C52000991F860F971FDC01A052B74F14962C91CC
:10C53000149723831482158216828A51974FFC0127
:10C54000808182958F7008958F929F92AF92BF9253
:10C55000CF92DF92EF92FF920F931F93DF93CF93CF
:10C560000F92CDB7DEB78C015B01FC01808190E0BA
:10C57000FC01EE0FFF1FE80FF91FEB51F74F808111
:10C580002181922F9F70F80121813281821B930BB0
:10C59000E42EF52E8E159F0508F47C0167014E01EF
:10C5A0000894811C911C25C0F8016381662321F148
:10C5B00084818F5F848370E0B4E0660F771FBA9543
:10C5C000E1F7680F711DC40141E050E00E94FD7762
:10C5D0008981F50181935F01F80184818F3030F00A
:10C5E000148283810E94D960F80183830894C10872
:10C5F000D108C114D104C1F6F801818192818E0D58
:10C600009F1D8C199D09928381838E2D8C190F900B
:10C61000CF91DF911F910F91FF90EF90DF90CF901E
:10C62000BF90AF909F908F9008958F929F92AF92FE
:10C63000BF92DF92EF92FF920F931F93CF93DF93FE
:10C640008C015B017A01C0E0D0E045E0842E912CA2
:10C65000880E991E3BC0F801858190E08F7790701D
:10C66000009741F4C801B40141E050E00E94A46287
:10C67000813079F5F80145813FE7D32ED4222D2D65
:10C6800030E0C7018C1B9D0B8217930710F4DE2C42
:10C69000DC1AB5016C0F7D1F47FF08C0CB0160E0BD
:10C6A00070E04D2D50E00E94F6770AC0C8014D2D74
:10C6B00050E00E94A4628D1519F0C80FD11D09C069
:10C6C000CD0DD11DF80185818D198583CE15DF052E
:10C6D00010F2CE01DF91CF911F910F91FF90EF905B
:10C6E000DF90BF90AF909F908F9008959F92AF92F0
:10C6F000BF92CF92DF92EF92FF920F931F93CF934F
:10C70000DF93EC018B01C42E8B81882389F489810E
:10C710009A81009769F4E880FF240E9433618B833B
:10C72000F701EE0FFF1FEE0DFF1DE052F74F848360
:10C73000DC2C6FE0962E44C0EF80F8840E940F0F2F
:10C74000E81AF90AF7FE02C082E004C08B81882350
:10C7500019F481E08E8337C09C819F3080F01C8269
:10C760000E94D960882339F4EB800E943361682FDE
:10C770008E2D0E94F0608B810E94D9608B838B810B
:10C78000882339F36C81992D961BED2C9D1508F4A7
:10C79000E92EAE2CBB2470E06F5F7F4F90E054E039
:10C7A000880F991F5A95E1F7680F791FC801A501F5
:10C7B0000E941C690A0D1B1D8C818E0D8C83DE1856
:10C7C000DD2009F0B9CF2C2D30E02D1931098981F8
:10C7D0009A81820F931F9A8389838C2D8D19DF9103
:10C7E000CF911F910F91FF90EF90DF90CF90BF906E
:10C7F000AF909F9008950F931F93CF93DF93EC0119
:10C80000890168831A82198270E0CB01880F991F11
:10C81000860F971FFC01E052F74F24812B831C8267
:10C820001D821E82FC01EB51F74F10824295407F22
:10C8300041830E940F0F080F191F18870F83DF9184
:10C84000CF911F910F9108951F93CF93DF93EC0128
:10C85000888190E0FC01EE0FFF1FE80FF91FEB51FC
:10C86000F74F898180839A819F708181807F892B96
:10C8700081838B81882389F00E94D960182F8823B7
:10C8800061F08B8160E00E94F0600E9407611123DB
:10C8900031F0812F0E94196102C010E0F6CFDF91C4
:10C8A000CF911F9108954F925F926F927F929F92C6
:10C8B000AF92BF92CF92DF92EF92FF920F931F93AE
:10C8C000DF93CF930F92CDB7DEB75C0129016801EA
:10C8D0002E2D30E00E94FB631982720100E010E00F
:10C8E00081E03E010894611C711CF70191917F0168
:10C8F000992341F4882349F49081992349F4992498
:10C9000093941EC0882371F403C09924939401C0AA
:10C91000992499819F3718F40C151D0561F588231A
:10C9200079F001C099248981882321F18068898365
:10C93000C501B30141E00E9476638130D1F025C08A
:10C9400089818823B9F0C501B30141E00E94766373
:10C950008130D9F44981B801641B7109640D751DDA
:10C96000C5010E9476639981891719F0981B9983F4
:10C970000CC01982892D99819F5F99830F5F1F4F8A
:10C98000C016D10608F0B1CF05C089818F77680144
:10C99000C81AD108C5010E942464C6010F90CF9126
:10C9A000DF911F910F91FF90EF90DF90CF90BF909C
:10C9B000AF909F907F906F905F904F90089580E030
:10C9C00094E0E0EAF9E0DF019C011D922150304043
:10C9D000E1F708950F931F93CF93DF93DA01119638
:10C9E000FA014491ED012196FD01A491B0E0179662
:10C9F00013E0B595A7951A95E1F71A2FDE01119668
:10CA0000FE019491929FE0011124AC0FBD1F00FD27
:10CA100008C001FF08C09091D00D51E096FD04C000
:10CA200002C051E001C050E066956695669570E0E1
:10CA30009B013695322F22273795279590E0280FB6
:10CA4000391F610F711D7695762F6627779567954B
:10CA5000680F791F042F10E014C0E901C056D64FAB
:10CA600080E090E008C0FD01E80FF91FE49151114A
:10CA7000E095E99301968417B0F3A00FB11F2058F9
:10CA80003F4F2617370749F7DF91CF911F910F913D
:10CA90000895FF920F931F93CF93DF93942F463106
:10CAA0003CF4440F490F440F22FFABC0440FA9C010
:10CAB000482F4A5F092F112707FD109520FD09C057
:10CAC00021FF0AC03091D00DFF24F39436FD05C03C
:10CAD00003C0FF24F39401C0FF2466956695669514
:10CAE00070E07695762F662777956795680F711DAC
:10CAF000EB01C056D64F22FF4FC09E3209F04A5F6D
:10CB0000C801809760E170E00E947F7780EA90E042
:10CB1000689F9001699F300D789F300D1124C801E6
:10CB2000880F991F53E0000F111F5A95E1F7800FEE
:10CB3000911F280F391F26543D4E85E0882369F048
:10CB4000F9019491E056FF4F54912F5F3F4FF90147
:10CB50006491E056FF4F749104C060E050E090E0B3
:10CB600070E0FF2021F09095609550957095DE0162
:10CB7000AF57BF4FFDE0A03ABF0740F498836983E9
:10CB8000FE01E058FF4F50837C93229681508F3FE7
:10CB9000C1F12F5F3F4FD2CF23FF0DC0FF2011F017
:10CBA0008FEF01C080E06056764FFB0180832196B5
:10CBB0004F5F91E001C090E09801220F331F220FD8
:10CBC000331F200F311F29583E4E85E0F9012F5F9A
:10CBD0003F4FE491992311F0843039F0FDE0C03AE1
:10CBE000DF0718F4F110E095E993815079F75DE0E3
:10CBF000C03AD50730F4FF2011F08FEF01C080E07C
:10CC00008883842FDF91CF911F910F91FF9008951A
:10CC100020E00E9449650895CF92DF92EF92FF9243
:10CC20000F931F93CF93DF93162FF22EF0E1EF2E89
:10CC3000E022C42EE6016E01D52EE6010CC0EE20E6
:10CC400011F0488102C0FE014491612F202F0E9403
:10CC50004965FA942196FF2091F7DF91CF911F91BA
:10CC60000F91FF90EF90DF90CF9008950F9300E029
:10CC70000E940C660F910895CF92DF92FF920F935E
:10CC80001F93CF93DF93162F022FA0E1FA2EF222EB
:10CC9000C42EE6016E01D52EE601FF2011F0488179
:10CCA00002C0FE0144912196442329F0612F202FD8
:10CCB0000E944965F2CFDF91CF911F910F91FF90B4
:10CCC000DF90CF900895982FAB0180E0692F20E08E
:10CCD0000E943C66089520E00E943C660895EF9211
:10CCE000FF920F931F93DF93CF930F92CDB7DEB7D1
:10CCF000182F062F7A01982F9C5E95504E2D4F705D
:10CD00004A301CF0495C28E002C0405D20E0892FD9
:10CD1000602F99830E9449659981911731F0B4E0A1
:10CD2000F694E794BA95E1F7E8CF0F90CF91DF91B1
:10CD30001F910F91FF90EF900895E62FE695E695ED
:10CD4000E695F0E0F695FE2FEE27F795E795E80FCC
:10CD5000F11DE056F64F8DE0E03AF80758F46770A1
:10CD600081E090E002C0880F991F6A95E2F7208168
:10CD700028272083089547FF02C0840F4195E62F9E
:10CD8000E695E695E695F0E0F695FE2FEE27F79509
:10CD9000E795E80FF11DE056F64F6770A1E0B0E0AF
:10CDA00001C0AA0F6A95EAF711C08DE0E03AF807D2
:10CDB00078F4822F90E09C013595279580FF04C080
:10CDC00080818A278083206841503196442369F707
:10CDD00008952FEF0E94BB6608950F931F93CF9382
:10CDE000DF93C82FD0E0E62FE695E695E695F0E0D4
:10CDF000F695FE2FEE27F795E795EC0FFD1FE05611
:10CE0000F64F062F10E0242F332727FD3095200FF3
:10CE1000311FC90168E070E00E947F777695762F18
:10CE20006627779567956C0F7D1F6056764F077064
:10CE3000107081E090E002C0880F991F0A95E2F718
:10CE400081959081892708C0E058FF4F8DE0E03A36
:10CE5000F807D0F4808180958083E617F707A0F368
:10CE60008DE0E03AF80780F4C90168E070E00E94C4
:10CE70007F7721E030E002C0220F331F8A95E2F76E
:10CE80002195808182278083DF91CF911F910F911F
:10CE900008952F923F924F925F926F927F928F925E
:10CEA0009F92AF92BF92CF92DF92EF92FF920F9339
:10CEB0001F93DF93CF9300D00F92CDB7DEB7182F1B
:10CEC000662E59016A01F02E802F05FF04C004FF71
:10CED00004C002E003C000E001C001E0E7FE04C0BE
:10CEE000E1942224239401C02224D7FE0BC0D094C5
:10CEF000C094B094A094A11CB11CC11CD11C4424AA
:10CF0000439401C0442482FF06C09CE09093A00D8E
:10CF10003AE0932E05C096E09093A00D25E0922E66
:10CF200086FF2FC04110190D28EEA21623E0B2068D
:10CF300020E0C20620E0D20614F0190D06C034E647
:10CF4000A316B104C104D10414F0190D06C08AE07F
:10CF5000A816B104C104D1040CF0190D002391F0FE
:10CF6000023039F4E4E6AE16B104C104D10454F43D
:10CF7000190DFAE0AF16B104C104D1041CF4190D67
:10CF800001C0191B8091A00D810F8093A00D02306C
:10CF900011F420EFF20E5524539492E0792E882458
:10CFA0002E2D332727FD3095862D8A5F89833B837D
:10CFB0002A8370C0C601B5012AE030E040E050E0AD
:10CFC0000E94B477E62E80E3382E3E0C812F662D2A
:10CFD000432D2F2D0E9449650515D9F5F2FE23C07A
:10CFE0008E2D8150833008F47394C601B5012AE078
:10CFF00030E040E050E00E94B477CA01B9012AE075
:10D0000030E040E050E00E94B477623011F06430CC
:10D01000C1F4E32DE43319F4812E839413C0812EDF
:10D020008A9473940FC01250812F8F5FF0FE05C059
:10D03000662D47E00E94ED6605C069810E949D66ED
:10D0400001C0812EFAE0AF16B104C104D1040CF086
:10D0500000E0C601B5012AE030E040E050E00E9467
:10D06000B47759016A01211531054105510581F453
:10D07000002331F0023059F4252D223040F408C04D
:10D08000F4FE10C0222021F430EFF30E01C000E0C6
:10D0900019195394852D90E0EA81FB81E817F9076F
:10D0A0000CF088CF882061F0662D645F882D472DB5
:10D0B0000E94E966662D635F882D472D0E94E96610
:10D0C000442039F0812F8919662D4DE22F2D0E94C1
:10D0D00049650F900F900F90CF91DF911F910F91A5
:10D0E000FF90EF90DF90CF90BF90AF909F908F9088
:10D0F0007F906F905F904F903F902F900895EF92A8
:10D100000F93022FFA019F01442737FD4095542FBA
:10D1100075E0E72E0E9449670F91EF90089520E097
:10D120000E947F680895A998AB98AC988BBBAD9A84
:10D13000AD98AB9AA99A089520E030E006C045E08A
:10D140004A95F1F700002F5F3F4F28173907BCF3CE
:10D150000895AA9885E08A95F1F7000085E08A9500
:10D16000F1F70000AA9A8CED95E00E949C6882EE8F
:10D170000E9493688EEA0E94936881EA0E949368F5
:10D1800086EA0E94936884EA0E94936882EA0E9479
:10D19000936880EC0E9493688FE20E94936885E216
:10D1A0000E94936881E80E94936882E20E949368DB
:10D1B0008FEA0E94936882E28093580108951F933A
:10D1C000182F81E80E949368812F0E9493681F9115
:10D1D00008951F93CF93DF9310E0C0EAD9E084E075
:10D1E0000E94936880E10E949368812F806B0E9467
:10D1F0009368A998AB9AAC98FE0180E290819BBBA2
:10D20000AD9AAD9891819BBBAD9AAD9892819BBB35
:10D21000AD9AAD9893819BBB3496AD9AAD988150F1
:10D2200069F7C058DF4FAB9AA99A1F5F1830B9F65B
:10D23000DF91CF911F910895BF92CF92DF92EF922D
:10D24000FF920F931F93CF93DF93EA01E82EF92EFD
:10D25000062F172F21C0F701B1907F0168010894B4
:10D26000C11CD11C04C0009739F00E94F3198091B1
:10D27000DC0890E082709070E199F5CF1FBB0EBB87
:10D28000E09A8DB3B81631F0BDBA8FB7F894E29A30
:10D29000E19A8FBF219786012097E9F6DF91CF9120
:10D2A0001F910F91FF90EF90DF90CF90BF90089566
:10D2B0008093D10D08958091D10D1092D10D0895D4
:10D2C000FC018081982F990F9E70807F892B80832D
:10D2D000662321F09160807F892B808381818F5F1D
:10D2E00081839281992391F020812F7079F4933674
:10D2F00059F0242F20622093D10D903111F4803108
:10D3000018F080818F7C8083118212828281883024
:10D3100009F443C0893058F4813009F446C08130A3
:10D32000A0F08230D1F1843009F052C036C08F3580
:10D3300049F1803620F4803109F04AC02EC0813690
:10D3400089F0823609F044C03DC08081982F9F70DB
:10D350009F30F1F591E6928391819131E0F08F7CDD
:10D36000808319C040664093D10D9081892F8295AA
:10D370008F708F5F83708295807F9F7C982B9083C6
:10D380008FE508C08181883111F4406818C0883267
:10D39000F9F480E18283118208959181903328F01D
:10D3A00090E09595879582831182828190E0019724
:10D3B000218130E082239323009751F4406440930D
:10D3C000D10D08958181803418F088E08283118224
:10D3D00008958E3091056CF4FC01EE0FFF1FE80FED
:10D3E000F91FEC55F24F90819F7081E09F30E9F575
:10D3F0003FC0823131F1833160F48F30C9F0803128
:10D4000018F48E3091F52AC0803161F0813169F5D0
:10D4100013C0843151F08431D0F08531E1F0863190
:10D4200021F51EC091B194701DC093B390781AC0BD
:10D4300090916300917016C09091630090959870E0
:10D4400011C08091630083FF12C091B102C091B1FD
:10D450009095907407C091B1907104C093B3F9CFC7
:10D4600091B1907281E0992319F480E0089580E0F1
:10D4700008958F708E3058F490E0FC01EE0FFF1F7E
:10D48000E80FF91FEC55F24F82E68283118208956E
:10D490008F708E3068F490E0FC01EE0FFF1FE80FF4
:10D4A000F91FEC55F24F83E6828380818F7C808365
:10D4B00008950F931F93CF93DF938091CE0D90919A
:10D4C000CF0D01969093CF0D8093CE0D8091D00D0E
:10D4D0008F5F8093D00D06B3009540E050E010E0E0
:10D4E00001C0AE01EA012196CA01880F991F840F7D
:10D4F000951FB8010C2E02C0759567950A94E2F746
:10D50000617070708C55924F50E00E946069C63017
:10D51000D10539F700B30095C0E0D0E0FE01E65830
:10D52000F44EE4919E012A5F3F4FC901880F991F75
:10D53000820F931F8C55924FE02361E009F460E065
:10D540009E012A5F422F50E00E9460692196C830F8
:10D55000D10521F7DF91CF911F910F910895FF928F
:10D560000F931F93CF93DF93F82EE4EAF1E080E06E
:10D5700090E0582F9C014081F41638F0442329F0A4
:10D5800001963A9681329105A1F75032B9F1E9013D
:10D59000CC0FDD1FC901A3E0880F991FAA95E1F701
:10D5A000C80FD91F8E010C551E4FA9014F5F5F4F49
:10D5B000CA01880F991FE3E0440F551FEA95E1F770
:10D5C000840F951F20953095205E3F4FA901440F91
:10D5D000551F63E0220F331F6A95E1F7420F531F77
:10D5E0008C559E4FB8010E94E4778AE0D8011D92C5
:10D5F0008A95E9F7C657DE4FFA8E02C004EA11E0B9
:10D60000C801DF91CF911F910F91FF90089580E4A1
:10D6100091E0E4EAF1E0DF019C011D9221503040ED
:10D62000E1F70895E0916E01F0E0EE0FFF1FEE0FBD
:10D63000FF1FE80FF11DE151FB4F84910895EF9218
:10D64000FF920F931F93DF93CF9300D000D0CDB7FD
:10D65000DEB719821A821B821C82E0917301F0E00E
:10D66000E852FB4F26E030E091E0E491EE2EFF24FB
:10D67000DE0111960FC06F5F7F4F0617170711F479
:10D68000FA01908364307105B1F79F5F22503040FA
:10D69000953089F060E070E0A701022E02C0559538
:10D6A00047950A94E2F7437050708A010F5F1F4F4D
:10D6B0004A0F5B1FE0CF882361F50E94076B8981C9
:10D6C0000E94AF6A8C0181E00E94126BF801818395
:10D6D00024E6F22EF2828A810E94AF6A8C0182E0F7
:10D6E0000E94126BF8018183F2828B810E94AF6AE3
:10D6F0008C0183E00E94126BF8018183F2828C819D
:10D700000E94AF6A8C0184E00E94126BF801818351
:10D71000F2820F900F900F900F90CF91DF911F9199
:10D720000F91FF90EF9008956F927F928F929F924A
:10D73000AF92BF92CF92DF92EF92FF920F931F931F
:10D74000CF93DF938091A00181FF03C060E075E07B
:10D7500002C060E074E090919D0184E69802C001EF
:10D760001124885A9D4FE091A301FF27E7FDF09512
:10D7700048EE53E0E49F9001E59F300DF49F300D9B
:10D78000112428533045AA24BB24A81AB90A281BFF
:10D79000390BFBE0EF2EF5E0FF2E40919A01440F8C
:10D7A000485F50E0440F551F440F551F4E52524FD3
:10D7B000E2EDFDE0CC24DD24C61AD70AA8E5B2E0EC
:10D7C000A81BB90B1CC0E701699079907E014B0141
:10D7D000661677060CF4430184018C149D040CF446
:10D7E0008601005A164FE501C01BD10B2C0F3D1FBF
:10D7F0000A0F1B1F11830083938382833496E417DF
:10D80000F50709F73183208393838283158214827D
:10D81000DF91CF911F910F91FF90EF90DF90CF900C
:10D82000BF90AF909F908F907F906F900895E09100
:10D830001201F09113018193F0931301E09312010F
:10D840000895FF920F931F93CF93DF93B9E0FB2EC0
:10D8500090E120E0C82FD0E08E01017010702017F9
:10D8600011F4905F07C0892F90E001970E94176C18
:10D87000202F90E1FA9431F0D595C795AE0140681C
:10D88000842FE8CF892F90E00F960E94176CDF91CC
:10D89000CF911F910F91FF9008951F93CF93DF9326
:10D8A000182F22ED3DE03093130120931201809157
:10D8B0001801877471F080919A01882319F08130E2
:10D8C00029F402C080E803C080E901C088E98093A0
:10D8D00018018091180187FF0BC086E190E00E943B
:10D8E000E969882329F4809118018F7780931801C2
:10D8F0008091180187FD5AC085E160E040E00E94F8
:10D900007E11882309F452C08091180180628093AF
:10D910001801809157018F5F80931901EAE1F1E0CE
:10D92000ABE0B5E080E01CC02D913D913595279589
:10D9300020503E4F37FD05C093E02F3F390724F4B8
:10D9400005C020E030E002C02FEF33E0932F93704A
:10D95000482F440F440F942B908321838F5F32967E
:10D96000811711F7C8E1D1E089910E94216C81E013
:10D97000C632D807C9F7809112019091130101971F
:10D9800090931301809312018FEF90E00E94176C27
:10D9900080E090E00E94176C82ED9DE0909317016B
:10D9A00080931601DF91CF911F9108958091180106
:10D9B0008F7DADCF1F920F920FB60F9211242F9330
:10D9C0008F939F93EF93FF9388B391E0892788BB50
:10D9D000E0911601F09117012191F0931701E09366
:10D9E0001601822F90E097BD86BD293C08F0C09AB1
:10D9F0008091620E81608093620EFF91EF919F9102
:10DA00008F912F910F900FBE0F901F9018951F921E
:10DA10000F920FB60F9211242F933F938F939F93E2
:10DA2000EF93FF9388B391E0892788BBE0911201BF
:10DA3000F0911301208130E020FD04C088B599B534
:10DA4000809603C088B599B5409699BD88BDC90137
:10DA500095958795009791F4CF01019690931301C6
:10DA6000809312018181882351F4809178009091F4
:10DA700079008053984F99BD88BD01C08083809103
:10DA8000620E81608093620EFF91EF919F918F9162
:10DA90003F912F910F900FBE0F901F901895EDE7BB
:10DAA000F0E08081857E808317981F9AAAE8B0E015
:10DAB0001C9210928B0082E88C938081806280831C
:10DAC0000895EDE7F0E080818F7D8083179AAAE8C2
:10DAD000B0E01C9210928B008AE08C938081886168
:10DAE000808308951F920F920FB60F9211248F9387
:10DAF0009F93AF93BF93EF93FF9380916E0E882314
:10DB000021F01F9A10926E0E04C01F9881E080933E
:10DB10006E0EA0911401B0911501FD0181919191BA
:10DB20009093870080938600F0931501E093140191
:10DB30008091650E9091660E90938500809384008D
:10DB400012968D919C911397009759F48AE19EE06B
:10DB500090931501809314018091A00181708093AE
:10DB60006E0E8091620E81608093620EFF91EF9144
:10DB7000BF91AF919F918F910F900FBE0F901F900B
:10DB80001895AF92BF92CF92DF92EF92FF920F93D0
:10DB90001F93CF93DF938091A00181FF03C040E0EA
:10DBA00055E002C040E054E0F0909A01FF0C80E1A3
:10DBB000F80E20919D0184E6280290011124285A34
:10DBC0003D4FE091A301FF27E7FDF09568EE73E07C
:10DBD000E69FC001E79F900DF69F900D112488539A
:10DBE0009045CC24DD24C21AD30A821B930B68EF24
:10DBF000E62EEF0CEAE1FEE000271127041B150BCF
:10DC000068E572E0621B730B21C0AE2DB0E0AA0F75
:10DC1000BB1FA55FBA4FAC901196BC90D5014A17B7
:10DC20005B070CF4DA01A017B1070CF4D801A05A75
:10DC3000B64FE601CA1BDB0B8C0F9D1F318320837F
:10DC4000A60FB71FB383A2833496E394EF14E8F2D0
:10DC50003183208393838283885E93409093660E02
:10DC60008093650E15821482DF91CF911F910F91E1
:10DC7000FF90EF90DF90CF90BF90AF9008951F92EC
:10DC80000F920FB60F9211242F933F934F935F93F0
:10DC90006F937F938F939F93AF93BF93EF93FF9374
:10DCA00078940E94C16DFF91EF91BF91AF919F91C8
:10DCB0008F917F916F915F914F913F912F910F9035
:10DCC0000FBE0F901F90189520916B0E30916C0E27
:10DCD00090E0822793279070880F991F8E57944E5B
:10DCE000FC0145915491232F33274227532750930A
:10DCF0006C0E40936B0E08959091670E96959695D5
:10DD0000982B9093670E8091680E8F5F8093680EBA
:10DD1000843068F0E091690EF0916A0E9193F0936F
:10DD20006A0EE093690E1092670E1092680E0895C5
:10DD300003C080E00E947C6E8091680E8823C9F742
:10DD4000E091690EF0916A0E10820895882339F0EF
:10DD500080916D0E8F5F80936D0E80E803C01092EE
:10DD60006D0E80EC0E947C6E80916D0E8530B8F750
:10DD700008950F931F93182F0E94646E08E0812F5F
:10DD800081700E94A66E16950150C9F71F910F91E0
:10DD9000089580EC0E947C6E80E80E947C6E80E892
:10DDA0000E947C6E80E80E947C6E80E80E947C6EFF
:10DDB00080E80E947C6E80E80E947C6E80EC0E946D
:10DDC0007C6E0895AF92BF92CF92DF92EF92FF9256
:10DDD0000F931F93CF93DF9382ED9DE090931301F8
:10DDE0008093120190936A0E8093690E10926C0ECC
:10DDF00010926B0E1092670E1092680E10926D0EBC
:10DE00000E94C96E80919A010E94B96E8091640E41
:10DE10000E94B96E80E00E94B96E1092640E0BE011
:10DE200015E054E0C52ED12CF80120813181C901C3
:10DE3000880F991F820F931FB6010E947F77EB0115
:10DE400022813381C901880F991F820F931FB60168
:10DE50000E947F7760507C4FC050DC4FF8E0C030AC
:10DE6000DF0710F0CFEFD7E07B0128E060307207CA
:10DE700020F0AFEFEA2EA7E0FA2E8C2F0E94B96EA9
:10DE80005E019B2D9F708E2D8295807F892B0E9435
:10DE9000B96EC701F4E096958795FA95E1F70E946F
:10DEA000B96E0C5F1F4F25E00B31120709F0BCCF94
:10DEB00000916C0E80916B0E0E94B96E802F0E94B3
:10DEC000B96E0E94C96E0E94986E80917800909100
:10DED0007900805C93469093790080937800C09A93
:10DEE000DF91CF911F910F91FF90EF90DF90CF9036
:10DEF000BF90AF900895809199019091630E98170B
:10DF000009F494C08093630E8130F9F0813030F0D1
:10DF10008230F1F1833009F089C05EC00E944F6DFC
:10DF20001EBC80E49CE99BBD8ABD1DBC1CBC87B7A0
:10DF3000837C87BF8CE386BF8FE380937C0087B7A9
:10DF4000806187BF1FBC8AE021C00E944F6D1EBC4C
:10DF50001DBC1CBC80E797E199BD88BD80EA9FE0AD
:10DF6000909379008093780087B7837C87BF8CE398
:10DF700086BF8FE380937C0087B7886087BF8091DE
:10DF80007D00816080937D001FBC82E08EBD4EC00D
:10DF90000E944F6D1EBC88EC90E0909379008093B6
:10DFA00078008CE291E09DBD8CBD80EE9BEA97BD30
:10DFB00086BD87B7837C87BF8CE386BF8FE3809362
:10DFC0007C0087B7806287BF80917D0081608093ED
:10DFD0007D001FBC8AE1DACF1EBC80E49CE99BBDBA
:10DFE0008ABD1DBC1CBC87B7837C87BF80917D0028
:10DFF0008E7F80937D008CE386BF8FE380937C00CF
:10E0000087B7806187BF1FBC8AE08EBD0E94C16D4B
:10E0100080E593EC909387008093860088E893E1F5
:10E0200090938500809384000E94616D8091990196
:10E03000813051F0813028F0823051F0833079F412
:10E040000CC00E94946B089578940E94E26E08952B
:10E05000789486E00E944D6C08950E94946B089518
:10E060001F920F920FB60F9211242F933F934F934D
:10E070005F936F937F938F939F93AF93BF93EF9330
:10E08000FF93809199018230C1F480E492EA97BDB8
:10E0900086BD80917800909179008F3F910538F48A
:10E0A00088E598E9909379008093780008C088EC1F
:10E0B00090E090937900809378000E947B6FFF91AD
:10E0C000EF91BF91AF919F918F917F916F915F91F0
:10E0D0004F913F912F910F900FBE0F901F90189569
:10E0E0001F920F920FB60F9211242F933F934F93CD
:10E0F0005F936F937F938F939F93AF93BF93EF93B0
:10E10000FF938CB59DB520916F0E222321F0C09A0C
:10E1100010926F0E04C0C09821E020936F0EA09162
:10E120002601B0912701FD01219131913BBD2ABD0E
:10E13000F0932701E09326012091AB063091AC06C5
:10E140002817390720F49093AC068093AB062091F2
:10E150000C0130910D018217930720F490930D016B
:10E1600080930C0112968D919C9113970097D9F48E
:10E1700082ED9DE090932701809326018091A0017C
:10E180008095817080936F0E87B78F7E87BF0E94C6
:10E190007B6F80919901882311F0833021F487B738
:10E1A000806187BF78948091620E81608093620E57
:10E1B000FF91EF91BF91AF919F918F917F916F915F
:10E1C0005F914F913F912F910F900FBE0F901F9035
:10E1D000189590916D019873903121F463E00E943D
:10E1E0005F770895983111F486950895983211F467
:10E1F000880F0895903319F4982F990F890F089577
:10E20000FC01A5E6B0E08C918B7F8C931482158283
:10E210001082118216A617A608950E940071089513
:10E2200021E0FC018481882309F420E0822F0895F5
:10E23000FC0181819081891B877098E0981B81E0A7
:10E24000933008F480E00895FC0184818823F9F07C
:10E250008150848382819381890F828386A588235C
:10E2600009F44CC087A5982F915097A7882331F0C7
:10E2700080916500846080936500089580916500B9
:10E280008B7F809365008091780187A708951B9804
:10E29000809165008B7F809365008581882319F0CC
:10E2A00081508583089580819181891739F190E0AB
:10E2B000DF01A80FB91F16962C9116972283569648
:10E2C0002C91569724831E962C911E9723835E963D
:10E2D0002C915E972583D0962C91D09726A717A6D0
:10E2E00096962C919697322F315096963C9396970E
:10E2F000222321F4019687709070808308958F9275
:10E300009F92AF92BF92CF92EF92FF920F931F9383
:10E31000DF93CF9300D0CDB7DEB74C01122F4A83E5
:10E3200069830E9418714A816981882331F1809143
:10E330006D01887311F1F401A180BB24C501019620
:10E3400097E0F92EF8228081F816B9F0662329F0BB
:10E3500080917701865F860F01C080E0A80CB91C10
:10E36000F5018683842F0E94E970F501868B168F54
:10E37000E0AA06A3C686F401F1820F900F90CF9118
:10E38000DF911F910F91FF90EF90CF90BF90AF90D2
:10E390009F908F900895AF92BF92CF92EF920F937C
:10E3A000DF93CF9300D00F92CDB7DEB75C012B8304
:10E3B0004A8369830E9418712B814A81698188236D
:10E3C00029F180916D01887309F1662329F080910C
:10E3D0007701865F860F01C080E0F5018283842F7C
:10E3E0002B834A8369830E94E970F50184832B8122
:10E3F0002583E6A617A6C382808181834A8169812D
:10E40000002321F00150C5010E947F710F900F90F1
:10E410000F90CF91DF910F91EF90CF90BF90AF9081
:10E420000895CF92EF920F93CF93DF93EC018091F9
:10E430006D01869586958695877028819981291723
:10E4400009F05CC1E62FF0E0E132F10508F056C1B9
:10E45000EA5BFF4FEE0FFF1F0590F491E02D09944A
:10E46000CE0166E44AE0DEC0CE0166E444E1DAC0F3
:10E47000CE0166E44EE1D6C0CE0164E64AE022E079
:10E4800002E0EE24E39452E0C52E36C1CE016FE5E2
:10E4900045E022E00AE0EE24E394CC240E947F7160
:10E4A000CE016FE545E02AE001E00E947F71CE01D8
:10E4B0006FE545E022E00AE01FC1CE0160E54AE0D9
:10E4C00023E002E0EE24CC24CA940E947F71CE01A6
:10E4D0006CE34AE023E0CC24C3940E947F71CE0118
:10E4E00066E44AE021E000E032E0E32E96C0CE018F
:10E4F00066E445E021E001E0EE24E394CC240E94B0
:10E500007F71CE0162E34FE022E00E947F71CE0175
:10E5100060E54FE022E0F0C0CE016EE645E021E08C
:10E5200002E0EE24E394CC240E947F71CE016CE7DC
:10E5300045E021E02AC0CE0162E345E025E000E0AD
:10E54000EE24CC240E947F71CE016AE545E025E0EF
:10E550000E947F71CE016EE643E024E002E0CCC071
:10E56000CE0160E545E02AE003E0EE24E394CC240C
:10E570000E947F71CE0160E545E024E101E00E9448
:10E580007F71CE0160E545E02AE003E0B5C0CE0131
:10E590006AE044E125E002E0EE24E394CC24C39455
:10E5A000ABC0CE0162E344E02AE002E0EE24E39453
:10E5B000CC240E947F71CE0166E448E024E101E0B2
:10E5C0000E947F71CE0162E348E02AE002E00E94EF
:10E5D0007F71CE0166E444E024E101E08DC0CE010C
:10E5E00068E745E02AE00AE016C0CE0168E745E0AA
:10E5F00022E30AC0CE0160E044E12AE001E00BC062
:10E60000CE0160E044E12AE002E005C0CE0160E016
:10E6100044E12AE003E0EE24E394CC246DC0CE0173
:10E6200066E448E221E000E048C0813009F466C0B9
:10E63000CE016BE405C0813009F460C0CE0161E415
:10E640004AE021E000E041C0CE01642F46E0F9CF6E
:10E65000CE0166E44AE022E0E6CF813009F44EC004
:10E66000CE0166E44AE022E0EDCFCE0168E7E8CFD4
:10E67000CE0168E74AE021E01FC0CE016AE74AE028
:10E6800021E00FC0CE016CE74AE021E004C0CE01DA
:10E6900068E74FE023E003E010C0CE0168E74FE0F9
:10E6A00023E002E00AC0CE0168E74FE023E004C0A7
:10E6B000CE0166E444E129E101E0EE24E39406C0E2
:10E6C000CE0166E44AE022E002E0EE24CC240E947F
:10E6D000CB7114C0CE016CE344E123E002E0EE24F0
:10E6E000CC24C3940E947F71CE0160E544E123E015
:10E6F000EE24E394CC24CA940E947F71DF91CF91E1
:10E700000F91EF90CF900895682F8FE294E046E448
:10E710000E941172089590919601987109F06AC053
:10E720009091C70E992321F48E3509F076C002C06E
:10E730008E3511F481E019C08D3521F481E080938C
:10E74000C80E08952091C80E222321F01092C80E01
:10E7500020E68227913021F48093C90E82E005C023
:10E76000923031F48093CA0E83E08093C70E0895EF
:10E770004091C90E4932D8F5382F20E08091CA0E59
:10E78000B901680F711DE42FF0E0EE0FFF1FE55394
:10E79000F14F71836083413149F420911D0F30E0C6
:10E7A0002617370724F560931D0F21C04630F9F472
:10E7B0008091D70E9091D80E592F52955F70E52F0A
:10E7C000F0E020912A0F30E0E217F3074CF0E5303B
:10E7D000F1051CF040932A0F03C05F5F50932A0F8E
:10E7E000E25EF04F6AE070E00E947F7760831092F3
:10E7F000C70E0895983089F49091990E923318F4C9
:10E800008093CA0E0895382F20E08091CA0E280FF9
:10E81000311D3093EC0E2093EB0E08951F920F9252
:10E820000FB60F9211242F938F939F93EF93FF9323
:10E830008091960E882379F090912B0FE92FF0E0CC
:10E84000ED57F14F20812CB99F5F90932B0F815092
:10E850008093960E01C05598FF91EF919F918F91F3
:10E860002F910F900FBE0F901F90189510922B0FA5
:10E87000559A0895CF92DF92EF92FF920F931F93D4
:10E88000CF93DF9390E09C01220F331F220F331FA1
:10E89000D901A85DBB4F40E050E0C62EDD24F90150
:10E8A000E65DFB4F89010556114FC416D50611F0E0
:10E8B000623020F18081282F2F7030E07A01EE0C39
:10E8C000FF1C02C035952795EA94E2F7237030705B
:10E8D0002115310599F0E801E8807C9182958370DB
:10E8E00090E0042E02C0959587950A94E2F780FF88
:10E8F00003C07E1518F40AC0E71640F04F5F5F4F63
:10E9000011964230510589F620E030E0C901DF91CF
:10E91000CF911F910F91FF90EF90DF90CF900895CE
:10E92000E82FF0E0EE0FFF1FEE0FFF1FE65DFB4F3D
:10E9300080818F70909179019150923038F590914B
:10E94000700197FF23C090E0660F02C095958795F0
:10E950006A95E2F78370823039F0833079F0813044
:10E96000A9F46091750103C06091750162956F70A3
:10E970008FE294E046E40E9411720895609176015E
:10E980006F708FE294E046E40E9411720895109235
:10E99000960E8AB188628AB90895549A579A089552
:10E9A000FC016E3721F06D3761F46DE501C06EE555
:10E9B0008081A82FB0E0AD57B14F9DE79C938F5F4A
:10E9C00080838081A82FB0E0AD57B14F6C938F5FEB
:10E9D000808308951F93DF93CF9300D00F92CDB71C
:10E9E000DEB71EE71093830E8093840E82E0898346
:10E9F000CE0101962B834A830E94D0748981A82F6F
:10EA0000B0E0AD57B14FFD014A8141932B81119682
:10EA10002C93DF0111961182FD01319611961C9203
:10EA2000DF0111961182FD01319611961C9211970A
:10EA300011821283885F8093960E0F900F900F9033
:10EA4000CF91DF911F910895FC0180818383108213
:10EA50000895FC018381861710F4681B01C060E0F3
:10EA600060838281861708F462838181882311F094
:10EA7000681708F461830895FF920F931F93CF9353
:10EA8000DF93EC0188818D3F40F4893F60F4863F3D
:10EA9000D1F1873F09F04DC02FC08D3FD9F18E3F96
:10EAA00009F047C013C090E0895F9040FC01EE0F71
:10EAB000FF1FE80FF91FE554F14F898182838A8196
:10EAC000817081838B818370808333C08BE99EE06A
:10EAD00069810E9429758FE99EE06A810E942975EB
:10EAE00083EA9EE06B810E9429756C81669587EAB6
:10EAF0009EE00E9429751DC089818093B80E8B818C
:10EB00008093BA0E16C089818093B70E8B81809353
:10EB1000B90E0FC009810D5F239613E0BCE3FB2EF5
:10EB200006C089910E948B73F092990E1F5F101797
:10EB3000C0F31092970E84E18093980EDF91CF91ED
:10EB40001F910F91FF9008951F920F920FB60F9291
:10EB500011242F933F934F935F936F937F938F93E2
:10EB60009F93AF93BF93EF93FF93579878949BB184
:10EB70008CB19C7129F01092970E1092300F4BC0FF
:10EB80009091970E992309F046C090912F0F9130E4
:10EB900039F09130C8F1923079F09330E1F524C02A
:10EBA0008E37C9F19091300F933160F5E92FF0E085
:10EBB000E059F14F808323C08D3711F483E029C0E1
:10EBC0008E3739F480E79EE00E943C7510922F0F3B
:10EBD00022C09091300FE92FF0E0E059F14F80838F
:10EBE0009F5F9093300F17C09091300F933150F486
:10EBF000E92FF0E0E059F14F20E2282720839F5FC2
:10EC00009093300F82E005C08E3729F41092300FB8
:10EC100081E080932F0FF894579AFF91EF91BF9165
:10EC2000AF919F918F917F916F915F914F913F91A4
:10EC30002F910F900FBE0F901F90189580E1EBE978
:10EC4000FEE0DF011D928A95E9F71092B00E109256
:10EC5000AF0E1092B60E1092B50E08958CE0EBEB4D
:10EC6000FEE0DF011D928A95E9F70E941E7610985A
:10EC700018981092900087E689B959981AB886E0DA
:10EC80008093950001C08CB15F99FDCF0E94C7743D
:10EC90000E94CD740895FC0182819381860F911D9D
:10ECA00093838283208131812817390748F4821B9E
:10ECB000930B9383828384819581019695838483CA
:10ECC00008958091980E882319F081508093980EB2
:10ECD0008091990E882319F081508093990E90911C
:10ECE0002C0F992309F471C080912D0F882321F0F6
:10ECF000815080932D0F69C08091960E882309F072
:10ED000064C0E0E081E0282F292321F4EF5F880F21
:10ED1000E730C9F78095892380932C0FE430C0F544
:10ED20008E2F87509E2F969521E0291B30E0F0E032
:10ED3000E095F095E170F070D901AA0FBB1FAA0F02
:10ED4000BB1FAE0FBF1FA85DBB4F6C91D901AA0FAF
:10ED5000BB1FAA0FBB1FA65DBB4F2C91422F429534
:10ED6000437050E00E2E02C0559547950A94E2F785
:10ED700041709091700197FD20C02F7030E0EE0F30
:10ED8000FF1F02C035952795EA95E2F7237016C05C
:10ED9000E63070F48E2F8170E82FF0E0DF01A95487
:10EDA000B14FE754F14F8A506C9140E0208106C08A
:10EDB000E63059F481EF60E040E020E00E94EA7420
:10EDC00085E080932D0F0E94367480912A048295ED
:10EDD000869586958370833031F48BEA9EE060914E
:10EDE0009B0E0E944B7680912E0482958695869587
:10EDF0008370833031F481EB9EE060919F0E0E941E
:10EE00004B7680912801815080932801882331F42A
:10EE100088EC8093280181E080939A0E0895EF9208
:10EE2000FF920F931F9310922A0F80912C0F8F60E7
:10EE300080932C0F2091270430E040E050E060E404
:10EE4000E62E6EE7F62E65E0062F112DC801B701FC
:10EE50000E94B4773093AC0E2093AB0E20912B041C
:10EE600030E040E050E0C801B7010E94B477309331
:10EE7000B20E2093B10E1F910F91FF90EF90089565
:10EE8000629FD001739FF001829FE00DF11D649F8E
:10EE9000E00DF11D929FF00D839FF00D749FF00D1A
:10EEA000659FF00D9927729FB00DE11DF91F639FBB
:10EEB000B00DE11DF91FBD01CF0111240895991B6B
:10EEC00079E004C0991F961708F0961B881F7A9561
:10EED000C9F780950895AA1BBB1B51E107C0AA1F63
:10EEE000BB1FA617B70710F0A61BB70B881F991FEB
:10EEF0005A95A9F780959095BC01CD01089597FB8F
:10EF0000092E07260AD077FD04D0E5DF06D00020C1
:10EF10001AF4709561957F4F0895F6F79095819555
:10EF20009F4F0895A1E21A2EAA1BBB1BFD010DC025
:10EF3000AA1FBB1FEE1FFF1FA217B307E407F507A9
:10EF400020F0A21BB30BE40BF50B661F771F881F85
:10EF5000991F1A9469F760957095809590959B011B
:10EF6000AC01BD01CF01089597FB092E05260ED0F7
:10EF700057FD04D0D7DF0AD0001C38F450954095D7
:10EF8000309521953F4F4F4F5F4F0895F6F790957D
:10EF90008095709561957F4F8F4F9F4F0895EE0F2D
:10EFA000FF1F0590F491E02D0994FB01DC01415015
:10EFB000504048F005900D920020C9F701C01D9205
:10EFC00041505040E0F708956817790768F4FB0155
:10EFD000DC01E40FF51FA40FB51F02C002900E92D2
:10EFE00041505040D8F708950C940D78DC0101C0D1
:10EFF0006D9341505040E0F70895DC01CB01FC01D6
:10F00000E199FECF06C0FFBBEEBBE09A31960DB290
:10F010000D9241505040B8F70895FB01DC0102C049
:10F0200001900D9241505040D8F70895F894FFCFC9
:10F030006C036D036E036F034AF0004DFF0722045B
:10F040007C5ED20D1A0ED20DFF0000AA05FF09FF4B
:0AF050000DFF135414AAD20DC800DE
:00000001FF
